:020000040800F2
:1080000010BE0020498100084D9A0008A594000880
:1080100035990008DB8F0008FBAF00080000000066
:1080200000000000000000000000000019A500088A
:10803000F390000800000000059F000895A50008C7
:108040006381000863810008638100086381000880
:108050006381000863810008638100086381000870
:108060006381000863810008638100086381000860
:108070006381000863810008638100086381000850
:108080006381000863810008638100086381000840
:1080900077A7000863810008638100080792000841
:1080A0006381000863810008638100086381000820
:1080B0000DA60008B5A6000861A7000863810008A6
:1080C0006381000863810008638100086381000800
:1080D00063810008638100086381000863810008F0
:1080E00063810008638100086381000863810008E0
:1080F00063810008638100086381000863810008D0
:1081000063810008638100086381000863810008BF
:1081100063810008638100086381000863810008AF
:10812000638100086381000863810008638100089F
:10813000DFF810D000F074F800480047D1F90008CB
:10814000AFF3008010BE0020064880470648004775
:10815000FEE7FEE7FEE7FEE7FEE7FEE7FEE7FEE7F7
:10816000FEE7FEE79DA50008318100080649074AA1
:108170000868504343F239021044086040087047D1
:108180000149086070470000EC0500206D4EC641B3
:1081900010B5431A934209D28318881803E010F8E7
:1081A000011D03F8011D521EF9D210BD40EA010362
:1081B0009B0703D009E008C9121F08C0042AFAD29D
:1081C00003E011F8013B00F8013B521EF9D210BD4B
:1081D000D2B201E000F8012B491EFBD27047002209
:1081E000F6E710B513460A4604461946FFF7F0FFB6
:1081F000204610BD30B504460020034600E05B1C5D
:10820000934203D2E05CCD5C401BF8D030BD034606
:1082100011F8012B00F8012B002AF9D118467047FC
:10822000064C074D06E0E06840F0010394E80700C3
:1082300098471034AC42F6D3FFF77EFFB4540108E0
:10824000D454010870B58C1810F8015B15F00703C1
:1082500001D110F8013B2A1106D110F8012B03E0DF
:1082600010F8016B01F8016B5B1EF9D12B0705D4E7
:108270000023521E0DD401F8013BFAE710F8013B30
:10828000CB1A921C03E013F8015B01F8015B521E4C
:10829000F9D5A142D8D3002070BD00002DE9F041EE
:1082A00007460C4615461E461EB980200B4908603D
:1082B00003E04FF4807009490860102229462046E7
:1082C00005F0B8FE8046102241463846FFF760FFB1
:1082D000404606F03FFBBDE8F0810000A405002009
:1082E0002DE9F04784B01F46DDF830A0914688465E
:1082F000060018BFB8F1000F4AD0002F18BFBAF11E
:10830000000F45D0B9F1000FA8BF19F00F0F1EBF25
:1083100040F61D4004B0BDE8F087307910F0020F40
:108320001EBF40F61E4004B0BDE8F0870024B9F13E
:10833000100FA8BF6D4625DB5FF0000004EB800145
:1083400058F8011009BA45F82010401C0428F5DB44
:108350006846014606F12802736A00F0BFF84FF044
:10836000000C00BF55F82C0004EB8C0100BA0CF196
:10837000010C7850BCF1040FF4DB04F12000103440
:108380004845D9DDCAF8004004B00020BDE8F087B8
:1083900004B04FF44260BDE8F087002812BF002A05
:1083A0004FF442607047017941F0020101710020F1
:1083B00010607047032300F04BBD00002DE9F0472B
:1083C00084B01F46DDF830A091468846060018BFED
:1083D000B8F1000F4AD0002F18BFBAF1000F45D0F6
:1083E000B9F1000FA8BF19F00F0F1EBF40F61D40D6
:1083F00004B0BDE8F087307910F0020F1EBF40F6E0
:108400001E4004B0BDE8F0870024B9F1100FA8BFEA
:108410006D4625DB5FF0000004EB800158F8011089
:1084200009BA45F82010401C0428F5DB68460146CF
:1084300006F12802736A00F0DFF94FF0000C00BF6C
:1084400055F82C0004EB8C0100BA0CF1010C7850AB
:10845000BCF1040FF4DB04F1200010344845D9DDF1
:10846000CAF8004004B00020BDE8F08704B04FF423
:108470004260BDE8F087002812BF002A4FF4426036
:108480007047017941F002010171002010607047CE
:10849000022300F0DDBC00002DE9F04180460C46CF
:1084A00015461E4600271EB980200B49086003E0D0
:1084B0004FF48070084908602946404606F02CF8C1
:1084C0000746102239462046FFF762FE384606F07E
:1084D00041FABDE8F0810000A40500202DE9F80F65
:1084E0004FF0030C0CEBE308DB1002EB431202F13C
:1084F0006003BE4A4FF0010CC2F808C0D2F808C0B1
:10850000D2F800C0CDF800C0BCF1FF3F08D1DDF8C3
:1085100000C0C2F800C012680092002A00F0E68095
:108520004268D3F804C0006882EA0C071A68424027
:1085300094466446AE483D0E02F0FF0A50F82560AE
:10854000C4F3074550F82AA050F8255004F0FF0B5B
:1085500086EA3526C2F3072550F82BB050F825508F
:10856000A8F101084FEA35490CF0FF0550F82550F5
:1085700089EA3565754053F8106CC7F307496E40BA
:108580004FEA1C6550F8299050F8255085EA3925A6
:10859000C4F30729240E50F8299050F824404FEADC
:1085A000394989EA3A6985EA090953F80C5CCCF340
:1085B000074A89EA05054FEA1269C2F30742CCF37C
:1085C000072C50F8299050F82AA050F8222050F893
:1085D0002CC089EA3A2984EA3222C7F3072A4FEAF3
:1085E0003C4407F0FF0C50F82AA050F82CC04FEA8A
:1085F0003A4A8AEA3B6A84EA3C6C89EA0A0982EAD6
:108600000C0253F808AC53F804CC203B89EA0A0961
:1086100082EA0C04B8F1000F7ADD320EC4F3074C85
:1086200050F8222050F82CC0EFB282EA3C22C9F365
:10863000072C50F8277050F82CC009F0FF0A4FEAB9
:108640003C4C8CEA376C82EA0C02D3F800C050F83C
:108650002AA082EA0C072A0E04F0FF0B50F822C071
:10866000C6F3074250F82BB050F822208CEA322C87
:10867000C4F30722240E50F8222050F824404FEA79
:10868000324282EA3A628CEA0202D3F804C0C5F3AD
:10869000074A82EA0C0C4FEA196250F82AA050F8F7
:1086A0002220C5F3072582EA3A22C6F3072AC9F336
:1086B0000749F6B250F82AA050F8255050F82990F2
:1086C00050F826604FEA3A4A4FEA35458AEA3B6A53
:1086D00084EA392485EA366582EA0A026C40D3F8D6
:1086E00008A0DD6882EA0A026C4024E70268D3F839
:1086F00000C09C6882EA0C074268D3F804C082EA92
:108700000C0C8268C0686240DC68444012E7FFE7F6
:10871000384850FA85F200EB166C12789CF800C0CD
:10872000C9F3072742EA0C62C4F3074CC75D10F88F
:108730000CC04FEA0C4C4CEA072C42EA0C02D3F86E
:1087400000C082EA0C020A6050FA89F200EB156C54
:1087500012789CF800C0C4F3072742EA0C62C6F303
:10876000074CC75D10F80CC04FEA0C4C4CEA072CC4
:1087700042EA0C02D3F804C082EA0C024A6050FAC2
:1087800084F200EB196C12789CF800C0C6F307273E
:1087900042EA0C62C5F3074CC75D10F80CC04FEA03
:1087A0000C4C4CEA072C42EA0C02D3F808C082EACF
:1087B0000C028A6050FA86F200EB146C12789CF876
:1087C00000C0C5F3072442EA0C62C9F3074C10F855
:1087D0000CC0005D4FEA0C4C4CEA00201043DA68F4
:1087E0005040C860BDE8F80F7047000000300240FC
:1087F0002C3F0108043A01082DE9F80F4FF0030C53
:108800000CEBE308C24B4FF0010CC3F808C0D3F8DF
:1088100008C0D3F800C0CDF800C0BCF1FF3F00F0A5
:10882000E5804368D2F804C0006883EA0C07136847
:1088300080EA0304A4466346B6483D0ECCF30746DF
:1088400050F8255050F8266004F0FF0985EA3625D7
:10885000C3F3072650F8299050F8266007F0FF0A66
:108860004FEA364686EA396675401669C3F307490A
:108870006E404FEA1C6550F8299050F8255050F88A
:108880002AA085EA3925C4F307290CF0FF0B50F81C
:108890002990CCF3072C4FEA394989EA3A6985EAED
:1088A0000905D2F81490C4F3074A85EA09054FEA8E
:1088B000136950F82AA050F82990240E89EA3A2921
:1088C000C7F3072AC7F30747DBB250F82AA050F8CE
:1088D0002CC050F82BB050F8244050F8277050F8B6
:1088E00023304FEA3A4A4FEA3C4C8AEA3B6A84EA30
:1088F00037248CEA336389EA0A0984EA030CD2F844
:1089000018A0D3692032A8F1010889EA0A098CEA83
:108910000304B8F1000F7CDD330EC5F3074C50F8AB
:10892000233050F82CC0E7B283EA3C23C9F3072C6C
:1089300050F8277050F82CC006F0FF0A4FEA3C4C64
:108940008CEA376C83EA0C03D2F800C050F82AA0F6
:1089500083EA0C072B0EC9F3074C50F8233050F86C
:108960002CC005F0FF0B83EA3C23C4F3072CC5F3AE
:10897000072550F82CC050F825504FEA3C4C8CEAA3
:108980003A6C83EA0C03D2F804C0C4F3074A83EAC2
:108990000C0C4FEA196350F82AA050F82330240E2B
:1089A00083EA3A23C6F3072AC6F3074650F8244061
:1089B00050F8266050F82AA084EA362409F0FF0611
:1089C00050F82BB050F826604FEA3A4A4FEA354546
:1089D0008AEA3B6A85EA366583EA0A036C40D2F884
:1089E00008A0D56883EA0A036C4026E7DDF800C0DA
:1089F000C3F800C01B68009363B14368D2F804C099
:108A0000006883EA0C07136880EA030C6346644637
:108A100012E710E00368D2F800C0946883EA0C07FC
:108A20004368D2F804C083EA0C0C8368C0686340D2
:108A3000D468444000E7384850FA84F300EB166CE1
:108A40001B789CF800C0C9F3072743EA0C63C5F301
:108A5000074CC75D10F80CC04FEA0C4C4CEA072CD1
:108A600043EA0C03D2F800C083EA0C030B6050FA0F
:108A700086F300EB156C1B789CF800C0C4F3072745
:108A800043EA0C63C9F3074CC75D10F80CC04FEA0A
:108A90000C4C4CEA072C43EA0C03D2F804C083EADE
:108AA0000C034B6050FA85F300EB196C1B789CF8B3
:108AB00000C0C6F3072743EA0C63C4F3074CC75D45
:108AC00010F80CC04FEA0C4C4CEA072C43EA0C039C
:108AD000D2F808C083EA0C038B6050FA89F300EBEC
:108AE000146C1B789CF800C0C5F3072443EA0C63A0
:108AF000C6F3074CD26810F80CC0005D4FEA0C4C6E
:108B00004CEA002018435040C860BDE8F80F704799
:108B1000003002402C3B01080439010870B50C46B6
:108B20008446002315462046B3EBA20F09DA00BFA6
:108B30005CF8231009BA40F823105B1CB3EBA20FBA
:108B4000F6DB214600F096F8E910052000EB410322
:108B5000002BD8BF70BD04F11002454800F5C56177
:108B6000D2F800C000EB1C64CCF307452478455DC7
:108B700051F8244051F8255084EA3524CCF30725D8
:108B8000455D51F825504FEA354550FA8CFC9CF86C
:108B900000C051F82CC085EA3C6C84EA0C0C42F809
:108BA00004CB52F804CB00EB1C64CCF307452478CB
:108BB000455D51F8244051F8255084EA3524CCF322
:108BC0000725455D51F825504FEA354550FA8CFC94
:108BD0009CF800C051F82CC085EA3C6C84EA0C0C6F
:108BE00042F804CC52F808CB00EB1C64CCF30745E8
:108BF0002478455D51F8244051F8255084EA352405
:108C0000CCF30725455D51F825504FEA354550FA1C
:108C10008CFC9CF800C051F82CC085EA3C6C84EABE
:108C20000C0C42F808CC52F804CC00EB1C64CCF3DA
:108C300007452478455D51F8244051F8255084EAD1
:108C40003524CCF30725455D51F825504FEA3545CD
:108C500050FA8CFC9CF800C05B1E51F82CC085EAD1
:108C60003C6C84EA0C0C42F804CC7FF479AF70BD04
:108C70000439010870B400239510002D15DDA0F112
:108C8000040C081F12F0040F03D05CF8044F40F8E6
:108C9000044FD21009D000BFDCF8044044605CF8F7
:108CA000084F40F8084F521EF6D1684C042DA4F529
:108CB000007005D0062D34D0082D6DD070BC7047E3
:108CC000CA6800EB126CC2F307459CF800C0455D12
:108CD0004CEA056CC2F30725455D2D0450FA82F677
:108CE000367845EA06254CEA050C54F823600D68F1
:108CF0005B1C75408CEA050CC1F810C04D680A2B4E
:108D00008CEA050CC1F814C08D688CEA050C8CEA5D
:108D10000202C1F818C0CA61B8BF1031D0DB70BC04
:108D200070474A6900EB126CC2F307459CF800C01B
:108D3000455D4CEA056CC2F30725455D2D0450FAEC
:108D400082F6367845EA06254CEA050C54F823608D
:108D50000D685B1C75408CEA050CC1F818C04D68A5
:108D6000082B8CEA050CC1F81CC08D688CEA050C38
:108D7000C1F820C0CD688CEA050CC1F824C0A4BF9E
:108D800070BC70470D698CEA050C8CEA0202C1F8D0
:108D900028C0CA621831C4E7CA6900EB126CC2F37A
:108DA00007459CF800C0455D4CEA056CC2F30725F9
:108DB000455D2D0450FA82F6367845EA06254CEAE0
:108DC000050C54F823600D685B1C75408CEA050C9B
:108DD000C1F820C04D68072B8CEA050CC1F824C0EF
:108DE0008D688CEA050CC1F828C0CD688CEA050CAA
:108DF000C1F82CC0A4BF70BC704750FA8CF52D7818
:108E000000EB1C66367845EA0665CCF30746CCF3E2
:108E1000072C865D10F80CC0360446EA0C2C45EA97
:108E20000C0C0D698CEA050CC1F830C04D698CEA58
:108E3000050CC1F834C08D698CEA050C8CEA02027D
:108E4000C1F838C0CA632031A6E70000043B01081E
:108E50002DE9F0410E46002818BF002E04D003F083
:108E600006012AB9022903D04FF44260BDE8F0811F
:108E7000D0F824C0BCF1100F1CBFBCF1180FBCF11E
:108E8000200F08D102290AD0D0F810C0ACF1010C93
:108E9000BCF1100F03D340F61F40BDE8F081C26063
:108EA00090F804C002292CF0060C80F804C048D0C9
:108EB000002141618161C1610162D0F810C0BCF143
:108EC000000F3EDD1CF0010F4FF01804A2F101026B
:108ED00004D012F8011F0906416101215FEA6C0C00
:108EE0002FD0CF1701EB977727F00307CF1B5578CB
:108EF0007F4204EBC70705FA07F721F00305054495
:108F0000D5F8148047EA08076F614D1C4FEAE578F1
:108F100005EB987828F00308A5EB080512F8027F06
:108F20006D4204EBC505AF404D1C25F0030505441B
:108F3000891CD5F81480BCF1010C47EA08076F6161
:108F4000CFD1017911F0010F0DD113F0010F86601F
:108F50001CBF062131EA030108D000F12801426A52
:108F60003046FFF7DBFD0020BDE8F08100F128016D
:108F7000426A0020B0EBA20F09DA00BF56F8203099
:108F80001BBA41F82030401CB0EBA20FF6DB0846BC
:108F9000FFF770FEE7E7000030B50246130100203E
:108FA00013E000210EE00A4C1C4404EB8004645CD6
:108FB000084D05EB81052D5C6C40064D05EB8105E8
:108FC0002C54491C0429EEDB401C0428E9DB30BD8D
:108FD0000C980020FC970020704700BFFEE772B697
:108FE0007047000070B5002600240DE0002508E061
:108FF00005EB84001C49085C1C4901EB8501085500
:109000006D1C042DF4DB641C042CEFDB0020FFF747
:10901000C3FF012609E001F0A3FA01F07FFA00F096
:109020008BFC3046FFF7B8FF761C1148006886427B
:10903000F1DB01F095FA01F071FA0D480068FFF7D5
:10904000ABFF00240DE0002508E0084800EB850098
:10905000005D05EB8401074A50546D1C042DF4DBC0
:10906000641C042CEFDB70BDCC970020FC97002023
:109070009C050020DC970020024600210AE00F4BEF
:1090800013F81100904203D14800401C185C70474F
:10909000481CC1B21229F2DB00210AE04800401C42
:1090A000064B185C904202D113F81100EFE7481C00
:1090B000C1B21229F2DB0020E9E70000A235010865
:1090C00030B591B004460D46402101A8FFF787F85E
:1090D00094208DF804000B208DF805002A462146C7
:1090E0000DF10600FFF754F801A809F0F3FE11B0E6
:1090F00030BD7047FEB506460C4617461D46022D8C
:1091000001D1012500E000250A484078012809D155
:1091100002A823463A461021CDE90005304601F069
:1091200087F905E02B463A4631462046FFF7B6F868
:10913000FEBD0000D44E002010B504460A2002F007
:10914000A1F910BD2DE9F04104460E46174606F080
:1091500007F8A02005F0A4FFC4F3072005F0A0FF46
:10916000E0B205F09DFF05F0FBFFA12005F098FFA0
:10917000002504E005F052FF7055681CC5B2BD42E1
:10918000F8DB06F011F80120BDE8F0812DE9F04789
:10919000054689461646002400BF281900F01F0026
:1091A000C0F120008046311B884203DB301B00F0F9
:1091B000FF0800E000BF05F0D3FFA02005F070FF1E
:1091C0002919C1F3072005F06BFF2919C8B205F072
:1091D00067FF002706E0E11919F8010005F060FFBC
:1091E000781CC7B24745F6DB05F0DEFF0A2004F025
:1091F000B7FB04EB0800C4B2B44200DB00E0CCE7EC
:1092000000BFBDE8F08710B5802005F02BFA28B12B
:10921000032008F00BF9802005F01EFA10BD0000B5
:10922000FEB506460D4617461C46022C01D1012408
:1092300000E000240A484078012809D102A82B4602
:109240003A461021CDE90004304601F02BF905E043
:1092500023463A4629463046FFF71EF9FEBD000078
:10926000D44E002000B587B072211F4805F00CFED7
:1092700040F207111D4805F007FE4FF440711C48ED
:1092800005F002FE72200190102002900020039051
:109290000420049001A9144800F045F840F207109A
:1092A000019010200290002003900420049001A956
:1092B0000E4800F038F88020019004200290002031
:1092C000039001A9084800F02EF84FF44070019077
:1092D00010200290002003900420049001A904486B
:1092E00000F021F807B000BD001001400008014067
:1092F000000C014070B504460D462A46214602483E
:1093000004F0CEFD70BD0000F805002000B5014658
:1093100000F026F8024600BF00F022F8801A8842CA
:1093200000D300BDF8E770B505460C462846D4E9E1
:109330000031E26805F004FE70BD70B504460D46CC
:109340002946204605F05AFE012804D12946204628
:1093500005F09AFD03E02946204605F097FD70BD13
:10936000014800687047000034030020024800688C
:10937000401C0149086070473403002000B587B0E5
:1093800040F2026007F078FE40F2046007F074FEDD
:109390004FF4C06007F070FE40F20C6007F06CFE06
:1093A0004023032210211F4805F0CAFDA0230322F9
:1093B00018211D4805F0C4FD4023032204211A484A
:1093C00005F0BEFD802303220421164805F0B8FDF8
:1093D000002001904FF482700090002002900590D0
:1093E0004FF400700390102006900020049069460E
:1093F0000E4808F014FB0D4808F0FEFA0022032185
:10940000172007F049F80721022005F04DFD012241
:109410000021802005F0C4F8802005F01DF907B078
:1094200000BD000000100140000801400030014074
:109430002DE9F04104460D4616464FF0000800277E
:109440000AE02A466D1C14F8011B064800F00CF8CF
:1094500040EA0808781C87B2B742F2DB0020BDE87A
:10946000F08100000030014070B506460D461446FC
:1094700000BF02210A4808F0CAFA0028F9D029469C
:10948000074808F0C2FA00BF0121054808F0BFFAFA
:109490000028F9D0024808F0B4FA2070207870BD96
:1094A0000030014000BFFEE770B5002600240DE04B
:1094B000002508E005EB84001C49085C1C4901EB11
:1094C000850108556D1C042DF4DB641C042CEFDBB6
:1094D00018480068FFF760FD16480068461E09E05E
:1094E00000F040F900F05EF93046FFF755FD00F05E
:1094F00025F8761E002EF3DC00F034F900F052F966
:109500000020FFF749FD00240DE0002508E0084891
:1095100000EB8500005D084901EB840148556D1C96
:10952000042DF4DB641C042CEFDB70BDCC97002011
:10953000FC9700209C050020DC9700202DE9FF47C8
:10954000002107E1DFF8189219F801908DF80C90CE
:10955000DFF80C9209F1040919F801908DF80890D0
:10956000DFF8FC9109F1080919F801908DF80490D1
:10957000DFF8EC9109F10C0919F801908DF80090D1
:10958000012056E00DF10C09814419F8019C4FEAC5
:10959000D91909EBC90909EB49090DF10C0A8244F3
:1095A0001AF801AC89EA4A090DF10C0A0AF8009090
:1095B0000DF10809814419F8019C4FEAD91909EB0A
:1095C000C90909EB49090DF1080A82441AF801ACEE
:1095D00089EA4A090DF1080A0AF800900DF1040918
:1095E000814419F8019C4FEAD91909EBC90909EB23
:1095F00049090DF1040A82441AF801AC89EA4A09C2
:109600000DF1040A0AF800900DEB000919F8019C0D
:109610004FEAD91909EBC90909EB49090DEB000A11
:109620001AF801AC89EA4A0909F0FF090DF800901F
:10963000401C0428A6DB9DF80E909DF80FA089EA37
:109640000A029DF80C909DF80FA089EA0A039DF884
:109650000A909DF80BA089EA0A049DF808909DF8ED
:109660000BA089EA0A069DF806909DF807A089EAF2
:109670000A079DF804909DF807A089EA0A059DF85D
:1096800002909DF803A089EA0A0C9DF800909DF8CD
:1096900003A089EA0A089DF80D9089EA020989EA7F
:1096A00006099DF809A089EA0A099DF804A089EA3B
:1096B0000A0989EA070989EA0809DFF8A4A00AF873
:1096C00001909DF8099089EA030989EA040989EA69
:1096D00005099DF805A089EA0A099DF800A089EA14
:1096E0000A0989EA0C09DFF878A00AF1040A0AF8E5
:1096F00001909DF80C9089EA020989EA06099DF813
:1097000005A089EA0A0989EA070989EA08099DF892
:1097100001A089EA0A09DFF848A00AF1080A0AF854
:1097200001909DF80D9089EA03099DF808A089EA47
:109730000A0989EA040989EA05099DF801A089EA6C
:109740000A0989EA0C09DFF818A00AF10C0A0AF8DC
:109750000190491C0429FFF6F5AEBDE8FF87000023
:10976000FC9700200E49C8798A79CA714A798A71B2
:109770000A794A710871087A897A094A1172114680
:109780008872487ACA7A4A72C872087B497B044A4E
:10979000117311468A7B4A73CA7B8A73C8737047F8
:1097A000FC97002000200FE000210AE0084A02EBAD
:1097B0008002525C074B9A5C054B03EB80035A54C2
:1097C000491C0429F2DB401C0428EDDB7047000033
:1097D000FC970020CC350108F8B5002500264F483D
:1097E000006882004E494F48FEF7D2FC4B4804689F
:1097F0008CE0601E4B4901EB8000006800904748F8
:10980000006894FBF0F100FB114080BB9DF80070F4
:109810009DF801008DF800009DF802008DF8010010
:109820009DF803008DF802008DF803709DF800008C
:109830003D49085C8DF800009DF80100085C8DF83A
:1098400001009DF80200085C8DF802009DF80300FD
:10985000085C8DF803003148006894FBF0F0334950
:10986000085C9DF8001048408DF8000024E0FFE7F8
:109870002A48006806281FDD2848006894FBF0F19C
:1098800000FB1140042817D19DF8000005F07CF979
:109890008DF800009DF8010005F076F98DF80100C3
:1098A0009DF8020005F070F98DF802009DF80300A4
:1098B00005F06AF98DF80300A006050E1748007838
:1098C000201A8006060E1748805D9DF8001048405B
:1098D000144948550846304440789DF801104840E6
:1098E0001049294448700F48304480789DF8021090
:1098F00048400C49294488700A483044C0789DF893
:109900000310484007492944C870641C084800688F
:10991000401C8000A0423FF76CAFF8BDA0050020BE
:10992000389900200C980020CC360108CC3701086B
:109930009C05002000BFFEE730B5002068E0364CF3
:10994000235C245C344D2D1D2D5C6C40324D08355C
:109950002D5C6C40304D0C352D5C84EA05022E4C9C
:10996000255C241D245C85EA0401CC0904EBC404B5
:1099700004EB440484EA4104E1B2274C245C81EA0C
:1099800002056C40244D2C542C1D245C08352D5CA4
:1099900084EA0501CC0904EBC40404EB440484EA22
:1099A0004104E1B21C4C241D245C81EA020565409F
:1099B000194C241D2554241D245C174D0C352D5C99
:1099C00084EA0501CC0904EBC40404EB440484EAF2
:1099D0004104E1B2104C0834245C81EA02056C4079
:1099E0000D4D08352C542C1D245C84EA0301CC0950
:1099F00004EBC40404EB440484EA4104E1B22C1DEA
:109A0000245C81EA02056C40034D0C352C54401C4B
:109A1000042894DB30BD0000FC9700200948008832
:109A200078B108480088401E80B20649088040B9D5
:109A3000002005494870C1F82404C1F82804C1F881
:109A40002C04704720050020944A00207047000035
:109A500070B505460C46002605F07005204600F05E
:109A6000E1F806460E4A32F814100E4A52F8240065
:109A700005F00AFA2146272004F01CFD45EA0600FD
:109A8000214604F017FD064A32F81410054A52F830
:109A9000240005F0FBF9204600F0C4F870BD00007A
:109AA000243501081435010810B504460A4A32F875
:109AB00014100A4A52F8240005F0E6F92146E22083
:109AC00004F0F8FC044A32F81410044A52F8240056
:109AD00005F0DCF910BD000024350108143501083B
:109AE00010B504460A4A32F814100A4A52F8240003
:109AF00005F0CAF92146E12004F0DCFC044A32F802
:109B00001410044A52F8240005F0C0F910BD0000FA
:109B10002435010814350108F0B5C1B005460E46DC
:109B200017461C460D4A32F814100D4A52F824000C
:109B300005F0AAF92846214604F0BCFC23463A4623
:109B4000314601A804F0C5FC044A32F81410044A56
:109B500052F8240005F09AF941B0F0BD243501080F
:109B60001435010870B505460C460D4A32F814103C
:109B70000C4A52F8240005F087F92846214604F0E3
:109B800099FC2146FF2004F095FC0646044A32F871
:109B90001410044A52F8240005F078F9304670BDDC
:109BA000243501081435010830B5C3B005460C460C
:109BB00021460720FFF7D6FFC0F342004190204620
:109BC00000F04EF842909DF80801202805DD20465F
:109BD000FFF76AFF002043B030BD104A32F814107E
:109BE0000F4A52F8240005F04FF92146612004F095
:109BF00061FC23469DF80821294601A804F069FC70
:109C0000064A32F81410064A52F8240005F03EF9CC
:109C10002046FFF749FF9DF80801DCE724350108DD
:109C20001435010870B504460B4A32F814100B4A7B
:109C300052F8240005F028F92146072004F03AFCE8
:109C40000546054A32F81410044A52F8240005F07B
:109C50001DF9284670BD000024350108143501089F
:109C600070B504460D4A32F814100D4A52F824001B
:109C700005F00AF92146602004F01CFC2146FF2073
:109C800004F018FC0546054A32F81410044A52F84C
:109C9000240005F0FBF8284670BD000024350108BB
:109CA0001435010870B504460D4629460620FFF715
:109CB00059FF20F0070604F0070006432A46314604
:109CC000062000F075F870BD2DE9F04104460E46FF
:109CD00015461F46052D01DD052000E028460546F6
:109CE000052C01DD052000E02046044604F10A01B0
:109CF000C8B23B462A46314600F032F8BDE8F08152
:109D000070B505460E46002431460620FFF72AFFAF
:109D1000044624F0280415B944F0200408E0012D7D
:109D200002D124F0280403E0022D01D144F00804FC
:109D300032462146062000F03BF870BD70B505465E
:109D40000C461646052C01DD052000E020460446A1
:109D5000334622462946102000F002F870BD00006C
:109D6000F0B5C1B005460E4617461C460E4A32F8FD
:109D700014100E4A52F8240005F086F845F0200031
:109D8000214604F097FB23463A4601A9304604F0E9
:109D9000A0FB054A32F81410044A52F8240005F0DA
:109DA00075F841B0F0BD00002435010814350108F4
:109DB00070B505460E461446104A32F81410104A83
:109DC00052F8240005F060F80E4A32F814100E4ADA
:109DD00052F8240005F058F845F02000214604F020
:109DE00069FB2146304604F065FB064A32F8141040
:109DF000054A52F8240005F049F870BD7035010895
:109E000060350108243501081435010870B5C0B06B
:109E100006460D461446202D00DC0DB940B070BD3D
:109E20000D4A32F814100D4A52F8240005F02CF8AF
:109E30002146B02004F03EFB23462A4669463046C0
:109E400004F047FB044A32F81410044A52F8240084
:109E500005F01CF800BFE1E72435010814350108BE
:109E60007FB5054611A103C9CDE90201002000908C
:109E700001902B46052202A91020FFF771FF2B4607
:109E8000052269461020FFF747FE00240AE002A8D9
:109E9000005D1DF80410884202D0002004B070BD9F
:109EA000601CC4B2052CF2DB0120F7E71122A3A449
:109EB000A500000010B5002807DA0A07140E054AAD
:109EC00000F00F031B1FD45403E00A07130E024ACD
:109ED000135410BD18ED00E000E400E0BFF34F8F15
:109EE0000648006800F4E06005490843001D034986
:109EF0000860BFF34F8F00BFFEE700000CED00E0ED
:109F00000000FA05704770B504460D4604F07F0165
:109F10002A460520FFF74CFF70BD10B504462146C8
:109F20007020FFF795FD10BD10B504460A4A32F8BF
:109F300014100A4A52F8240004F0A6FF214601201A
:109F400000F00EF8044A32F81410044A52F82400C3
:109F500004F09CFF10BD0000703501086035010859
:109F600070B504460E46002531460020FFF7FAFD85
:109F7000054614B925F0010503E0012C01D145F097
:109F80000105324629460020FFF712FF70BD000090
:109F90007CB5044619488169684688477CB99DF8B4
:109FA00000109DF8012011449DF8022002EB0121D0
:109FB0009DF803208818FEF7E3F800207CBD012CF3
:109FC00014D10F4807F066FE9DF800109DF801209F
:109FD00011449DF8022002EB01219DF80320114459
:109FE00045182846FEF7CCF80120E7E7FEF7BEF853
:109FF000B0FBF4F104FB1100E0E70000380300209F
:10A00000001000402DE9F04104460D461646EFF3DE
:10A0100011808046202080F3118800BF00BF3246A7
:10A020002946204600F00AF8074608F0FF0080F3B2
:10A03000118800BF00BF3846BDE8F0812DE9F74F19
:10A040008346174600BF2248007808B901F02AFA73
:10A0500000BF0BEB4B011E48603000EBC106DDF882
:10A0600004903569D6F80CA04FF00008554515D975
:10A07000B068441BBC4201D2204600E0384604468A
:10A080007068411922464846FEF782F8A044A14470
:10A090003F1B2544B068A84200D10025AAEB050467
:10A0A000BC4201D2204600E0384604464CB17068FC
:10A0B000411922464846FEF76BF8A044A1443F1BD5
:10A0C0002544B8F1000F00D035614046BDE8FE8F51
:10A0D000589900202DE9F04104460D46164600BF70
:10A0E0000D48007808B901F0DDF900BFEFF31180E9
:10A0F0000746202080F3118800BF00BF3246294662
:10A10000204600F00BF88046F8B280F3118800BFBB
:10A1100000BF4046BDE8F081589900202DE9F04786
:10A12000074688461646C24607EB47011B4800EB28
:10A13000C109D9F8140020B1012811D0022826D174
:10A140001EE0484601F0E6F90546B54201D200247A
:10A1500005E0344632465146484601F030FB18E0EF
:10A16000484601F0D7F90546B54201D2284600E03D
:10A170003046044622465146484601F020FB08E09E
:10A1800032465146484601F0E1FA044601E0002417
:10A1900000BF00BF2046BDE8F08700007099002096
:10A1A0000FB438B5044606A800906A4620460599C3
:10A1B00000F007F8054600200090284638BC5DF8FE
:10A1C00014FB2DE9F04F99B082460D46144603A8C2
:10A1D00014904020159000201690CDF860A01790A4
:10A1E00000BF2E786D1C06B9DDE0252E79D1002741
:10A1F0004FF0010900BF2E78232E12D02B2E0CD049
:10A200002D2E02D0302E10D103E047F001076D1C37
:10A210000EE047F002076D1C0AE047F004076D1CD2
:10A2200006E047F008076D1C02E04FF0000900BF90
:10A2300000BFB9F1000FDED14FF0000800BF2E784B
:10A24000302E01DB392E00DD07E06D1CA6F1300059
:10A2500008EB880100EB4108F1E700BF00201390F4
:10A260002E782E2E12D16D1C00BF2E78302E01DBE1
:10A27000392E00DD09E06D1CA6F13000139901EBC9
:10A28000810100EB41001390EFE700BF2E7800BF83
:10A290006C2E01D0682E02D16D1C2E7800E000E0FB
:10A2A000F6E700BF702E5DD008DC252E6AD0582E50
:10A2B00035D0632E09D0642E69D113E0732E3CD0C3
:10A2C000752E1DD0782E62D128E02168081D2060EF
:10A2D000D1F8009009F0FF0B594614A801F014FAC8
:10A2E00056E058E02168081D2060D1F80090CDE9C3
:10A2F00000870A22494614A8139B01F019F947E088
:10A300002168081D2060D1F80090CDE900870A225D
:10A31000494614A8139B01F081F939E000BF216878
:10A32000081D2060D1F80090CDE900871022494631
:10A3300014A8139B01F072F92AE02168081D20601F
:10A34000D1F800B000BF9BF800600BF1010B06B91B
:10A3500006E0314614A801F0D7F917980028F2DA80
:10A3600000BF15E02168081D2060D1F80090002092
:10A3700008210B461022CDE90010494614A801F02F
:10A380004DF905E0252114A801F0BEF900E000BF59
:10A3900000BF6D1C03E0314614A801F0B5F9179811
:10A3A0000028BFF61EAF00BF179800280ADD1698D8
:10A3B00020B103A95046169AFFF78CFEDDE916106E
:10A3C00008441790179819B0BDE8F08F62B670472F
:10A3D00000B587B0182101A8FDF701FF4FF4007008
:10A3E000019048200290012003900320049001A9CD
:10A3F0000248FEF798FF07B000BD0000000C0140C6
:10A4000000B587B0182101A8FDF7E9FE4FF40070F0
:10A41000019010200290012003900320049001A9D4
:10A420000248FEF780FF07B000BD0000000C0140AD
:10A430002DE9F047C8B006460F4690469946DDF82C
:10A4400044A1509C0025002001908DF80C00BAF129
:10A45000000F02D110200B9001E020200B90002271
:10A46000414602A8FDF7A6FF0546BDB901A84B4627
:10A470003A463146009002A8FDF732FF05466DB915
:10A4800001982060206800EB090101AA02A8FDF7ED
:10A4900084FF05462068019908442060284648B09A
:10A4A000BDE8F0872DE9F047C8B006460F46904654
:10A4B0009946DDF844A1509C0025002001908DF8BC
:10A4C0000C00BAF1000F02D110200B9001E0202007
:10A4D0000B900022414602A8FDF7DAFF0546BDB900
:10A4E00001A84B463A463146009002A8FDF766FFA8
:10A4F00005466DB901982060206800EB090101AAAA
:10A5000002A8FDF7B8FF05462068019908442060BD
:10A51000284648B0BDE8F087704700000F49087929
:10A5200049790E4A117111468A794A71CA798A713C
:10A53000C871087A897A094A117211468872487A74
:10A54000CA7A4A72C872087BC97B044A11731146E1
:10A550008A7BCA734A7B8A7348737047FC970020D2
:10A5600000200FE000210AE0084A02EB8002525C62
:10A57000074B9A5C054B03EB80035A54491C042992
:10A58000F2DB401C0428EDDB70470000FC97002044
:10A59000CC36010810B5FEF7E9FE10BD08B5184825
:10A5A000006840F47000164908601648006840F0E2
:10A5B0000100144908600846406840F08000486087
:10A5C0000020009002E00098401C009044F62061BA
:10A5D00000988842F7D300200A494860C8620846BC
:10A5E000006809490840074908604FF41F00886067
:10A5F0000846006820F48020086007F0D1FA08BD02
:10A6000088ED00E000100240FFFFF6FE10B50121CA
:10A61000880707F0A2FB40B10121880707F09AFBE9
:10A620000249C868804708F081FA10BD380300204D
:10A630001FB50020009001900290039040F2AF40BF
:10A64000ADF800000020ADF80200ADF80400F920DC
:10A6500002900020ADF806008DF80C0069464FF01E
:10A66000804007F023FB002203211C2005F014FF8B
:10A6700000214FF0804007F011FB002240F2AF4173
:10A680004FF0804007F075FBF921880707F000FBC9
:10A690000121880707F056FB0121880707F05AFBC4
:10A6A0000121880707F052FB4FF0804007F0F8FACD
:10A6B0001FBD000010B50121064807F04EFB40B158
:10A6C0000121044807F046FB03490869804708F068
:10A6D00028FA10BD00040040380300201FB50020F8
:10A6E000009001900290039040F2AF40ADF800005E
:10A6F0000020ADF80200ADF8040040F2CF700290E7
:10A700000020ADF806008DF80C006946134807F0EC
:10A71000CDFA002204211D2005F0BEFE00210F48C5
:10A7200007F0BCFA002240F2AF410C4807F021FBD1
:10A7300040F2CF71094807F0ABFA0121074807F052
:10A7400001FB0121054807F005FB0121034807F043
:10A75000FDFA024807F0A4FA1FBD00000004004003
:10A7600010B50121880707F0F8FA18B10121880710
:10A7700007F0F0FA10BD10B508F05AF810BD00004F
:10A7800000B591B0402101A8FDF729FD2C4890F8B3
:10A790004E008DF804002A4890F84F008DF805000F
:10A7A000274890F850008DF80600254890F8510091
:10A7B0008DF80700FE208DF8080048208DF809006C
:10A7C000DE208DF80A007F208DF80B0001208DF827
:10A7D0000C0002208DF80D00302219495231002062
:10A7E00000F030F800909DF800008DF80E009DF804
:10A7F00001008DF80F00124840788DF810003022CB
:10A800000F49523105A8FDF7C3FC30210C485230E6
:10A81000FDF7E5FC00200A4981F88200202101A80B
:10A8200000F0C4FB00F0D8FB142000F03FF820211A
:10A8300009A800F0BBFB00F0CFFB11B000BD000089
:10A840000067002070B506460C461546294620468E
:10A8500003F07EFA0646304670BD000010B504468F
:10A86000074890F8310440B14FF480620449113137
:10A870002046FDF78DFC002010BD0120FCE7000004
:10A88000CC62002030B50A46CD1701EB5575C5F3F3
:10A89000C703CD1701EB5575ED10A1EBC505ECB263
:10A8A000C25C0125A540AA43C25430BD10B5044680
:10A8B000204603F072F810BD30B502460846CD17A9
:10A8C00001EB5575C5F3C703CD1701EB5575ED10B9
:10A8D000A1EBC505ECB2D05C0125A540284008B12C
:10A8E000012030BD0020FCE770B505460E46144639
:10A8F00009482968C0F84E10A0F88860C0F8844064
:10A90000C4F38F20044988800846B0F8881003A05B
:10A9100005F05DF870BD0000006700200A433A258D
:10A920007800000001464878AA2808D18878BB281A
:10A9300005D1C878CC2802D10879DD281FD01B4862
:10A9400090F84E004A78904201D002207047174894
:10A9500090F84F008A78904201D00220F6E7134821
:10A9600090F85000CA78904201D00220EEE70F48DC
:10A9700090F851000A79904201D00220E6E7487928
:10A980007F2801D00120E1E78879DE2801D001206D
:10A99000DCE7C879482801D00120D7E7087AFE28EB
:10A9A00001D00120D2E70020D0E70000006700209E
:10A9B00070B58AB005460C46242101A8FDF70FFCAE
:10A9C000E0B28DF80400224629460DF10500FDF79E
:10A9D000DFFB01A8FFF7A6FFA0B99DF80E008228B3
:10A9E00001D00AB070BD0120274908702748DDF862
:10A9F000111001609DF80F00254908709DF81000A6
:10AA00004870EEE72048007801283AD100201E491E
:10AA1000087020220DF10501FFF714FF06461C48BF
:10AA20000088B0422CD11BA004F0D1FF1B4890F845
:10AA30008200102810DA194890F882001749523124
:10AA400001EB8000114909680160144890F8820008
:10AA5000401C124981F8820000200FE001AA411C2D
:10AA6000515C49B10D490A31095C01AB421C9A5C49
:10AA700011430A4A0A321154411CC8B22028EDDBA6
:10AA8000AFE700BFADE70000440500204805002007
:10AA9000460500200A43524354000000006700208E
:10AAA00070B58AB005460C46242101A8FDF797FB36
:10AAB0000026344890F84E008DF80400314890F894
:10AAC0004F008DF805002F4890F850008DF80600D3
:10AAD0002C4890F851008DF8070042208DF80800AE
:10AAE00001208DF80900274800788DF80A008DF8BC
:10AAF0000B50FF208DF80C008DF80D0000208DF814
:10AB00000E008DF80F008DF810008DF811001D4813
:10AB100090F884008DF812001A4890F885008DF89E
:10AB20001300184890F886008DF81400154890F826
:10AB300087008DF81500134890F888008DF81600EE
:10AB4000104890F889008DF817000E4880788DF82D
:10AB500018001B2202A90020FFF774FEC6B28DF870
:10AB600023600AE0202101A800F020FA00F034FA66
:10AB70003220FFF79BFE601EC4B2002CF2D10AB057
:10AB800070BD00000067002030B589B00546242163
:10AB90006846FDF724FB344890F84E008DF800001D
:10ABA000314890F84F008DF801002F4890F8500080
:10ABB0008DF802002C4890F851008DF80300FE201B
:10ABC000294981F84A004821274880F84B10DE21A6
:10ABD00080F84C107F2180F84D1090F84A008DF8D5
:10ABE0000400214890F84B008DF805001E4890F8AD
:10ABF0004C008DF806001C4890F84D008DF80700B9
:10AC000020208DF8080001208DF80900164890F8E2
:10AC10008E048DF80A00144890F88F048DF80B000C
:10AC2000114800788DF80C008DF80D5020216846F1
:10AC300000F0BCF900F0D0F9C820FFF737FE00247F
:10AC40000EE009498A31202202FB0410114600F06F
:10AC5000ADF900F0C1F91420FFF728FE601CC4B262
:10AC6000202CEEDB09B030BD0067002010B50120BC
:10AC70000749087007480078401C0649087041F2EF
:10AC80007070054908600548816B0020884710BD39
:10AC900038050020006700203C0500203803002014
:10ACA00070B505460C460020034981F83104214661
:10ACB0000A2007F027F970BDCC62002070B5AF48BC
:10ACC000006878B1AD480068401EAC49086048B9DA
:10ACD000AB48007830B1AA480078052802D005209A
:10ACE000A7490870A648007806287CD2DFE800F063
:10ACF000030443B9D8FE3EE11E210120FFF7D0FE38
:10AD0000A0480088401C9F490880084600882828E1
:10AD100030DD00219C48A0F88A1440F2FF11A0F811
:10AD20008C140120984908720020487230219648FE
:10AD30005230FDF754FA0020934981F8820091497E
:10AD4000088091498871FF2240218F480A30FDF721
:10AD50003FFA8D4A92F88A149079FFF7A1FF0021FB
:10AD600089480A30FFF78EFD00208749C87102200C
:10AD700083490870FFE08448B0F88A1483A004F087
:10AD800026FE8148C079012816D07F488A30FFF717
:10AD900065FD88B901207C49C871002048724FF4D4
:10ADA00080628A31FFF74EFD7749A1F88E0408468C
:10ADB000B0F88A14A0F88C147348B0F88C0440F2F0
:10ADC000FF11884219D07048407A401CC0B26E49C9
:10ADD0004872C82801DDC82048726B4991F88C047C
:10ADE000FFF7D2FE00E0C5E04FF4E160FFF75EFD43
:10ADF000654991F88C04FFF7C7FE6348407A6249C1
:10AE0000097A88422CDB6048C079012828D10020CB
:10AE10005D49C87100241EE021465B480A30FFF7F7
:10AE20004BFD70B1214658480A30FFF72BFD5648BC
:10AE3000A0F88A44024692F88A149079FFF730FF0E
:10AE40000DE051488088401EA04202D103204C49A9
:10AE50000870601CC4B24C488088A042DCDC00BF93
:10AE600089E000204749088047488078401C4649CF
:10AE70008870202144480A30FDF7B1F90420404988
:10AE80000870414841784078401C3F4A5070C829BA
:10AE900002DD0120114648703EA004F098FD6AE0F2
:10AEA000FFF76EFC37480088401C3649088008468A
:10AEB0000088322846DB002500200880002409E0B5
:10AEC000214631480A30FFF7F7FC08B1681C85B20B
:10AED000601C84B22C488088A042F1DC294630A056
:10AEE00004F075FD2DB90520254900E02BE0087020
:10AEF00041E025488079401C234988710820087268
:10AF0000002416E0214620480A30FFF7D5FC70B136
:10AF100021461D480A30FFF7B5FC1B48A0F88A44BB
:10AF2000024692F88A149079FFF7BAFE05E0601C99
:10AF3000C4B215488088A042E4DC00BF022010495A
:10AF4000087018E017E01E210220FFF7A9FD0D4848
:10AF50000088401C0B49088008460088282808DD26
:10AF6000002006490860074908800549087006F076
:10AF700021FF00E000BF00BF70BD00003C050020C5
:10AF80003805002042050020006700200A533A25BA
:10AF900064000000444F574E5F5155455259000020
:10AFA0000A4C4E756D3A25640000000070B50546E8
:10AFB0000C46002006F0CEFC0549C86A80470646CC
:10AFC000E1B204483246836A28469847012070BDA2
:10AFD00038030020B802002010B54FF4FA7408E0DE
:10AFE00003F038FF00B110BD0220FFF75FFC601EC8
:10AFF00084B2002CF4D100BFF5E700BFFEE70021CA
:10B0000007E048F2782100BF0A1EA1F1010399B2BE
:10B01000FAD1021EA0F1010398B2F2D170470000EC
:10B0200010B590B0044620798DF8000020791B28D7
:10B030007AD2DFE800F0791E0E5B2A79797979AA55
:10B040009E8A7A7979C6C17979CBCADDCCEFF0EDE9
:10B05000EC000D22A649601D04F04BFD01F000FA42
:10B060000D22A349C02002F09DFB01208DF80000B5
:10B0700000BF0D220DF101019D4804F03AFD0E22A2
:10B0800069460B2005F0D2FB2EE106229949601D8E
:10B0900004F02FFD984890F8820028B1964890F867
:10B0A00082009449491E88709248401E807820B1E1
:10B0B0009048401E8078042803DD01208D49491EF8
:10B0C00088708C48401E80788C49497A884204DD1B
:10B0D0008A48407A8749491E88708649491EC8783F
:10B0E00005F0D8FD04208DF8000000BF824890F8DC
:10B0F0008400292800D1F7E07F4890F884002828B0
:10B1000000D1F1E07C4890F88400332800D1EBE0D6
:10B1100006220DF10101774804F0EBFC0722694695
:10B120000B2005F083FBDFE0D8E0734890F87F0048
:10B1300000B9D9E003227249601D04F0DAFC032251
:10B140006F49D82002F02EFB00BF6B4890F87F00BB
:10B1500000B9C9E00B208DF8000003220DF10101B8
:10B16000674804F0C6FC042269460B2005F05EFB2C
:10B17000BAE0614890F8800000B9B5E06079012834
:10B1800002D11E205F49487000BF5B4890F88000E4
:10B1900000B9A9E009208DF800005A48407800283D
:10B1A00001DD012000E000208DF801000222694647
:10B1B0000B2005F03BFB97E04F48816A204688470B
:10B1C00000BF4D49C86A80478EE000BF8CE018225E
:10B1D0004D49601D04F08DFC4B48401E807818B12D
:10B1E000012006F07BFB02E0002006F077FB00BFA9
:10B1F00015208DF8000018220DF10101424804F0DD
:10B2000078FC192269460B2005F010FB6CE029E060
:10B2100058E000E01AE00D223C49601D04F069FC92
:10B2200001F01EF934480C21D0F80C213748401C9D
:10B2300090473149D1F8FC0080470D223349C020A6
:10B2400002F0B0FA17208DF8000000BF0D220DF1BA
:10B2500001012E4804F04DFC0E2269460B2005F03A
:10B26000E5FA41E003222A49601D04F042FC284827
:10B27000401EC178807801EB00204EF660218842A4
:10B2800007DDEA202249491E887060212048401EBF
:10B29000C1701F4A521ED378927803EB022290B2FB
:10B2A000154AD2F8041188471349D1F8FC008047A9
:10B2B000032217494FF4856002F074FA19208DF8C3
:10B2C000000000BF03220DF10101114804F011FC40
:10B2D000042269460B2005F0A9FA05E00648D0F8DB
:10B2E000E4102046884700BF00BF10B010BD00002A
:10B2F000F5170020C0030020EC0300208820002068
:10B30000BC030020B9030020781700200318002098
:10B31000C80300202DE9F0418CB0044600262079B6
:10B320008DF810002079072871D2DFE800F09A0428
:10B3300027286271900008226946402001F0ACFC89
:10B340000822A11D684604F0C3FB40B900204B4908
:10B350000870084600788DF8110002250DE00120E4
:10B3600046490870084600788DF8110008220DF152
:10B370001201684604F0BDFB0A2574E000BF607945
:10B38000042810DD00208DF811004C208DF81200EB
:10B390004F208DF8130043208DF814004B208DF8BA
:10B3A0001500062524E002208DF8100060798DF844
:10B3B0001100207902280BD16179502202EB011093
:10B3C0002F4910224B6A0DF11201984712250FE008
:10B3D0006179502202EB0110294910220B6AA11D4C
:10B3E000984710220DF11201A01D04F082FB1225D6
:10B3F00039E008220DF11201402001F04DFC03203C
:10B400008DF8100000208DF811000A252BE028E0AF
:10B410000822A11D402002F0C5F903F087FC074671
:10B42000A01D02F067FB804615483A460421036CD4
:10B430004046984700208DF811008DF81200082230
:10B440000DF11301A01D04F054FB0B250BE00020AF
:10B450008DF811000A4841690DF1120088470E2548
:10B4600001E0012600BF00BF26B92A4604A9092031
:10B4700005F0DCF90CB0BDE8F0810000A503002068
:10B48000B8020020002106E01E2100BF0A1EA1F123
:10B49000010399B2FAD1021EA0F1010398B2F3D1CF
:10B4A0007047000010B5124C03202061606111A0AC
:10B4B000A0611349E1614FF4805121620021A16232
:10B4C0006162E1620BA020660E4961661021A166EF
:10B4D00000212167E16661670BA1E01DFCF797FE83
:10B4E0000AA12046FCF793FE2020A07110BD0000A9
:10B4F000589900205465726D696E616C00000000FF
:10B50000009A002000AA0020525454005345474797
:10B510004552000010B501460A69CB689A4204D82A
:10B520008C68641EE41AA01801E0D41A601E10BDD5
:10B530002DE9FC5F06460F4692469846DDE90C452C
:10B54000002F01DA784200E0384683464FF00109C7
:10B5500003E09BFBFAFB09F10109D345F9DAC84581
:10B5600000D9C14634B1002F03DB05F004000428E4
:10B5700000D1641E05F0020010B1B8F1000F11D027
:10B5800005F0010070B96CB108E0641E202130465E
:10B5900000F0BAF8F068002800DA02E00CB1A1452A
:10B5A000F3D300BFF068002836DB002F05DA7F42B6
:10B5B0002D21304600F0A8F807E005F0040004282B
:10B5C00003D12B21304600F09FF8F068002823DBE0
:10B5D00005F00200022814D105F0010088B9B8F185
:10B5E000000F0ED16CB108E0641E3021304600F02F
:10B5F0008BF8F068002800DA02E00CB1A145F3D323
:10B6000000BFF068002807DB434652463946304603
:10B61000CDE9004500F002F8BDE8FC9F2DE9FC5F94
:10B620008046894615461E460C9CCDF8049001279D
:10B63000BB4605E00198B0FBF5F001900BF1010B62
:10B640000198A842F6D25E4500D9B3460D9800F0A5
:10B650000100D0B9CCB10D9800F00200022803D14E
:10B6600016B93020009001E02020009009E0641E0F
:10B670004046009900F048F8D8F80C00002800DA9D
:10B6800002E00CB1A345F2D300BFD8F80C000028AB
:10B6900035DB09E0012E01D9761E04E0B9FBF7FA8B
:10B6A000AA4500D201E06F43F4E700BF00BFB9FB39
:10B6B000F7FA0AFB1799134810F80A10404600F0F1
:10B6C00023F8D8F80C00002800DA03E0B7FBF5F700
:10B6D000002FECD100BF0D9800F0010078B174B1DB
:10B6E00009E0641E2021404600F00EF8D8F80C0056
:10B6F000002800DA02E00CB1A345F2D300BFBDE898
:10B70000FC9F0000CB38010870B504460E46A568C2
:10B71000681C6168814206D320684655681CA06099
:10B72000E068401CE060D4E9011088420DD1A268B5
:10B7300021682069FEF7CEFCA168884203D04FF053
:10B74000FF30E06001E00020A06070BD2DE9F0470F
:10B750000446894617464FF0000AE56800BFD4F852
:10B760001080A84503D9A8EB0500461E04E0A5EB10
:10B770000800401CA1680E1AA068401BB04201D905
:10B78000304601E0A068401B0646BE4201D230466A
:10B7900000E0384606466168481932464946FCF7DB
:10B7A000F7FCB244B144BF1B3544A068A84200D1A5
:10B7B0000025E560002FD2D15046BDE8F0872DE985
:10B7C000F047044689461546E668A068871BAF42E5
:10B7D00008D9616888192A464946FCF7D9FC7019CE
:10B7E000E06010E0B8466168881942464946FCF7B7
:10B7F000CFFCA5EB070809EB070142466068FCF7A0
:10B80000C7FCC4F80C80BDE8F08702E008C8121F2E
:10B8100008C1002AFAD170477047002001E001C139
:10B82000121F002AFBD1704770B590B004460E4637
:10B830001546382D00DD38252A46314602A8FCF78A
:10B84000A7FCC5F1380102AA50192022FCF7C0FC60
:10B8500061208DF8000063208DF801006B208DF8C9
:10B8600002002D208DF8030020788DF80400607808
:10B870008DF80500A0788DF806003A208DF80700B5
:10B880000348402182696846904710B070BD0000AF
:10B89000B80200201FB50020009001900290039094
:10B8A00010226946FEF7AEFBA0B19DF800003128DA
:10B8B00002D0322808D102E000F060F809E006A1C9
:10B8C0000020FEF76DFC04E004A10020FEF768FCF8
:10B8D00000BF00BF1FBD0000320A0000556E737527
:10B8E00070706F7274656420696E737472756374BE
:10B8F000696F6E73210A00007047000010B50024C4
:10B900002CE004EBC40101EB0411164A881819213C
:10B91000FCF765FC04EBC40101EB0411124A881822
:10B920001921FCF75CFC04EBC40101EB04110F4A84
:10B9300088181921FCF753FC04EBC40101EB041136
:10B940000B4A88181921FCF74AFC0020094921F804
:10B950001400094921F81400601CC4B2282CD0DB63
:10B9600010BD000028070020100B0020F80E00205A
:10B97000E0120020C816002018170020F8B5002695
:10B9800002F014FB07462748427827490020FEF7BB
:10B9900007FC07F0030018B124A10020FEF700FC0B
:10B9A000002437E0254830F814000090244830F88F
:10B9B0001430621C23A10020FEF7F2FB00260025B4
:10B9C0001AE004EBC40000EB041027490844435D6F
:10B9D0002A4626A10020FEF7E3FB701CC6B2052E06
:10B9E00008DD00261EA10020FEF7DAFB41F28830B8
:10B9F00001F0C6FF681CC5B2214800788542E0DB33
:10BA000020A10020FEF7CCFB41F2883001F0B8FF06
:10BA1000601CC4B2282CC5DB1BA10020FEF7C0FBB4
:10BA2000F8BD000090170020645401084B65797040
:10BA3000616420525820455252210A0018170020F4
:10BA4000C8160020534E3A253033642052785F6385
:10BA50006E743A25642041434B5F636E743A2564EB
:10BA60000A202020200000002807002072784B5078
:10BA70005B253033645D3D3078253032782C2000F2
:10BA8000A40300200A0000000A2A2A2A2A2A2A2AB5
:10BA90002A2A2A2A2A2A2A2A2A2A2A2A2A2A2A2A06
:10BAA0002A2A2A2A2A2A2A2A2A2A2A2A2A2A2A2AF6
:10BAB0002A2A2A2A2A2A2A2A2A2A2A2A2A2A2A2AE6
:10BAC0002A2A2A0A0000000010B5CA7872B1CA7882
:10BAD000282A0BDCCA78521E054B33F81220521C60
:10BAE00093B2CA78521E024C24F8123010BD0000E6
:10BAF000181700207047000010B50446A079D0B197
:10BB0000A079282817DCE27A511EA279521E02EB96
:10BB1000C20303EB0212084BD01802F07DFAA079A1
:10BB2000401E064931F81000401C81B2A079401E29
:10BB3000024A22F8101010BD28070020C816002065
:10BB40007047704730B591B0044606252022402149
:10BB500001A8FCF73DFB2A4604F1080101A8FCF707
:10BB600017FB402201A902A0FFF75EFE11B030BD15
:10BB700066756E000146C21700EB5272C2F3C7022F
:10BB8000014B1A7070470000A403002070B50546F1
:10BB9000284600F028F8041E00D170BD61782046C8
:10BBA00002F082FB08B90020F7E70120F5E770B545
:10BBB0000446002502F0C0FB051E00D170BD7022B6
:10BBC00021462846FCF7E4FA02F086FB0646314699
:10BBD000284602F0A5FB0120F0E700B502F084FB47
:10BBE00002F08EFB00BD70B50646002512E0284627
:10BBF00002F068FB041E00D10AE00422314604F181
:10BC00006000FCF7F7FA10B96570204670BD00BF00
:10BC1000681CC5B202F060FBA842E8DC0020F5E732
:10BC2000704710B50346D3F8A400806868B153F894
:10BC3000A40F806880781C68A468E47840EA042037
:10BC4000108053F8A409806810BD0020108000BF48
:10BC5000FAE710B5034653F8A40F406880781C68D3
:10BC60006468E47840EA0420108053F8A40940682E
:10BC700010BD0346D3F8A400006800781080D3F804
:10BC8000A4000068704770B504460D46E07C50B1D2
:10BC900000BFD4F8AC10A06C0022CB6A11469847C4
:10BCA00000BF0021E174A078032808D1D4F8A800CF
:10BCB000006920B1D4F8A8000169204688472046D1
:10BCC00006F042F9607830B1D4F8AC00C168204683
:10BCD00088470020607070BD2DE9F04104460D4694
:10BCE000A078032808D1D4F8A800406920B1D4F87E
:10BCF000A80041692046884705EB450704F1140672
:10BD000006EB870000210A460B4641600281438111
:10BD100000BF204606F021F9BDE8F0812DE9F04191
:10BD200004460F460125D4F8AC0000221146036BEF
:10BD300004F10B0098470646082E04D0204606F072
:10BD400016F9BDE8F081E07A00F0600020B120280B
:10BD500009D0402815D10DE004F10B01204606F072
:10BD6000C5FE05460EE004F10B01204606F01EF963
:10BD7000054607E004F10B01204606F0CFFE05461C
:10BD800000E000BF00BFC5B9B4F8110018B92046E3
:10BD900006F0E3F814E0E07A00F0800048B100BF5C
:10BDA0004C20035B00212046A26C06F0BDFA00BFC8
:10BDB00006E0204606F0C8F802E0204606F0D7F874
:10BDC00000BFBEE770B504460D460026287800F097
:10BDD000030020B101282ED002282DD111E0A07837
:10BDE000022802D0032809D100E000BF688801289A
:10BDF00003D100212172002070BD00E000BF00BF10
:10BE00001BE02E79A078032814D1688890B98EB1F0
:10BE1000802E0FD000BFD4F8AC003146826B204694
:10BE2000904700BFD4F8A8002946C2682046904732
:10BE30000020E1E701E000E000BF00BF0120DBE7F8
:10BE400070B504460E460125A078022802D00328CA
:10BE500008D103E0207800B9002504E0207800B183
:10BE6000002500E000BF00BF35B901231A46214676
:10BE700004F1440006F08AF8284670BD2DE9F04729
:10BE800006460D460027B8464FF0010906F1440466
:10BE9000287800F0030020B101284BD0022852D1AD
:10BEA00050E06888070A95F80280102F3FD2DFE83B
:10BEB00007F03E08182331323334353E3E3E3E3ED5
:10BEC0003E36781E304951F8203004F108024146D0
:10BED000304698476060E888402801D108202081DA
:10BEE00026E0781E284951F8203004F10802414626
:10BEF0003046984760601BE0B8F1060F09DA781EFB
:10BF0000214951F8203004F1080241463046984753
:10BF100060600DE000BF00BF00BF00BF08E004F19B
:10BF2000080241463046FFF77CFE606000E000BF3B
:10BF300000BF09E0D6F8A8002946C26830469047FD
:10BF4000814601E000E000BF00BF2089C8B1E88859
:10BF5000B8B12089E988884201DA208900E0E888C0
:10BF600020812189B6F81100814208DA20892188D0
:10BF700090FBF1F201FB120008B90121F1744FF0BE
:10BF800000094846BDE8F0879400002070B50446DB
:10BF90000D46A078012804D0022803D0032810D130
:10BFA00001E00FE00EE0287950B9D4F8A800411C58
:10BFB00001231A4604F1440005F0E8FF002070BD9B
:10BFC00000E000BF00BF0120F9E700002DE9F041CB
:10BFD00004460E4635790127307800F0030020B181
:10BFE000012823D0022845D126E0A078022802D0DB
:10BFF000032818D100E000BF207918B1012024499E
:10C00000087002E0002022490870207A30B12048F0
:10C01000007840F002001E49087002E000201C4930
:10C020000870002700E000BF00BF24E0A0780328CC
:10C0300001D105B900271EE0A078032819D105F029
:10C04000800080280BD105F07F0000EB400104F157
:10C05000440000EB810080780D49087008E005EB92
:10C06000450104F1140000EB810080780849087054
:10C07000002700E000BF00BF37B902231A46044979
:10C0800004F1440005F082FF3846BDE8F08100006D
:10C09000A00000200246012070470246888888B927
:10C0A000C88878B9887800F07F00507090780328AD
:10C0B00008D0507810B10220907001E001209070FB
:10C0C000002070470120FCE770B504460D460126AC
:10C0D000A8782549087008460078012842D8A07839
:10C0E00001283CD0022802D0032839D110E01E4894
:10C0F000007858B1D4F8A80042681B48017820465F
:10C1000090471948007820700320A070002628E08E
:10C110001548007860B9D4F8A80082681248017800
:10C12000204690471048007820700220A07014E04C
:10C1300020780D49097888420FD02178D4F8A800DA
:10C14000826820469047084800782070D4F8A800FC
:10C1500042680548017820469047002601E000E04B
:10C1600000BF00BF304670BDA20000200246002084
:10C17000704770B504460D460026287800F003008D
:10C1800020B1012828D0022827D111E0A078022868
:10C1900002D0032809D100E000BF6888012803D13C
:10C1A00001212172002070BD00E000BF00BF15E03A
:10C1B0002E79A07803280ED1688860B95EB1802EF0
:10C1C00009D000BFD4F8AC003146426B20469047FE
:10C1D00000BF0020E7E701E000E000BF00BF012052
:10C1E000E1E702469078012804D0022803D0032812
:10C1F0000BD101E00AE009E0087928B98878D2F883
:10C20000A83058700020704700E000BF00BF012038
:10C21000F9E702460020704710B50346D3F8A44062
:10C22000E46854F821000478148010BD10B50A4861
:10C2300090F8900000B910BD04F03AFF01200749C2
:10C24000487002F06FFC04F04FFF00BF00F06AF886
:10C250000028FBD000BFEEE7EC030020D44E002006
:10C2600070B5124890F8900000B970BD1048007881
:10C2700000B9FAE70E48807800B1F6E70D4805F0FE
:10C2800009FD0546FBF77CFF002407E0FBF76EFF86
:10C29000C1B2074823300155601CC4B2202CF5DB25
:10C2A0000348233007F0C2F800BFDEE7EC030020AC
:10C2B000D44E00200010004010B50446154890F8F8
:10C2C000900000B910BD1448007800B9FAE713498E
:10C2D000086A8047032801DD132060711048007848
:10C2E00080F001000E4908700B480078A0730846E2
:10C2F000007808B10320A07207482330084A12785A
:10C30000102313FB02011A4604F10F00FBF740FF54
:10C3100000BFD7E7EC030020D44E002038030020F4
:10C320002805002030B589B01C208DF800001120B0
:10C330008DF801008DF802008DF803008DF80400DF
:10C3400013208DF80500062406E004F15B00C0B25E
:10C350000DF80400601CC4B2212CF6DB684604F022
:10C36000D3FF20208DF80000684604F02FFF202026
:10C370008DF800009DF80600612809D19DF81D0088
:10C38000782805D19DF81E00792801D1012500E00B
:10C390000025284609B030BD10B5044644B101213E
:10C3A000084802F071FD0221074802F06FFD07E026
:10C3B0000221054802F068FD0121024802F066FDF5
:10C3C00010BD00000008014000100140194890F81D
:10C3D0007B0020B1174890F87B00174988701548FA
:10C3E00090F87C00A0B114488078022802D1012086
:10C3F00011498870104880781A2802D119200E49F6
:10C4000088700D488078502802D14F200A498870E2
:10C4100009488078002806DD07488078054991F8AA
:10C420007510884204DD01200349887000207047A0
:10C430000120FCE7EC030020AC0300200748407813
:10C44000012803DB05484078202804DD012003494A
:10C450004870002070470120FCE70000AC0300207A
:10C46000114890F87D0020B10F4890F87D000F49E9
:10C4700048700D4890F8810030B10C48407804288D
:10C4800002DA04200949487008484078012803DB93
:10C4900006484078092804DD01200449487000203E
:10C4A00070470120FCE70000EC030020F417002097
:10C4B0000221084AD17000219180002006E006493F
:10C4C00001EB800100220A60411C88B2C828F6DB1B
:10C4D000704700004C6200202C5F002001460020C5
:10C4E00008E0094A02EB800201EB80031B6813603D
:10C4F000421CD0B21E28F4DB0122034B9B1FDA70D2
:10C5000000229A80704700005262002010B500207F
:10C5100005494870087008710449886A80470249D3
:10C5200048710120C87010BD290500203803002083
:10C5300010B51A4890F8C40000B910BD1848C07B67
:10C5400000B9FAE71648407C802800DBF5E7144A7A
:10C55000517C907C00F02AF81148407C401CC1B20C
:10C560000F484174807C00EB80220E4800EB4200B3
:10C57000407881420FDB002109484174007C401C57
:10C58000C1B2074801740A2905DB0021C1730648BE
:10C59000816B0120884700BFCFE70000EC0300203B
:10C5A000175F00201A4F00203803002070B58AB0B2
:10C5B00004460D4620208DF804002A4881690DF1BB
:10C5C000050088472749086A8047032801DC312095
:10C5D00000E032208DF8090000208DF80A008DF867
:10C5E0000B002049886C804704EB84221E4911F817
:10C5F000121060F31F11C8B28DF8100000208DF8E2
:10C60000110004EB8421184800EB410040788DF8BC
:10C6100012008DF8135004EB8422134800EB420003
:10C62000801C00EB0511102205A8FBF7B1FD1B21B2
:10C630000DF1090001F08CFBC0B28DF824009DF8CB
:10C6400013309DF8102009A10020FDF7A9FD054930
:10C65000C86A8047064603483146426B01A89047A6
:10C660000AB070BD380300201A4F002070643A25CC
:10C670003032782C7365713A25640A002DE9F04157
:10C6800090B0804620208DF800000DF1010002F0EE
:10C69000ABFA00208DF806008DF80700B8F1010F05
:10C6A00023D1002618208DF805007D4890F87F00E2
:10C6B00080B37C484078002801DD012000E00020A4
:10C6C00078498978002901DD012100E0002100EB93
:10C6D00041007449C978002901DD012100E00021F1
:10C6E00000EB81008DF806001AE0052619208DF870
:10C6F00005006B4890F87F0060B16A4840780028D8
:10C7000001DD012000E0002066498978002902DD72
:10C71000012101E004E0002100EB41008DF806005A
:10C720000025B5E06048C07AA84200D1AEE05F487D
:10C7300090F82000002869D1002422E005EBC50212
:10C7400002EB4513584A0C321A44521C331902EBBF
:10C7500083019DF80500FFF7B7F905EBC50202EB71
:10C760004513514A0C321A44521C331902EB830010
:10C7700002AA052303FB04211A4603F0BAF9601C40
:10C78000C4B2052CDADB464890F88400332878D10F
:10C79000434890F88500012873D102F049FD002834
:10C7A0006FD00424002004EB4401062202EB410177
:10C7B0000DF8010004EB4401072202EB41010DF8E2
:10C7C000010004EB4401082202EB41010DF80100D5
:10C7D00004EB4401092202EB41010DF801001D2187
:10C7E0000DF1050001F0B4FA0746381204EB4401DC
:10C7F0000A2202EB41010DF80100F8B204EB4401FA
:10C800000B2202EB41010DF801003AE0002422E086
:10C8100005EBC50202EB4513234A0C321A44521CA5
:10C82000331902EB83019DF80500FFF74DF905EB85
:10C83000C50202EB45131C4A0C321A44521C331930
:10C8400002EB830002AA052303FB04211A4603F02E
:10C8500050F9601CC4B2042CDADBFF208DF81C00F8
:10C860008DF81D008DF81E001A210DF1050001F054
:10C870006FFA074638128DF81F00F8B28DF82000C5
:10C8800000BF2946684600F0FBFD00BF681CC5B22A
:10C890000548007AA8423FF745AF10B0BDE8F081E7
:10C8A000EC030020BB03002088200020F8060020B5
:10C8B00070B588B01C208DF800000DF1010002F069
:10C8C00093F915208DF80500002440E02348C07A34
:10C8D000A04200D139E0002513E004EBC40202EBD2
:10C8E00044131E4A0C321A44521C02EB85000DF10F
:10C8F0000602022303FB05211A4603F0FAF8681C1E
:10C90000C5B20A2DE9DB164890F88400332817D108
:10C91000134890F88500012812D102F089FC78B103
:10C9200000208DF81A0016210DF1050001F010FA13
:10C93000064630128DF81B00F0B28DF81C0000BFC7
:10C940002146684600F09CFD00BF601CC4B203484D
:10C95000007AA042BADC08B070BD00008820002038
:10C96000EC0300202DE9F04190B0064623208DF81D
:10C9700000000DF1010002F037F916208DF80500D6
:10C98000012E01D1002000E005208046002567E04F
:10C990003748C07AA84200D160E0002415E005EBDA
:10C9A000C50202EB4513324A0C321A44521C08EB02
:10C9B000040302EB83000DF10602042303FB0421B0
:10C9C0001A4603F096F8601CC4B2052CE7DB294830
:10C9D00090F8840033283CD1264890F8850001283F
:10C9E00037D102F025FCA0B30424002004EB44015D
:10C9F000062202EB41010DF8010004EB440107227D
:10CA000002EB41010DF8010004EB4401082202EBA6
:10CA100041010DF8010004EB4401092202EB410140
:10CA20000DF801001D210DF1050001F091F90746F7
:10CA3000381204EB44010A2202EB41010DF8010017
:10CA4000F8B204EB44010B2202EB41010DF80100A6
:10CA500000BF2946684600F013FD00BF681CC5B240
:10CA60000348007AA84293DC10B0BDE8F0810000D2
:10CA700088200020EC03002010B58AB0154800780B
:10CA800010B900200AB010BD002012490870202003
:10CA90008DF80000104881690DF1010088471A20C7
:10CAA0008DF8050001208DF806000C480068CDF8CF
:10CAB00007000949886A80478DF80B000649086B12
:10CAC0008047044604482146426B6846904701204F
:10CAD000D8E7000030050020380300203105002091
:10CAE00010B51A48007A1949C97900EB012084B2BF
:10CAF000601C84B220121549C8710846047205F002
:10CB00007BF813480078401CC0B2114908701928FE
:10CB100019DB002008700F4890F8800038B10E48EB
:10CB2000407820B10C484078401E0B4948700B48B3
:10CB3000807828B90A48806A401C0949886202E066
:10CB400000200749886204F033FD10BD68170020FB
:10CB5000D7030020EC030020B90300209017002029
:10CB6000F8060020704710B500F09EFB06F074F93F
:10CB700010BD000010B50020064988700022052174
:10CB80000448C01C02F0C0FF0020034981F82000C7
:10CB900010BD000090170020F806002010B500F02E
:10CBA00099F803F04BFA06F04BF900F06FF800F03B
:10CBB00031F8034908688047FEF79EFE10BD00006B
:10CBC0008405002010B500F030F802F095FEFEF765
:10CBD00061FE0548807D28B100200349887503491E
:10CBE000C86E804710BD0000F8060020EC0300204E
:10CBF00010B50749086A8047032804D00449086A29
:10CC00008047062801D1012010BD0020FCE700006C
:10CC10003803002010B502F09DFE05F0B1F802F0D7
:10CC200065FC012000F0F0F910BD00B591B0684638
:10CC300003F0B8FF08B911B000BD9DF801006028ED
:10CC400003D09DF80100612809D19DF8020030B1A0
:10CC500001F0B8FF9DF80210884200D0EBE704F025
:10CC60008DFA9DF80100602803D1684603F0ACFC02
:10CC70000AE09DF80100612803D1684603F028FE10
:10CC800002E0684603F078FF00BFD4E710B503F078
:10CC9000A3FF05F081F810BD70B5C0B005460E4683
:10CCA0001446601CC2B20A486946436A284698473F
:10CCB0009DF80000F52808D1224631460DF101000B
:10CCC00002F017FF012040B070BD0020FBE700001C
:10CCD000B802002010B5C0B00D226946C020FFF791
:10CCE000DBFF88B10D22BA49684602F002FF0D222F
:10CCF000B849684602F0FDFEB7480C21D0F80C2177
:10CD0000B448401C904710E00120B149491E4870CA
:10CD100000220C21AE48401C02F0F6FEAE480C2169
:10CD2000D0F80C21AB48401C9047FFF799FB032239
:10CD300069464FF48560FFF7AFFF80B10322A74932
:10CD4000684602F0D6FEA54A521ED378927803EBCD
:10CD5000022290B2A04AD2F80411884704E09E480B
:10CD6000D0F8041100208847072269460020FFF709
:10CD700093FF28B107229A49684602F0BAFE1EE0E6
:10CD80000121974A521E5170917011460979D2784B
:10CD900001EB022188B201200112914A521ED1708A
:10CDA000114608718979527901EB022188B201207C
:10CDB00001128B4A521E51711146887100BFFFF754
:10CDC0003DFBFFF703FB0D2269460820FFF764FFD8
:10CDD00028B10D228349684602F08BFE05E0FF2250
:10CDE00006218048C01C02F08FFE04F059FD042289
:10CDF00069461820FFF750FF28B104227A49684697
:10CE000002F077FE04E0FF220421774802F07CFE66
:10CE1000062269463020FFF73FFF28B106227349FA
:10CE2000684602F066FE0AE000207049491E48701C
:10CE30004870C87008710A204871082088711A2249
:10CE40006946A020FFF728FFE0B11A22684968462A
:10CE500002F04FFE604890F8C400C0B16448401E24
:10CE600080780E2813D16248401EC07814280ED155
:10CE70005949D1F8D400804748B901205D4981F86B
:10CE8000200004E000221A21594802F03DFE082249
:10CE900069464020FFF700FF60B1002055498885B2
:10CEA0009DF80000402811D0684600F023FE51494B
:10CEB00088850BE00924224669464F4802F019FE96
:10CEC00022466946402000F06DFC00BF04226946FE
:10CED000D020FFF7E1FE28B104224849684602F05D
:10CEE00008FE04E000220421444802F00DFE032263
:10CEF0006946D820FFF7D0FE28B103224049684692
:10CF000002F0F7FD06E001203D49491E487000206F
:10CF10008870C87006226946F020FFF7BDFE48B34E
:10CF200006223849684602F0E4FD2B4890F882005A
:10CF300028B1294890F882003249491E887031484A
:10CF4000401E807820B12F48401E8078042803DDE1
:10CF500001202C49491E88702A48401EC07820496B
:10CF6000491E8978884219D01D49491E887804F0E5
:10CF70002BFD13E0184890F8820030B1164890F865
:10CF800082002049491E887003E001201D49491E86
:10CF900088701349491E887804F016FD01226946FD
:10CFA0004FF4A070FFF778FE20B19DF80000114902
:10CFB000C8750AE0084890F8850018B101200D49AD
:10CFC000C87502E000200B49C87540B010BD0000D4
:10CFD000F517002003180020EC030020C8030020F0
:10CFE000AD030020E7170020B503002069170020DB
:10CFF00091170020F806002078350108A7030020CB
:10D00000BC030020C00300200149087070470000E5
:10D010007C20002030B58BB000F014FE08B10BB0BE
:10D0200030BD02F063FA20208DF804000DF10500F8
:10D0300001F0DAFD10208DF8090001F0C3FD8DF834
:10D040000A00A5208DF80B0001F0C8FD8DF80C003A
:10D05000554840798DF80D00534880798DF80E00C1
:10D0600008220DF10F01514802F043FD4F48401EC8
:10D07000C07800F00F008DF8110001F0A9FD022822
:10D0800003D001F0A5FD052805D19DF8110040F061
:10D0900080008DF811004648007820B1012815D095
:10D0A000022837D120E001208DF817000C2206A9B4
:10D0B000404802F01EFD404890F884001E2801D12F
:10D0C000012000E002203A49087027E003208DF893
:10D0D0001700092206A9394802F00BFD34480078F0
:10D0E000401C3349087019E002208DF817003448BD
:10D0F00040788DF818003348007A8DF81900042222
:10D100000DF11A012F48001D02F0F3FC0020284900
:10D11000087003E000202649087000BF00BF00240B
:10D1200035E02848C07AA04200D12EE001F0F6FD9B
:10D1300020B12448001D005D8DF80C001E4890F8B9
:10D1400084001E280CD01C4890F88400332817D186
:10D15000194890F88500012812D102F069F878B1D9
:10D160001A210DF1090000F0F3FD054628128DF893
:10D170002300E8B28DF8240020208DF8040000BFC1
:10D18000214601A800F07CF900BF601CC4B20D4824
:10D19000007AA042C5DC03200B49087000204870CB
:10D1A000887000BF3BE70000AC0300206917002037
:10D1B000D1030020F6170020EC0300200507002013
:10D1C000BF030020882000207C20002010B588B0FC
:10D1D0001F208DF80000134881690DF10100884778
:10D1E00010208DF8050001F0EDFC8DF806001822E6
:10D1F0000DF107010C4802F07CFC002405E02146FB
:10D20000684600F03DF9601CC4B20848007AA042AC
:10D21000F5DC03200649087000204870887008B0CB
:10D2200010BD00003803002078170020882000205F
:10D230007C20002030B589B004461F208DF8040002
:10D24000154881690DF10500884733208DF80900E4
:10D2500034B917220DF10A01104802F04AFC05E02A
:10D2600017220DF10A010E4802F043FC01F0B6FC52
:10D270008DF8230001F058FD0546294601A800F06D
:10D28000FFF803200749087008464078401C4870A2
:10D290000020887009B030BD38030020CF1700206F
:10D2A000111800207C20002010B502F025FE7048E7
:10D2B000007800B910BD6E480078082879D2DFE800
:10D2C00000F0D20412153A576AA701F081FC032836
:10D2D00006DD684890F87A0010B100F031F901E0FD
:10D2E000FFF798FEC0E000F02BF9BDE060488078C1
:10D2F000401CC0B25E4988700A2813DA5D48D0F835
:10D30000F410012088475B48007850B101F060FCC0
:10D31000082803D001F05CFC092802D155490869AE
:10D320008047A1E05348D0F8F4100020884704203B
:10D330004F49087098E001F04BFC032805DCFFF72B
:10D34000B7FA06204A49087011E001F041FC0328B1
:10D3500007DD484890F87A0018B10120FFF78EF9F0
:10D3600002E00120FFF7FEFA0520414908707BE04A
:10D3700001F02EFC032807DD3E4890F87A0018B132
:10D380000220FFF77BF902E00220FFF7EBFA06200C
:10D390003749087068E002F0C9FE03F09FFB48B10E
:10D3A00000203349487208723348486007200870EB
:10D3B0002DE058E02F4890F8340068B12D49486CB2
:10D3C000804748B100202A49487208722948C06B3A
:10D3D0004860072008701AE001F0FAFB032803DD1B
:10D3E000244890F87A0048B921484078022805DBA3
:10D3F00000201F494870FFF70DFE08E002F01AFDFB
:10D4000010B900F09DF802E00020FFF7FDFD2BE0D1
:10D4100017494868804770B11548407A401C144944
:10D4200048720846407A50281CDB012013490870D6
:10D430000F49087016E00E49097A491C0C4A11720E
:10D440000C4991F884101E2901D1142000E05020CD
:10D450000749097A814204DB0121084A1170044A14
:10D46000117000BF00E000BF00BF00BF22E7000056
:10D470007C200020EC030020DD0A0108D1030020FD
:10D4800030B591B005460C462878401CC2B26946BA
:10D49000284602F02EFB124890F87E0060B19DF8FD
:10D4A0000000001FC0B28DF800009DF800200DF1B3
:10D4B0000101081D02F01DFB0A49085D04F0F8F89F
:10D4C0000748D0F8A410684688470648025D9DF8D2
:10D4D00000100548836A0DF10100984711B030BD76
:10D4E000EC03002088200020B802002010B590B086
:10D4F0000446F5208DF80000AA208DF801008DF873
:10D5000002002078401CC2B20DF10301204602F057
:10D51000F0FA9DF80320D21CC2F14002D1B29DF86E
:10D5200003206B461A44D01C002202F0EDFA034897
:10D53000402182696846904710B010BDB8020020B3
:10D5400030B58BB000F096FB08B10BB030BD01F0E8
:10D55000CDFF8B48D0F8D01000208847012800D19B
:10D56000F3E700F0C9FD87484079401C85494871C0
:10D5700008464079072801DD002048718249886803
:10D58000804780B18148007880F001007F490870B1
:10D590000846007820B17C494868804700B1D4E74C
:10D5A000072078494871764890F87F0040B1744868
:10D5B00090F87F0000287DD07548C0780028FAD008
:10D5C00020208DF804000DF1050001F00DFB01F0A5
:10D5D000FFFA032801DC132000E014208DF8090075
:10D5E00001F0F6FA032806DD654890F87A0010B1DC
:10D5F00017208DF809006748C0798DF80A00654842
:10D60000007A8DF80B001A2203A9634802F071FA20
:10D610005B48007878B101F0DBFA082803D001F00C
:10D62000D7FA092807D15C48401E807840F04000B6
:10D630008DF80D0006E05848401E807820F040002C
:10D640008DF80D004E48016A01A8884720B14C4969
:10D65000D1F8B000804770BB01F0BAFA032841DD71
:10D66000474890F87A0038B317208DF80900042253
:10D670000DF121014348401C02F03BFA414840793A
:10D680008DF8200001F0A4FA052801D1012000E066
:10D6900000203C49497808438DF8210039488078BA
:10D6A0008DF8220001F09AFA8DF82300344890F8A2
:10D6B000840002E059E01CE014E0282804D030483F
:10D6C00090F88400292808D11B210DF1090000F0F1
:10D6D0003FFBC0B28DF824000BE02A4800798DF89A
:10D6E000240006E0A5208DF8210001F077FA8DF8DE
:10D6F0002200002435E02948C07AA04200D12EE063
:10D7000001F00CFB20B12548001D005D8DF82200C2
:10D710001B4890F884001E280CD0194890F884000B
:10D72000332817D1164890F88500012812D101F04E
:10D730007FFD78B11A210DF1090000F009FB0546C3
:10D7400028128DF82300E8B28DF8240020208DF8EF
:10D75000040000BF214601A8FFF792FE00BF601C35
:10D76000C4B20E48007AA042C5DC03200C49087000
:10D7700008464078401C48700020887000BFE4E6EE
:10D78000EC030020A603002084050020D60300201F
:10D79000BB0300206817002091170020882000207C
:10D7A0007C20002070B5C0B006460C461546F5201A
:10D7B0008DF800002A460DF10101204602F099F98A
:10D7C000681CC2B203486946036A30469847012084
:10D7D00040B070BDB80200200348407808B1012075
:10D7E00070470020FCE70000644600200020034949
:10D7F0004870034908800349088070476446002048
:10D80000100500201205002030B59BB03748407845
:10D81000082866D2DFE800F065040D10393D575B3B
:10D82000324AD078324A516B8847FF202F494870DE
:10D8300058E0FFF7DBFF55E02C4800892B49C988E9
:10D8400000EB01212B480088401C80B2294A10803F
:10D85000814200DC46E020208DF84400002403E0F3
:10D8600011A80455601CC4B2202CF9DB2249C86AF7
:10D870008047054620482946426B11A890471B4A1D
:10D88000907A1B4AD16888472CE000201B49088009
:10D8900028E09DF80400202801D01BB030BD9DF881
:10D8A000050000B1F9E79DF80600012800D0F4E773
:10D8B0009DF80700022800D0EFE710480088401CC0
:10D8C0000E4908800EE000200D4908700AE00D485E
:10D8D000007800B906E00649886B8047084908705F
:10D8E00000E000BF00BF00BFD7E700006446002093
:10D8F000B802002010050020380300201205002087
:10D900001405002015050020114A4368136003899F
:10D910009380837A9371521E52780A700C4A521E79
:10D9200092784A700A4A521E12798A70094A1288FD
:10D930001212CA70074A12780A71074A1288121224
:10D940004A71054A12788A71044A1278CA7170477E
:10D950006546002010050020120500201405002057
:10D96000002107E048F2782100BF0A1EA1F101035F
:10D9700099B2FAD1021EA0F1010398B2F2D1704718
:10D98000002105E01E2100BF0A1EA1F10101FBD10B
:10D99000021EA0F10100F5D17047002105E01E2113
:10D9A00000BF0A1EA1F10101FBD1021EA0F101007E
:10D9B000F5D1704710B504464FF4C8714FF4E150EB
:10D9C000FBF70AFB10BD000070B586B004460020CE
:10D9D00002900390049005903D4800680190012654
:10D9E000E0780B2804D00C2808D00D2864D15DE025
:10D9F0003848A1880180A17981705FE020790128F1
:10DA000002D02079022827D1A079802800DB55E0B8
:10DA10002079401EC5B2217905EB85222D48C01C16
:10DA200000F8121000F6FD708574617905EB85220F
:10DA3000A0F6FD7000EB4200417005EB8522254900
:10DA4000C91C01EB4201891CA27901EB02101022D2
:10DA5000E11DFAF79DFB28E0207900F0800020B35B
:10DA6000A079802800DB29E0207920F08000401E8A
:10DA7000C5B205EB85211748C01C00EB410040787A
:10DA80008DF80500A0798DF8060005EB8522114878
:10DA9000C01C00EB4200801CA27900EB0211102296
:10DAA0000DF10700FAF774FB132607E00A486168D6
:10DAB0000160A168416001E0002600BF00BF2EB1F7
:10DAC000E178334601AA602005F040F806B070BD49
:10DAD000C8350108174F00201E5F0020014604488A
:10DAE0008078401E132202EB4010C0B27047000045
:10DAF0005097002010B5024600230024002108E0C2
:10DB0000505C1844C3B2081D105C2044C4B2481CC9
:10DB1000C1B20429F4DB83F0A50384F0A50403EB70
:10DB2000042080B210BD0000014601F10800C0B21F
:10DB30000246044B93F87530984201DD012070478E
:10DB40001046FCE7EC03002010B50146132901DC68
:10DB5000012012E0A1F11303D81703EBD0604011AC
:10DB6000401C1A46D41702EBD4646411A2EB44148F
:10DB70000CB1012400E000242044C0B210BD0146D5
:10DB800009B9002003E0481E132202EB4010C0B286
:10DB9000704702461320704710B50146002000234D
:10DBA00014E04FF6FF7404EA83028C5C4CB9541CF9
:10DBB0000C5D34B9941C0C5D1CB9D41C0C5D04B90B
:10DBC00002E0441CE0B200BF5C1CA3B20A2BE8DBFD
:10DBD00010BD00000C480078401CC0B20A49087013
:10DBE000FA2801DA0020704700200749087008462B
:10DBF00040782D2803DB002048700120F3E7002047
:10DC0000014948700220EEE7290500200448007809
:10DC100020B10348007908B1012070470020FCE7DB
:10DC200018050020064890F87500401CC0B2044951
:10DC300081F87500012801DB012070470020FCE716
:10DC40005097002010B501F069F808B9002010BD08
:10DC50000748007880F00100054908700846007800
:10DC600018B1FFF7B3FA0120F1E70020EFE7000059
:10DC7000D203002010B5244890F8210080B3234837
:10DC8000007880F001002149087048B31E4890F8E0
:10DC90002300A0B11C4890F8240080B11C480078F3
:10DCA00018B90020FFF7C6FA02E00120FFF7C2FA18
:10DCB0001748007880F00100154908700EE01248FE
:10DCC00090F8230018B10020FFF7B4FA06E00E48E0
:10DCD00090F8240010B10120FFF7ACFA012010BD2C
:10DCE000FFE7094890F8220060B10A48807848B9F7
:10DCF0000020054981F8220081F8210081F82300E5
:10DD000081F824000020EAE7F8060020D403002070
:10DD1000D5030020901700200020014908707047AB
:10DD2000800500200246002107E00748405C904241
:10DD300001D108467047481CC1B20348407A884266
:10DD4000F3DCFF20F6E70000882000207047000089
:10DD500070B5024600201CE003134FF6FF7404EA7E
:10DD600000101478E51704EB157583EA25150C4EA1
:10DD700036F81550684003134FF6FF7404EA00109C
:10DD8000147804F00F045C40354635F814406040C8
:10DD9000521C0C1EA1F10105A9B2DDD170BD00001D
:10DDA000DC3801087047000070B505460E46D5F80E
:10DDB000B040012E18D12078F52805D16078AA2826
:10DDC00002D1A078AA2802D02046FFF7BFFF00208A
:10DDD00003F0ACFD0548C16CE01C88474023224697
:10DDE0000121284604F01DFA70BD00003803002010
:10DDF00070B504460D468121204604F09BF90121AF
:10DE0000204604F097F9002070BD000070B504466C
:10DE10000E4643211B48FAF7E2F91B4B4FF4A07260
:10DE20000021204604F0ECF9174BDB1D4FF4807203
:10DE30000021204604F0E4F94023124A0121204643
:10DE400004F0EFF911488169C4F88810C169C4F879
:10DE500084100C48C4F8B000D4F8B40078B10025A0
:10DE60000BE0D4F8B40050F8250020B1D4F8B41079
:10DE700051F825008047681CC5B2042DF1D300205D
:10DE800070BD0000B4060020D10000208C020020EC
:10DE9000024619B1C2F8B410002070470220FCE716
:10DEA00070B506460C4615462B4622468121304663
:10DEB00004F03AFA002070BD2DE9F04105460C4609
:10DEC0000127D5F8B06060780C2865D2DFE800F053
:10DED000642D394364640664644D595F608822216F
:10DEE000B1EB202F0ED1E088202801D9202000E0BE
:10DEF000E088024600232B4905F1440004F04AF86B
:10DF0000002711E060882121B1EB202F0CD1E0889F
:10DF1000092801D9092000E0E088024600232249AF
:10DF200005F1440004F036F837E0E088022807D114
:10DF300000230222314605F1440004F02BF80027AB
:10DF40002BE00023012206F1410105F1440004F019
:10DF500021F8002721E00023012206F1420105F10A
:10DF6000440004F017F8002717E0A07886F8400076
:10DF7000E2880023314605F1140004F00BF8002775
:10DF80000BE06088001286F84100002705E0A078C9
:10DF900086F84200002700E000BF00BF3846BDE819
:10DFA000F0810000F4340108C800002010B5002002
:10DFB000002126E000220CE001EBC10303EB01137A
:10DFC000114C23449B5CFF2B01D040F00100531CFB
:10DFD000DAB20E4B1B789A42EEDB0D4B33F8114050
:10DFE0000A4B1B78B4EBC30F07DB0A4B33F8114025
:10DFF000064B1B78B4EBC30F01DA40F002004B1C58
:10E00000D9B22829D6DB10BD28070020A4030020A0
:10E01000C81600201817002030B500220023C1F3D5
:10E02000C70201F00703845C01259D402C43845402
:10E0300030BD00002DE9F04105460E4690461A49D4
:10E040000868C11700EBD1614911184A11601046E8
:10E050000068801D16490860102001F003FD074686
:10E0600010213846FAF7BBF8002403E0305D11496F
:10E070000855641C0D480068B4EB800FF6DB0024E3
:10E0800003E0285D0C490855641C102CF9DBFBF7F4
:10E09000A3FBFBF709FA102208493846FAF778F88B
:10E0A0003846BDE8F0810000A4050020A00500204E
:10E0B0009C05002038990020CC970020DC97002098
:10E0C00010B50A48007978B9084890F8060858B998
:10E0D00000210748C1730749886E80470548816B56
:10E0E00001208847012010BD0020FCE7174F0020C9
:10E0F000175F00203803002010B50C480078401C42
:10E10000C0B20A4908700A280ADD084600780C28BF
:10E1100001DD002008700648816D0120884703E07A
:10E120000348816D0020884710BD0000D303002004
:10E13000B802002070B50446A01CFDF754FD051E72
:10E1400011D095F86400617A88420CD1B5F86C6002
:10E150006978284600F0A8F820B1627AA11C012055
:10E1600000F00AF900BF70BD30B59DB00546687873
:10E170001E490978884201D11DB030BD68781B491D
:10E180000870022400BF285D052800DA2BE0285D16
:10E19000401FC0B28DF86300601C284400681990CD
:10E1A000601D285C8DF868005D210DF10600FAF70E
:10E1B00016F89DF86320A01D29180DF10600F9F747
:10E1C000E7FF00F071FD1B900020ADF8700001A882
:10E1D000FDF726FD01A8FDF7EAFC285D401C204460
:10E1E000C4B200BFCFE700BF00BFC5E78005002075
:10E1F000F0B589B004460D4624216846F9F7EFFFD3
:10E2000020208DF80000264881690DF10100884723
:10E2100037208DF8050094F8600001066120005D4C
:10E2200001EB00416220005D01EB00216320005DF5
:10E23000084418B1206ECDF8060002E00020CDF8A9
:10E2400006008DF80A5094F864008DF80D0094F8DB
:10E250005F000021FFF79DFC07463A46A11C0DF127
:10E260000E00F9F795FF2846FFF738FC07463946B8
:10E27000A01CFFF76DFD064630128DF80B00F0B2C2
:10E280008DF80C0000F052FD07469DF8001005487F
:10E290003A46836A0DF10100984709B0F0BD0000CD
:10E2A00038030020B802002070B504460D46FF2058
:10E2B00020702946024800F0C1FB0646304670BD7A
:10E2C0007405002010B504462146024800F0E0FB2A
:10E2D00010BD00007405002010B5024800F0EAFBF4
:10E2E00010BD000074050020034804490860486020
:10E2F00000200881704700006C0500207405002094
:10E30000002008E0FF21C0EBC002044B03EB021227
:10E310001170411C88B26428F4DB7047906B0020B8
:10E3200070B504460D462A462146024800F0C6FB59
:10E3300070BD000074050020002116E0C1EBC10093
:10E340000C4A02EB00100078FF280CD10120C1EB31
:10E35000C102084B03EB02121070C1EBC1001A4658
:10E3600002EB00107047481C81B26429E6DB0020F4
:10E37000F8E70000906B002070B590B006460C46A0
:10E3800015460EB1022000E001208DF80000206843
:10E39000CDF801000020ADF805008DF807008DF8DC
:10E3A000085009216846FAF78BFE10B070BD0000D6
:10E3B0002DE9F0413D48806F401C3C4988670024AE
:10E3C000084690F8740020B1012819D0022867D1BE
:10E3D00032E0FFF781FF00B963E000F04DFA00B9C9
:10E3E0005FE00020314981F87500084680780128F7
:10E3F00001DD022000E001202C4981F8740000BFFB
:10E400002A488178001DFFF7F3FE01202749C870D4
:10E4100008468078012803DD022081F8740009E0B5
:10E42000FFF700FC012801D0012000E000201F4977
:10E4300081F87400012434E01C48C078401C1B495A
:10E44000897888422BDC00F071FC0646174AD178A7
:10E4500092F86300FFF79DFB07461449C878FFF761
:10E460008EFB01461148801D0D1811483246394671
:10E47000836A284698470D48C078401CC0B20B49B3
:10E48000C8708978884209DBFFF7CCFB012801D0EE
:10E49000012000E00020054981F87400012400E01B
:10E4A00000BF00BF2046BDE8F0810000509700206B
:10E4B000B802002033B581B00D460122694601A89B
:10E4C000FAF7B6FF044614B99DF800003EBD0020DF
:10E4D000FCE72DE9F04104460D46164698463246C3
:10E4E00029462046FAF7A4FF074617B90120BDE8E0
:10E4F000F0810020FBE7002107E048F2782100BF0F
:10E500000A1EA1F1010399B2FAD1021EA0F1010382
:10E5100098B2F2D1704700002DE9F04105460E4651
:10E5200019490868C11700EBD1614911174A1160F8
:10E5300010460068801D1649086010460068870074
:10E54000102001F08FFA804610214046F9F747FE6F
:10E55000002403E0305D0F490855641CBC42F9DB20
:10E56000002403E0285D0C490855641C102CF9DBDD
:10E57000FBF732F9FAF736FD102208494046F9F761
:10E5800007FE4046BDE8F081A4050020A00500205C
:10E590009C05002038990020CC970020DC970020B3
:10E5A00010B52C4B1B6883432A4C2360231D1B682A
:10E5B0008343241D2360231D1B688343241D236084
:10E5C000231D1B688343241D236011B101290ED133
:10E5D00005E0204B1B6803431E4C236008E01D4BE5
:10E5E0001B1D1B6803431B4C241D236000E000BF60
:10E5F00000BF22B1012A0FD0022A27D119E0154B02
:10E6000008331B680343134C08342360231D1B6825
:10E610008343241D23601AE00E4B08331B68834399
:10E620000C4C08342360231D1B680343241D236006
:10E630000DE0084B08331B680343064C0834236085
:10E64000231D1B680343241D236000E000BF00BF9F
:10E6500010BD00000004014001490860704700003F
:10E660001404014001460748006800EA0102054819
:10E670001438006800EA010312B10BB101207047A1
:10E680000020FCE71404014070B504466079282896
:10E6900019D1A07900B970BD012015490870607AC0
:10E6A000217A00EB012012494880A079012802D18B
:10E6B0000020487002E051200D4948700D49D1F802
:10E6C000A000804712E00A48007878B1002008498D
:10E6D00008700949C86A804705460749886A804723
:10E6E000064606482946C26A3046904700BFD2E730
:10E6F00018050020EC03002038030020B802002099
:10E7000070B504462848007808B9002070BD274835
:10E710000078B8B92649C86A804705462249487832
:10E720002449CA6A294690470120A0722049886A74
:10E730008047E0721C484088001220731A48807895
:10E74000607323E01A49C86A804706461849886AF8
:10E750008047054617483146C26A28469047164802
:10E7600090F87A0068B10120A0721149886A804748
:10E77000E0720D484088001220730B488078607367
:10E7800004E00020A072E072207360730A48D0F8A1
:10E790009C10204688470548007880F00100034916
:10E7A00008700120B2E70000180500201E050020B7
:10E7B00038030020B8020020EC03002008B50F2029
:10E7C0008DF80000044800798DF8010002226946A6
:10E7D0000B2000F003F808BD1805002070B590B0BC
:10E7E00004460D46164640216846F9F7F8FC1F20FE
:10E7F0008DF80000E1208DF801000949C8698047C3
:10E800008DF802008DF803403246294601A8F9F739
:10E81000BFFC0348416C6846884710B070BD0000DB
:10E82000380300204179014A117170471805002012
:10E8300001480078704700001805002001460D4887
:10E84000007808B9002070470A48408800280EDD8B
:10E8500048780A7800EB0220064A5288904206D196
:10E8600004484088401C034A50800120EBE7002008
:10E87000E9E700001805002070B50025002470218C
:10E880003348F9F7ACFC00203149091F8870C87083
:10E8900000BF2F49091F4878FFF714FD041E43D01D
:10E8A00000F002FAA16E884204D300F0FDF9A16ED7
:10E8B000401A03E000F0F8F9A16E081A0646B6F512
:10E8C000967F0CD304F16000FDF760F958B394F81B
:10E8D000642004F160010020FFF74EFD23E0702268
:10E8E00021461B48F9F754FC94F85F00FFF72CF918
:10E8F0001749091F88700120C870B4F86C00401CCB
:10E90000A4F86C00FFF7E8FC1149091F4978491C7D
:10E91000C9B20F4A121F5170884202DC0020114612
:10E920004870012511E000BFFFF7D6FC0849091F18
:10E930004978491CC9B2064A121F5170884203DC4B
:10E9400000201146487000E0A3E700BF284670BDD4
:10E950005497002010B5002821D0114B0022001F31
:10E96000196803E0814203D80A4649680029F9D1B1
:10E9700052B11368841A9C4204D100681844106094
:10E98000104602E0506000E0186039B102680B1ACE
:10E99000934203D10B681A4402604968416010BD7C
:10E9A000F00500207FB5044626796579B54200DD83
:10E9B0007FBD012D03D100201E49C1F800041D4870
:10E9C000D0F800043330B0F5806F03D3002019492C
:10E9D000C1F800041749D1F80014164A88183322E8
:10E9E00004F10801F9F7D4FB1248D0F800043330E1
:10E9F0001049C1F8000420798DF8000060798DF885
:10EA00000100A0798DF80200E0798DF8030004215F
:10EA1000684601F02BFFB5420AD10648007801286C
:10EA200004D10548C1680348884700E000BF00BF23
:10EA300000BFBDE760420020840500202DE9F041C1
:10EA400004460E462089B04202DA0020BDE8F0817B
:10EA50000E49086880472568002002E06D68411C67
:10EA600088B2B042FADB6F68686840686860D7F8BF
:10EA700000803846FFF76EFF208910B12089401EC4
:10EA800020810249486880474046DFE7B8020020FD
:10EA900010B502461089884201DA002010BD1068C6
:10EAA0004368002002E05B68441CA0B28842FADBA5
:10EAB0001868F3E701460889704700002DE9F04126
:10EAC0000546884617462889B84202DA0020BDE884
:10EAD000F081134908688047082000F0C3FF04460E
:10EAE00004E00F49486880470020F0E7002CF8D088
:10EAF00000206060C4F800802E6800BF02E07668E5
:10EB0000411C88B2B842FADB7068606074600449E6
:10EB1000486880472889401C28810120D7E70000E9
:10EB2000B802002010B520211448F9F758FB202224
:10EB3000134912482030F9F72BFB00240AE00F4854
:10EB40002030005D0F49095D48400C4920310855CF
:10EB5000601CC4B2202CF2DB0023084A3032074983
:10EB600001F12000FAF75CFB0023044A2032A2F1F5
:10EB7000100101F12000FAF753FB10BDD74E002021
:10EB800081350108CC35010801460148405C7047D9
:10EB9000CC36010810B50446202202492046F9F778
:10EBA000F7FA10BDF74E0020044890F8900008B91D
:10EBB0000020704702480078FBE70000EC030020CB
:10EBC000D44E00200148407870470000AC0300207C
:10EBD0000148407870470000F41700200148007990
:10EBE000704700008820002010B504460B4840788C
:10EBF000032803D009484078062808D1AA202070AD
:10EC0000BB206070CC20A070DD20E07004E0042206
:10EC10002146034800F06DFF10BD0000F4170020EE
:10EC2000B503002001480078704700007C200020D8
:10EC300017488078282803D104201649C87224E098
:10EC40001348807810280FD11248C07A032807D0C3
:10EC50001048C07A022803D002200E49C87214E07E
:10EC600003200C49C87210E00948807818B10120CF
:10EC70000849C87209E00648807818B90520054996
:10EC8000C87202E000200349C8720248C07A704787
:10EC900090170020F8060020042101700221417025
:10ECA00000218170704700000148806F70470000AC
:10ECB0005097002010B5054890F8740020B9FFF770
:10ECC0000BFB08B9002010BD0120FCE75097002085
:10ECD00001484078704700009017002030B5014689
:10ECE0000022002010E00B4C235C03EB43040A4D90
:10ECF00005EB4404A478082C04DD441CE5B2541C44
:10ED00000D55E2B2441CE0B2024C647A8442EADC63
:10ED10000A7030BD8820002038210020014800788A
:10ED200070470000D00300200020704701480078A1
:10ED30007047000088200020014601EB8100400060
:10ED400070470000F0B503460C4606251F201E78CC
:10ED50001D2E46D2DFE806F0450F1C1E2124274554
:10ED600045452A2C2F3145454545454534383C45D8
:10ED70004545454041001E4EB67806F07F06052EFB
:10ED800003D1042107261E7001E0082103252BE092
:10ED9000042129E002210C2526E00121172523E08A
:10EDA0000221092520E0012115251DE004211BE099
:10EDB0000121162518E0042116E002210B2513E09D
:10EDC000032110253C200FE0032110253C200BE0FF
:10EDD00001211B253C2007E000BF02211A253C2011
:10EDE00002E00121162500BF00BF21701570F0BDA3
:10EDF000901700200148007870470000F8060020B6
:10EE00000148007970470000F80600200348017BA4
:10EE10000020024A1073084670470000F8060020E0
:10EE20001EB50146002009E083061A0E084B134464
:10EE3000D3F8E8374DF82030431CD8B20328F3DB71
:10EE4000009B0B60019B4B60029B8B601EBD000012
:10EE500000F0FF1F014800787047000030030020D9
:10EE600000BF04488078052801D1012070470020A8
:10EE7000FCE70000F80500200248C07A0149085C60
:10EE80007047000088200020416170470161704791
:10EE900010B54FF4807303221021024800F050F89F
:10EEA00010BD00000008014010B500228B071C0FA8
:10EEB0000F2303FA04F204290EDA204B9B689343D4
:10EEC0001E4CA36023469B688C07240F00FA04F4B1
:10EED00023431A4CA3602FE008290EDA174BDB6896
:10EEE0009343164CE3602346DB688C07240F00FA3B
:10EEF00004F42343114CE3601EE00C290EDA0F4B9F
:10EF00001B6993430D4C236123461B698C07240F17
:10EF100000FA04F42343094C23610DE0074B5B69BD
:10EF20009343064C636123465B698C07240F00FA08
:10EF300004F42343014C636110BD00000000014054
:10EF4000F0B5044616460025002201F00F0501F039
:10EF5000100747B1042E05D145F00305E76B1F43A9
:10EF6000E76300E0354300201EE0012787401F4093
:10EF7000C7B122684FEA800C0F2707FA0CF7BA4393
:10EF8000870005FA07F73A43282904D1012787406B
:10EF90001F40676105E0482903D1012787401F40D2
:10EFA00027612260471CB8B20828DED3082022E07F
:10EFB000012787401F40E7B16268A0F108074FEAC8
:10EFC000870C0F2707FA0CF7BA43A0F10807BF0018
:10EFD00005FA07F73A43282904D1012787401F4043
:10EFE000676105E0482903D1012787401F40276159
:10EFF0006260471CB8B21028DAD3F0BD02469068B0
:10F00000084008B1012070470020FCE7002101E022
:10F010004A1C91B28142FBDB7047000070B50024AE
:10F02000FBF7D6F900251BE06006040E4FF4807153
:10F030001A48FFF72BFF0520FFF7E8FF4FF4007198
:10F040001648FFF7DBFF08B144F001044FF480716C
:10F050001248FFF719FF0520FFF7D8FF681CC5B25B
:10F06000082DE1DBFBF7CCF94FF400710B48FFF7FB
:10F070000BFF0520FFF7CAFF4FF480710748FFF729
:10F0800005FF0520FFF7C2FF4FF480710348FFF72B
:10F09000FBFE0520FFF7BAFF204670BD000C0140C3
:10F0A00070B50546FBF7ACF9002427E005FA04F03B
:10F0B00000F0800040B14FF400712848FFF7E6FEF1
:10F0C0000520FFF7A3FF07E04FF400712348FFF787
:10F0D000DBFE0520FFF79AFF4FF480711F48FFF712
:10F0E000D5FE0520FFF792FF4FF480711B48FFF714
:10F0F000CBFE0520FFF78AFF601CC4B2082CD5DBCD
:10F10000FBF766F94FF480711448FFF7BFFE052046
:10F11000FFF77CFF002413E04FF400710F48FFF766
:10F120006DFF58B94FF480710C48FFF7ADFE052014
:10F13000FFF76CFFFBF764F9012070BD601CC4B2DF
:10F14000642CE9DB4FF480710448FFF79DFE052035
:10F15000FFF75CFFFBF754F90020EEE7000C0140DD
:10F1600010B54FF400710F48FFF790FE0520FFF730
:10F170004DFF4FF480710B48FFF788FE0520FFF725
:10F1800045FF4FF400710748FFF77EFE0520FFF7AB
:10F190003DFF4FF480710348FFF776FE0520FFF72F
:10F1A00035FF10BD000C014010B54FF400710F4841
:10F1B000FFF76AFE0520FFF729FF4FF480710B4827
:10F1C000FFF764FE0520FFF721FF4FF400710748A9
:10F1D000FFF75CFE0520FFF719FF4FF4807103482D
:10F1E000FFF752FE0520FFF711FF10BD000C014094
:10F1F00030B50B46002100BF16E00A24B4EB107FA7
:10F2000005D9302404EB107403F8114005E04124C3
:10F2100004EB10740A3C03F81140000100254C0077
:10F22000641C1D554C1CE1B29142E6DB30BD7047B9
:10F2300010B50849D1F8B000804708B1002010BDD2
:10F24000044890F8850008B90020F8E70248C07D1E
:10F25000F5E70000EC030020F8060020F0B591B0BF
:10F2600004460F46474890F8800028B14648407849
:10F2700010B9002011B0F0BDA0780C2807D1607A39
:10F28000042804D13F48D0F8D010012088473D48D9
:10F29000007808B3FFF79CFC082803D0FFF798FC20
:10F2A000092819D1374890F87F0010B13748C07845
:10F2B00020B13749086A8047082806D13148C1681B
:10F2C000E01C884708B90020D4E72E484169204651
:10F2D000884708B10020CDE7A078042805D116267C
:10F2E00025781B2D15DD1B2513E0A078092802D1F8
:10F2F0001C261B250DE0A078072802D0A07808283E
:10F3000002D11B261B2504E015262578102D00DDD3
:10F3100010258DF804602A460DF10501A01C00F0AF
:10F32000E8FB607C012814D11649D1F80001804720
:10F33000227CE17B02EB0121884204D01149D1F803
:10F340000001804758B901A803F0C4FD38B9002076
:10F3500090E701A803F0BEFD08B900208AE73A460D
:10F360000421E01C00F000F908B9002082E72046E3
:10F37000FCF7C2FB0348416A04F10F0088470120F3
:10F3800078E70000EC030020B9030020BB03002055
:10F39000380300202DE9F04391B005460E464FF0AA
:10F3A00003090022402101A800F0AEFB05274FF021
:10F3B00004082879242857D2DFE800F0121C1E2008
:10F3C0002428565656565656565656494E56565652
:10F3D0002C2D2E2F30313233345656565639434465
:10F3E000404880780E2803D10D244FF0090800E032
:10F3F0000A243DE001243BE0022439E04FF00A08F2
:10F40000032435E04FF00708052431E04FF01408DD
:10F4100006242DE000BF00BF00BF00BF00BF00BF3B
:10F4200000BF00BF4FF015080424042720E00C247F
:10F430004FF00308052702208DF807004FF004095C
:10F4400016E000BF4FF004080C24042710E04FF032
:10F4500004080C2404270BE04FF014080B24224866
:10F46000416AA81C884703E0002011B0BDE8F08382
:10F4700000BF8DF80440A8788DF80500E8788DF875
:10F48000060001AA02EB0901E819424600F031FB2F
:10F4900028790F2802D101208DF807002879222829
:10F4A00002D02879232809D19DF807001F2805DB01
:10F4B0009DF807001F38C0B28DF8070001A803F0BF
:10F4C00009FD08B90020D0E72846FCF715FB3246B5
:10F4D0000221A81C00F048F808B90020C5E7012067
:10F4E000C3E7000090170020EC03002070B5002453
:10F4F0001BE0002104EBC40000EB44120E488154D1
:10F5000000250EE004EBC40101EB44120A4911444A
:10F51000491C01EB85000022042100F0F5FA681C6B
:10F52000C5B20A2DEEDB601CC4B203480C38407A29
:10F53000A042DEDC70BD00009420002001468878E7
:10F540000B280AD1487A032807D10548D1F80320AF
:10F5500002600120034A107070470020FCE70000A1
:10F5600031050020300500202DE9F04105460F4609
:10F570001446062F02DD0020BDE8F081042C01DBDB
:10F580000020F9E731490868804704EBC40000EB2C
:10F5900044112F48465C0A2E52DA04EBC40000EBFB
:10F5A00044122B481044401C00EB86013A46284682
:10F5B00000F09FFA274890F87A0050B1297A04EBBE
:10F5C000C40000EB441222481044401C00EB8600AB
:10F5D0000171A87B012825D11E49D1F8000180477F
:10F5E0006A7B297B02EB0121884204D01949D1F8BA
:10F5F0000001804758B90B2104EBC40000EB441212
:10F6000013481044401C00EB860001710AE00A21F7
:10F6100004EBC40000EB44120D481044401C00EB06
:10F620008600017104EBC40000EB44110848405C03
:10F63000401CC1B204EBC40000EB441204488154E6
:10F64000024948688047012096E70000B802002080
:10F6500094200020EC0300202DE9F041064670784C
:10F66000042801DABDE8F0818249086B804728B997
:10F670008048816E701C884700B1F3E77D48D0F860
:10F68000A810701C884700B9ECE73078FEF74AFBF9
:10F690000746FF2800D1E5E7741CFFF7C9FD0028E5
:10F6A00047D06079912808D06079922805D0607998
:10F6B000932802D0607994283BD16E4890F8850059
:10F6C00002280BD1207FE17E00EB012085B21621BC
:10F6D000601DFEF73DFBA8422AD0C3E7654890F8BD
:10F6E0008500032817D1207FE17E00EB012085B241
:10F6F0001621601DFEF72CFBA84219D094F82000BB
:10F70000E17F00EB012085B21A21601DFEF720FB8E
:10F71000A8420DD0A6E794F82000E17F00EB01207D
:10F7200085B21A21601DFEF713FBA84200D099E7AD
:10F7300000BF6079912814D06079922811D0607947
:10F7400093280ED0607994280BD04A4890F8340062
:10F7500038B14848016C2046884710B101F022FDBD
:10F7600080E7444890F87E0048BB6079932802D136
:10F77000A0790E2819D0FFF72BFA032815D0FFF730
:10F7800027FA062811D03B48007838B1FFF720FA55
:10F7900008280AD0FFF71CFA092806D004223649A7
:10F7A000601C00F095F900B95CE72078001FC2B238
:10F7B000611C601D00F09DF92078001F20706078AA
:10F7C000802800DA4EE701F0EDFC6078912804D142
:10F7D00039462046FFF7DEFD49E06078922804D1E3
:10F7E0003946204600F056F841E0224890F87A0069
:10F7F00050B16078932802D06078942804D13946BB
:10F800002046FFF72BFD32E06078B72804D11B4873
:10F810000169204688472AE02078182815D16078A9
:10F82000A178884211D16078E17888420DD1607862
:10F830002179884209D160786179884205D11048E0
:10F840000068401C0E4908600CE70A48D0F8E81030
:10F8500020468847074890F8340028B10548016CD5
:10F860002046884700B1FDE6204600F067F800BF5B
:10F87000F8E60000EC030020B5030020840500201A
:10F88000CC03002010B504462046FFF7E5FE01201A
:10F8900010BD000030B589B004460D46A0780C2894
:10F8A00007D1607A042804D11248D0F8D010012082
:10F8B000884714208DF8040010220DF10501A01CCA
:10F8C00000F017F901A803F005FB10B9002009B0FA
:10F8D00030BD2046FCF710F92A460621E01CFFF750
:10F8E00043FE08B90020F2E70248416AE01D88475C
:10F8F0000120ECE7EC03002010B592B00D49086838
:10F90000804740230A2201A90B4801F02FFA044640
:10F9100008494868804714B9002012B010BD9DF80E
:10F920000400801CC0B28DF8040001A8FDF7DEFDC4
:10F930000120F2E7B80200205821002010B504464B
:10F9400040230A222146024801F0DAF910BD0000E6
:10F950005821002010B541230F220249024801F02E
:10F96000FDF910BD801C0020741C002010B5044659
:10F97000012C04D104210848FFF786FA0AE0022C82
:10F9800004D104210448F9F7D8FC03E0042102481B
:10F99000FFF77CFA10BD00000008014010B50446D6
:10F9A000012C04D102210848FFF76EFA0AE0022C6C
:10F9B00004D102210448F9F7C0FC03E00221024807
:10F9C000FFF764FA10BD000000080140704770475F
:10F9D0004FF40041080300F0CBFD72B601F0F0FADD
:10F9E0001A491B48FEF754FA1A4A1B49184802F0F4
:10F9F000D5FE00F041FDFFF74BFA02F0D5F8F9F71C
:10FA000031FC00BF1248D0F8AC0081680120884763
:10FA100005200F49887000BFF9F7B0FC0F4948680E
:10FA200080470F49D1F89400804762B6FAF700FE8C
:10FA3000FAF754FE00BF064880780328FBD104E0A3
:10FA400006498868804700F02BFAF9E7000000209B
:10FA5000F80500208C0200207C02002038030020E2
:10FA6000EC030020F0B50B30154D20F00701002409
:10FA7000144A0FE003688B420BD38B4205D95E1A00
:10FA800043184768C3E9006700E04368136002C099
:10FA900004E0021D10680028ECD12046002802D1A5
:10FAA000286808B10020F0BD064A07481060074AE0
:10FAB000121A22F00702C0E9002401202860D7E7CB
:10FAC000F4050020F005002014AA002010AE00204C
:10FAD00030B503460C46002107E0585C655CA8423F
:10FAE00001D0002030BD481CC1B29142F5DB01209D
:10FAF000F8E710B50346002003E01C5C0C54441CDE
:10FB0000E0B29042F9DB10BD10B50346002002E0E0
:10FB10001A54441CE0B28842FADB10BD30B591B0F3
:10FB200004460D46402101A8F8F759FB1F208DF827
:10FB30000400E1208DF805000B49C86980478DF865
:10FB400006000A208DF807002A46214602A8F8F789
:10FB50001FFB0549886D804718B10348416C01A817
:10FB6000884711B030BD00003803002000B589B0CF
:10FB70003A4890F8600008B909B000BDFEF72AF8CD
:10FB8000012802D0022865D151E03548C07800280C
:10FB900040D033480079314991F87510884218DD1A
:10FBA00000202F49C87003208DF804002D49886A71
:10FBB00080478DF805004D208DF8060014208DF843
:10FBC000070005208DF80800052101A8FFF7A6FF12
:10FBD0002CE023484079401C2149487108460079AF
:10FBE000401C087108464079002806DD0846407927
:10FBF0001A4991F87510884202DD012018494871B0
:10FC000000201749087048700A465079154A516A11
:10FC100088470BE003208DF804001249886A80476A
:10FC20008DF80500022101A8FFF778FF13E00C48CA
:10FC3000C07800B9A0E700200949C87004208DF8F9
:10FC40000400084640798DF80500022101A8FFF75D
:10FC500065FF00E000BF00BF00BF8DE7EC030020A0
:10FC6000290500203803002010B50446184890F8F4
:10FC7000600008B9002010BD6079102805D1154931
:10FC8000886A8047217A884214D06079132802D08C
:10FC90006079142805D10F49886A8047A17F88427E
:10FCA00008D06079172810D10A49886A8047E17F17
:10FCB00088420AD108484078FA2804DA0648407891
:10FCC000401C054948700120D5E70020D3E700001B
:10FCD000EC030020380300202905002010B504465D
:10FCE000A0B2FDF74DFE10BD10B504464F48D0F848
:10FCF0002404B8B94FF484614C48801CF8F76FFABB
:10FD0000A0794A49C1F82804217AE07901EB001072
:10FD10004649C1F83004217AE07901EB001098B12E
:10FD2000012010BD217AE07901EB00103F49D1F8A4
:10FD30003014884201D10220F3E7217AE07901EB07
:10FD400000103A49C1F830043848D0F82404303063
:10FD5000B0F5846F12D90020344948704FF48461A3
:10FD60003248801CF8F73BFA00203049C1F82404DF
:10FD7000C1F82804C1F82C040320D2E72B48D0F89E
:10FD80002C04401C2949C1F82C040846D0F82C0446
:10FD9000D1F82814884212D90020244948704FF421
:10FDA00084612248801CF8F71AFA00201F49C1F824
:10FDB0002404C1F82804C1F82C040420B1E71B492D
:10FDC000D1F82424891C5018302204F10901F8F7D5
:10FDD000DFF91648D0F8240430301449C1F824045F
:10FDE0000520134908801148D0F83004401C0F4901
:10FDF000D1F82814884216D30C48D0F824040B49B3
:10FE0000C1F8340401204870084690F82304401CCF
:10FE100081F823040020C1F83804012081F83D0452
:10FE200000200349088000207BE70000944A00205E
:10FE30002005002010B51749086D8047052801D01E
:10FE4000002010BD1448407808B90020F9E7134895
:10FE5000407907280BD1002010494871012000F09B
:10FE6000BFF80B200C4981F83C040120E9E70A485F
:10FE7000D0F83804401C0849C1F838040846D0F8C6
:10FE80003804B0F5967F03D900204870C1F83804D3
:10FE90000020D6E738030020944A0020A603002063
:10FEA00010B51348007800B910BD114890F83D0412
:10FEB00090B100200E4981F83D040846811CD0F81D
:10FEC00024240C48F8F764F900200949C1F82404F7
:10FED000C1F82804C1F82C04064800F025F80220D7
:10FEE000FDF792F800200249087000BFDCE700002F
:10FEF000944A0020704600200A4890F83C0480B1E3
:10FF0000084890F83C040B2803DD0B20054981F8D4
:10FF10003C04044890F83C04401E024981F83C042B
:10FF200000BF7047944A002070B58AB0054628216A
:10FF30006846F8F754F90026002427488169684686
:10FF40008847FE208DF8040048208DF80500DE204B
:10FF50008DF806009E208DF807002048B0F8340484
:10FF60001F30C0F347108DF8080001208DF80900FC
:10FF70009DF8080041012846FDF7EAFE06463012CA
:10FF80008DF80A00F0B28DF80B00144890F82304A5
:10FF90008DF80C0013210DF10D00F8F720F9202148
:10FFA000684600F023F800F037F8C820FFF796FE07
:10FFB0000BE02819202100F019F800F02DF832206C
:10FFC000FFF78CFE04F1200084B20448D0F834041A
:10FFD000A042EED80AB070BD38030020944A002039
:10FFE0000149087070470000944A002070B505462A
:10FFF0000C46002001F0AEFC0549C86A8047064661
:020000040801F1
:10000000E1B204483246836A28469847012070BD11
:1000100038030020B802002010B54FF4FA7408E04D
:10002000FEF718FF00B110BD0220FFF757FE601E5B
:1000300084B2002CF4D100BFF5E7000070B50125B3
:10004000002035494872002415E0FF203249085548
:100050003248005DFF2807D03048005DFE2803D0FD
:100060002E48005DFB2804D12B48407A401C2A49C9
:100070004872601CC4B2042CE7DBFF202649C8721A
:1000800000241FE02548005DFB280FD0FE2807D084
:10009000FF2813D12048047000201F4988720EE009
:1000A0002846691CCDB21C490C5408E01A48C57298
:1000B0002846691CCDB218490C5400E000BF00BFAF
:1000C000601CC4B2042CDDDB002406E0124A105D83
:1000D000134AD16B8847601CC4B20F48407AA042D3
:1000E000F4DC104880780C49497A884203DD0A48DC
:1000F000407A0C49887001F033FC0B48808D48B180
:10010000FEF714FE06460849888D054932460B6CF9
:100110000421984770BD0000882000206204002060
:10012000B8020020BF030020F806002070B51E486A
:10013000407A012800DC70BD1C49086B804700B183
:10014000F9E71B480078401CC0B2194908700A281A
:1001500000DAF0E700201649087001F0A7FA12480B
:100160000578002405E01049601C085C0855601CF7
:10017000C4B20D48407A401EA042F4DC0A48407ADE
:10018000401E09490D54002408E0074B195D1B1D52
:10019000185D084BDA6A9047601CC4B20248407A86
:1001A000A042F2DC00BFC6E788200020EC0300205C
:1001B000E0030020B802002010B54FF4C87000F032
:1001C0005DF8044908700846007808B93C200870BA
:1001D00010BD00004C05002002460C2901DA002069
:1001E0007047044883681360C36853600069906077
:1001F0000120F5E74C0500200148407D70470000D4
:100200004C05002001484078704700004C05002054
:1002100001488088704700004C05002070B50446F6
:100220001348807D78B10020114988751149C86A4A
:10023000804705460F49886A804706460E4829468A
:10024000C26A304690478CB10948007860B10848CE
:100250000078401E064908700846007830B900F062
:100260005DF8FFF7A9FF01E0FFF7A6FF70BD0000F2
:100270004C05002038030020B80200202DE9F04191
:1002800006461048808B10B90120F9F781FE0D4811
:10029000808BFA2803DD00200A49888304E009489E
:1002A000808B401C07498883B5082846F9F770FE03
:1002B0000446281903498969471A02488461384667
:1002C000BDE8F0814C05002070B505460C460C2CAD
:1002D00001DD002070BD224629460248F7F758FF8D
:1002E0000120F7E75405002018B10121034A517598
:1002F00002E00021014A5175704700004C050020C2
:1003000002484078401C0149487070474C05002065
:1003100001498880704700004C05002030B58BB043
:10032000282101A8F7F75BFF20208DF804004E4834
:1003300081690DF10500884751208DF809004B486F
:1003400040788DF80A004A48007858B1FEF740FC22
:10035000082803D0FEF73CFC092803D102208DF8C1
:100360000B0002E001208DF80B003F49886A8047AE
:100370008DF80C0000208DF80D008DF80E008DF822
:100380000F008DF810008DF811003848407D30B115
:100390009DF8110040F001008DF8110005E09DF876
:1003A000110000F0FD008DF811002F49086D804705
:1003B000042806D19DF8110040F002008DF81100CC
:1003C00005E09DF8110000F0FD008DF811009DF88A
:1003D0000B00022806D19DF8110040F004008DF8B2
:1003E000110005E09DF8110000F0FB008DF81100F0
:1003F0001E488088000A8DF812001C4800798DF88C
:10040000130000208DF814008DF81500174881683E
:10041000CDF81610C168CDF81A100069CDF81E008D
:100420001B210DF10900FDF793FC0446200A8DF80D
:100430002300E0B28DF8240001200C4988750A4998
:10044000C86A804705460B482946C26A0020904783
:100450000549C86A8047054603482946426B01A8FA
:1004600090470BB030BD0000380300204C05002041
:10047000EC030020B802002010B54FF4806000F0BB
:100480006DF800220221142000F006F8002201215C
:10049000132000F001F810BD2DE9F04103460D4690
:1004A000164600240027A0462A48006800F4E060B1
:1004B000B0F5E06F03D100BF4FF0040830E02548ED
:1004C000006800F4E060B0F5C06F03D101274FF081
:1004D000030825E01F48006800F4E060B0F5A06F55
:1004E00002D10227B8461BE01A48006800F4E06019
:1004F000B0F5806F03D103274FF0010810E01548D5
:10050000006800F4E060B0F5407F03D104274FF0AD
:10051000000805E04FF4A06000F020F80227B8467C
:10052000C7F1040005FA00F4C8F104010F20C84027
:100530003040044324010848C45403F01F01012043
:1005400088405911890001F1E021C1F80001BDE89E
:10055000F08100000CED00E000E400E002490143FE
:10056000024A1160704700000000FA050CED00E03F
:10057000034A0A400243034B1A60BFF34F8F704790
:1005800080FFFF1F08ED00E070B590B004460D46F7
:100590001646002240216846FFF7B6FA1F208DF864
:1005A0000000E0208DF80100FEF70CFB8DF8020042
:1005B0008DF80340324601A92846FFF79AFA6846AB
:1005C000FCF794FF10B070BD38B50446E0781028F1
:1005D00073D2DFE800F0FD1E0895249C9FBDAAFDA4
:1005E000FDC8C9CAF7D00E227E49201DFFF781FA47
:1005F0000E227C493020FDF7D5F87A48401E407A1B
:10060000032805D10922784904F10D00FFF771FA9A
:1006100000BF0E2273490120FFF7B6FFDEE020790C
:1006200072494978884208D0FBF768F9207AFBF7CD
:10063000A1FA00206C490D39488360796B498978AB
:10064000884204D0012068490D3981F82200607980
:100650000E2833D1A079142802D0A0791E282DD1DC
:10066000607962498978884209D160795F498978DF
:10067000884223D15D48C078A17988421ED05C4968
:10068000D1F8CC008047A079142804D159A10020CA
:10069000F9F786FD03E058A10020F9F781FDA27962
:1006A00056A10020F9F77CFDA079142811D1012072
:1006B0004D490D3981F820000BE089E060790E2862
:1006C00002D1A079142804D0002047490D3981F8BF
:1006D00020001A224549491C201DFFF70AFA2379F8
:1006E000627949A10020F9F75BFD1A223F49491CB4
:1006F000A020FDF757F83E48C1692046884700BF53
:100700001A223A49491C0320FFF73EFF66E002F037
:10071000B9FB63E001200090201D02F0F3FB0122F1
:1007200069460620FFF730FF58E0314890F87A001C
:1007300000B953E004223A49201DFFF7DAF90422F8
:100740003749D020FDF72EF80520FAF758FC00BFF6
:10075000274890F87A0000B940E004223049072089
:10076000FFF712FF3AE000BF00BF2148D0F8C810E1
:100770002046884732E0207901280DD117222949E7
:10078000201DFFF7B6F9012017490D3981F8230024
:10079000002081F822000FE0207902280CD11722D6
:1007A0002149201DFFF7A5F901200F490D3981F8D6
:1007B0002400002081F8220001200B490D3981F826
:1007C000210000BF172217490E20FFF7DDFE05E0CC
:1007D0000748D0F8DC102046884700BF00BF012042
:1007E00038BD000069170020050700209017002081
:1007F000EC030020540A0000410A000044434D4429
:100800003A25640A000000005379736D6F64653AFD
:1008100025642C44617461706F733A25640A00008A
:10082000A7030020CF1700201118002070B590B04A
:1008300004460D461646002240216846FFF764F93B
:100840001F208DF80000E1208DF80100FEF7BAF9B5
:100850008DF802008DF80340324601A92846FFF7C3
:1008600048F96846FCF742FE10B070BD30B591B053
:1008700005460C46402101A8F7F7B1FCF5208DF89C
:100880000400AA208DF805008DF8060004F1080088
:10089000C0B28DF80700E1208DF808000A49C86948
:1008A00080478DF8090013208DF80A00224629465A
:1008B0000DF10B00F7F76CFC04484021826901A898
:1008C000904711B030BD000038030020B80200206E
:1008D00030B589B00446E0781B2876D2DFE800F016
:1008E000E1360E493C5A4F63E1767A95999AA5AB69
:1008F000ACE1E1A6E1E1ADC1C2D7D30007226E4968
:10090000201DFFF7F6F8FBF799FDFBF75FFD6A493D
:10091000491E887800F0D8F9FEF708FA05466649BE
:10092000491EC87965490A6B29469047002508E0A9
:100930006149491EC87961490A6B29469047681C7C
:10094000C5B25F48407AA842F2DC00BF07225A498C
:100950000120FFF76BFFAAE00D225A49201DFFF787
:10096000C8F800F09DFF0D2256490820FCF71AFF39
:1009700000BF0D2253490320FFF758FF97E00422E0
:100980005149201DFFF7B5F804224F491820FCF704
:1009900009FF00BF01A8FEF727F9042201A90520DD
:1009A000FFF744FF83E001208DF804004348012253
:1009B00001A9036A2E209847404988688047012290
:1009C00001A90720FFF732FF71E06AE02046FAF73D
:1009D000A1FC6CE02079012802D0207902280DD1F9
:1009E0002079012801D0012000E000208DF80400CA
:1009F000012201A90A20FFF719FF05E02079042848
:100A000002D13249486E804751E02046FAF708FB90
:100A10004DE04CE02D4801A9C26D204690470922C7
:100A200001A90D20FFF702FF41E040E028480168DE
:100A3000204688473BE03AE039E02648807858B1C4
:100A400060791E2808D000202249887000220521E4
:100A50002048C01CFFF758F81C48816B2046884787
:100A600025E000BF1948D0F8981020468847E07864
:100A7000182807D1217909B1012100E00021084699
:100A800000F032FF13E0207900F02EFF00BF124883
:100A9000C07D8DF80400012201A91920FFF7C6FED0
:100AA00005E00A48D0F8E0102046884700BF00BFA4
:100AB000012009B030BD0000AD030020B8020020C5
:100AC00088200020E7170020B5030020EC03002059
:100AD000E803002090170020F806002030B593B0FE
:100AE00040230A2202A9214800F040F910B9002051
:100AF00013B030BD9DF80800001DC0B28DF8040091
:100B00000DF10500FEF770F8FEF708F960B100245A
:100B100005E0214601A8FCF7B3FC601CC4B21448F0
:100B2000007AA042F5DC1FE0124890F884001E28ED
:100B300013D1104890F8850078B11A210DF1090001
:100B4000FDF706F9054628128DF82300E8B28DF866
:100B5000240020208DF8040000BFFEF7E5F80546CC
:100B6000294601A8FCF78CFC0120C1E7E423002002
:100B700088200020EC03002070B50446074908686F
:100B8000804740230A222146054800F0B9F805466F
:100B9000024948688047284670BD0000B80200201E
:100BA000E423002070B50446402311222146034867
:100BB00000F0DCF80546284670BD0000281800202B
:100BC00010B50446402311222146024800F098F84F
:100BD00010BD00002818002010B540231122024942
:100BE000024800F0BBF810BD34180020281800207F
:100BF00010B504460D4890F8C40008B9002010BD97
:100C0000012C07D1FDF75CFA08B10020F7E708488E
:100C1000C47409E00648C07C30B100210448C174A6
:100C200000F016FF0120EAE70020E8E7EC030020CF
:100C3000175F002010B588B00446E078182814D15A
:100C400020791249087060798870F5208DF80000CD
:100C500020798DF8010060798DF802000C4803229C
:100C60006946036A4FF484609847084800788DF815
:100C70000000064880788DF8010002236A4617219B
:100C8000612001F063FF08B010BD0000D44E0020C9
:100C9000B802002010B504460948847000F060FED8
:100CA00006220849F020FCF77DFD0A20FDF723FC11
:100CB00007220349491C0020FCF774FD10BD000009
:100CC000AC030020C003002010B50446204600F00D
:100CD0007BFE00F045FE06220749F020FCF762FD8E
:100CE0000A20FDF708FC054884700722411C0020FB
:100CF000FCF758FD10BD0000C0030020AC0300202D
:100D00002DE9F0410446884615461E4612490868FA
:100D1000804720886188884204D1A088A84201DBEE
:100D2000002712E06288A06802FB060132464046B6
:100D3000FEF7DFFE6088401C90FBF5F105FB11001B
:100D40006080A088401CA080012703494868804734
:100D50003846BDE8F0810000B802002010B581607F
:100D6000448804800024848010BD00002DE9F041F7
:100D70000446884617461D46114908688047208862
:100D80006188884203D1A08808B9002612E0228831
:100D9000A16802FB05102A464146FEF7AAFE2088FC
:100DA000401C90FBF7F107FB11002080A088401E3B
:100DB000A08001260249486880473046BDE8F0819E
:100DC000B802002070B504460E460A4908688047FC
:100DD00020886188884203D1A08808B9002503E0F3
:100DE00020887043A1680D5C024948688047284606
:100DF00070BD0000B80200202DE9F0470446884687
:100E000017461D46DDF82090154908688047208860
:100E10006188884203D1A08808B900261AE020889A
:100E20006843A168085C484501D0022612E0228888
:100E3000A16802FB05102A464146FEF75AFE2088AB
:100E4000401C90FBF7F107FB11002080A088401E9A
:100E5000A08001260249486880473046BDE8F087F7
:100E6000B80200202DE9F04F8CB0074600200A9010
:100E70004AA090E8004CC068CDE905BECDF810A0AE
:100E800007900FF21C1ADAE9000ACDE9020A0FF204
:100E9000101ADAE9000ACDE9000A44484068C0F3B4
:100EA00081000B900B9820B1012804D002283FD17B
:100EB00003E03F4A3EE03F4A3CE03C48406800F4E3
:100EC000803CBCF5803F12D13848C06A00F08048B1
:100ED000B8F1000F01D1374B00E0374B3348406881
:100EE00000F40039B9F5003F02D15B0800E0334B54
:100EF0002E484068C0F383412C48406800F00060F1
:100F000008B141F010012948406800F0804008B164
:100F100041F020010F2901D2891C06E00F2903D3DB
:100F20003E2901D8491C00E03F2103FB01F201E00A
:100F30001F4A00BF00BF1D484068C0F3031504A846
:100F4000465D22FA06F419484068C0F3022502A85B
:100F5000465D24FA06F0099014484068C0F3C225A3
:100F60001DF8056024FA06F0089037B1012F06D06D
:100F7000022F06D0032F0AD106E00A9208E00A9455
:100F800006E009980A9003E008980A9000E000BF84
:100F900000BF0A980CB0BDE8F08F00000000000010
:100FA00000000000010203040607080900100240C7
:100FB00000127A000024F400006CDC0200093D00FD
:100FC00010B50020FFF74EFF044640F2026000F02B
:100FD00053F82548844204D14FF4800000F05CF8B7
:100FE00015E02248844203D1002000F055F80EE0BD
:100FF0001F48844204D14FF4400000F04DF806E051
:101000001C48844203D14FF4000000F045F840F240
:10101000026000F031F840F2036000F02DF840F279
:10102000046000F029F840F2056000F025F84FF464
:10103000C06000F021F840F2177000F01DF84FF486
:10104000E06000F019F840F2017000F015F840F28D
:10105000027000F011F840F20C6000F00DF840F260
:101060000F7000F009F810BD006CDC0200A24A0409
:1010700000D8B805000E2707064A02EB9011096850
:1010800000F01F0301229A401143024B03EB901220
:101090001160704700100240044A516821F4400179
:1010A00041EA0002014B5A60704700000010024004
:1010B0001CB50B4803226946436A4FF48460984785
:1010C0009DF80000F52807D19DF80100054908703A
:1010D0009DF80200887002E00020024908701CBDE3
:1010E000B8020020D44E00201FB5224810226946C5
:1010F000436A9001984700240EE0C4F10E001DF8E9
:101100000000C4F10F011DF801104840C4F10F01A7
:101110000DF80100601CC4B20F2CEEDB16480378FA
:10112000C21C00F123016846F7F7E4FF11481022C2
:101130006946436A4FF48260984700240EE0C4F188
:101140000E001DF80000C4F10F011DF80110484009
:10115000C4F10F010DF80100601CC4B20F2CEEDBCE
:1011600005480378C21C00F133016846F7F7C2FF57
:101170001FBD0000B8020020D44E002010B5074863
:10118000C16C022088470120054908700020488072
:10119000012008710020C88010BD0000B8020020A6
:1011A000F806002010B50748407A00B910BD0020AD
:1011B0000449487288720448016D0120884700BFC5
:1011C000F4E70000F8060020B8020020F0B58DB06A
:1011D00005464B4890F8900010B901200DB0F0BDC5
:1011E0004848007808B90120F8E72122294604A8D8
:1011F000F6F7CEFF9DF81500F7F73EFF061E01DD5E
:101200008DF8156006240DE004A8005D80F0A506A9
:1012100004A9601C085C80F055000855601C0E5441
:10122000A01CC4B21F2CEFDB00240DE0C4F11F0092
:1012300004A9085CC4F1200104AA515C4840C4F12F
:1012400020015054601CC4B21A2CEFDB00240CE0C7
:1012500004F1160004A9085CA11D04AA515C4840D1
:1012600004F116015054601CC4B20B2CF0DB1022A8
:101270000DF116016846F6F78BFFFBF7B9FC40B19C
:1012800020480378C21C0DF116016846F7F732FFBB
:1012900018E09DF815004C2809D01A48037800F191
:1012A00023020DF116016846F7F724FF0AE01548FE
:1012B0000378C21C0DF116016846F7F71BFF1320D7
:1012C0008DF81500212204A92846F6F761FFE87F72
:1012D000002803DC95F8200000280FDD1A21681D86
:1012E000FCF736FD0746E87FB0EB272F04D1F8B2B4
:1012F00095F82010884201D000206FE701206DE7AB
:10130000EC030020D44E0020F0B589B005464548D6
:1013100090F8900008B909B0F0BD4348007800B9D2
:10132000F9E71A21681DFCF713FD07463812E87724
:1013300085F8207020202870212229466846F6F77B
:1013400027FF6879F7F798FE061E01DD8DF8056026
:101350009DF80500412803D09DF8050042280FD1D3
:101360009DF8090028280BD14C208DF805002E4847
:101370000378C21C0DF10601A81DF7F751FF14E018
:10138000FBF736FC40B128480378C21C0DF106017A
:10139000A81DF7F745FF08E02348037800F1230272
:1013A0000DF10601A81DF7F73BFF00240CE004F146
:1013B0001600285CA11D1DF80110484004F116011B
:1013C0000DF80100601CC4B20B2CF0DB072409E00F
:1013D000601E1DF800001DF8041048400DF80400C0
:1013E000601CC4B2212CF3DB06240FE01DF80400BE
:1013F00080F05506601C1DF8000080F0A5000DF877
:101400000400601C0DF80060A01CC4B21F2CEDDBB2
:10141000212269462846F6F7BBFE2020287000BF2F
:1014200079E70000EC030020D44E002030B591B0E5
:10143000044621460720F8F795FB05462246294633
:101440000720F8F7B5FC05F0400060B18DF80040CA
:1014500021460DF10200F8F7A7FB8DF801000E48B8
:10146000016C6846884705F0200028B1012000F093
:1014700071FA204600F02AF9084A32F81410084A96
:1014800052F82400FDF700FD2046F8F746FD2046FF
:10149000F8F74AFD11B030BD380300205835010877
:1014A0004835010870B506460D461446284A32F8FC
:1014B0001410284A52F82400FDF7E6FC21460020CB
:1014C000F8F74EFD244A32F81410244A52F824004A
:1014D000FDF7DAFC2146E120FCF7ECFF1E4A32F86A
:1014E00014101E4A52F82400FDF7D0FC202D00DD18
:1014F0002025FCF78BFB40B1194A32F81410194A29
:1015000052F82400FDF7C0FC07E0154A32F8141029
:10151000144A52F82400FDF7B9FC2025224629463A
:101520003046F8F773FC0A4A32F81410094A52F8A8
:101530002400FDF7ABFC3220F7F7FEFD044A32F839
:101540001410044A52F82400FDF79EFC70BD000000
:10155000703501086035010824350108143501088B
:10156000583501084835010800B591B000224021E6
:1015700001A8FEF7C9FA1F208DF80400E1208DF8BC
:1015800005000A49C86980478DF806000A208DF8D1
:10159000070006208DF808000DF10900FDF79EFBFD
:1015A0000248416C01A8884711B000BD38030020F3
:1015B00010B512480078012800D010BD0F484068CF
:1015C000401C0E49486040F2DC5188420ED20B4864
:1015D00040686421B0FBF1F201FB120058B90848E1
:1015E000C16D01208847FFF7BFFF04E002200349D7
:1015F00008700020486000BFDFE70000D80300202B
:10160000B802002010B504462046F8F729FC214610
:101610007020F8F71DFA224601211D20F8F7C8FBBB
:10162000224620211120F8F7C3FB22461E2100206C
:10163000F8F7BEFB224600210120F8F7B9FB22464D
:1016400001210220F8F7B4FB224603210846F8F7EF
:10165000AFFB154890F87400012803D12146F8F734
:101660004FFB0CE0104890F87400022803D121468B
:10167000F8F746FB03E021460020F8F741FB21463E
:101680000320F8F70FFB224605214AF2554000F0EF
:1016900055F82046F8F724FA2046F8F705FA2046D0
:1016A000F8F742FC10BD0000EC030020704700007A
:1016B00000EB4001044A12F81110491C00EB4002F3
:1016C000014B03F8121070473821002000EB400155
:1016D000054A02EB41014978491C00EB4002024BEC
:1016E00003EB4202517070473821002070B5044668
:1016F0000D46FCF78BFA20B129460720F8F7D2FAFD
:101700001BE0012C04D0022C07D0032C0FD109E0E0
:1017100029460220F8F7C6FA0EE029460120F8F71C
:10172000C1FA09E029460020F8F7BCFA04E029468E
:101730000320F8F7B7FA00BF00BF70BD7CB50446C0
:101740000D4616460AA103C9CDE9000120128DF805
:101750000200E0B28DF80300324629466846F8F7E9
:10176000EDFA33462A4669460020F8F7ADFA7CBD0B
:101770001998A4250100000070B505460C46F7F73E
:101780002EFC21462846F8F7BEFB2046F8F7CCFB96
:10179000F8F71CFE70BD000010B504460548007C3B
:1017A00028B12178601CF9F703F9012010BD002051
:1017B000FCE70000CC62002070B5054600240DE077
:1017C000094800EB840104222846F6F713FD18B9F6
:1017D000054800EB840070BD601C84B203480078AB
:1017E0008442EDDB0020F6E72C5F00202F0500206F
:1017F00030B591B004460D462078401CC2B269460F
:101800002046FEF776F9104890F87E0060B19DF80A
:101810000000001FC0B28DF800009DF800200DF1FF
:101820000101081DFEF765F90748D0F8A4106846C5
:1018300088479DF8001005482A46836A0DF101008B
:10184000984711B030BD0000EC030020B802002022
:101850002DE9F04104462078062813D00E4805688B
:10186000001D0668001D07683D4455B10822A11CF3
:101870002846FDF7BDFC042204F112013046FDF7B5
:10188000B7FC06E00549086810B16080010CA18032
:1018900000BFBDE8F0810000E8F7FF1F0021024013
:1018A000A0200C4988720C4890F8700048700D20F8
:1018B00088700120C870084890F87100C872064806
:1018C00090F8721003480173034890F873100148B0
:1018D00041737047E6170020EC03002001490870AF
:1018E00070470000D003002010B504460D4890F862
:1018F000850058B10B49D1F8B000804718B10120DC
:101900000949C87505E00848C47502E00020064989
:10191000C8750122044917314FF4A070FBF742FF4C
:1019200010BD0000EC030020F806002006490978ED
:1019300001B1704728B90121034A11700349044AD3
:10194000916100BFF5E70000B3020020F5920008A6
:10195000B8020020014908707047000030030020E1
:1019600010B51648807816490872002204211448E0
:10197000001DFEF7C9F81248027A011D0F48C01C6D
:10198000FEF7B7F80E48C07A0D49097A884204DAA2
:1019900000210B48C27A001D8154002408E0084B46
:1019A000195D1B1D185D074BDA6A9047601CC4B2B5
:1019B0000348407AA042F2DC10BD0000BF030020C3
:1019C00088200020B802002010B504460948C470E1
:1019D0000146C878FCF7A8F8064908710879FCF7B1
:1019E000A3F8044948714879FCF79EF801498871C9
:1019F00010BD0000BF030020016841F040010160FC
:101A000070470146C86880B27047C160704702469F
:101A10009068084008B1012070470020FCE70246AA
:101A20000020106800F441500B6818434B681843BD
:101A30008B681843CB6818430B6918434B691843EC
:101A40008B6918431060D36923F40063D361704736
:101A500010B50D4890F8C40000B910BD0B48C07B0C
:101A6000012800D1F9E70A48816B00208847074820
:101A7000007D401CC1B2054801750121C1730021E0
:101A80000174417400BFE8E7EC030020175F0020F9
:101A900038030020002000213E4A126842F48032C0
:101AA0003C4B1A6000BF401C3A4A126802F40031F5
:101AB00019B94FF6FF729042F5D1364A126802F416
:101AC00000320AB900BFFEE7324AD26942F08052C2
:101AD000304BDA61304A126842F440422E4B1A60B1
:101AE0002C4A52682B4B5A601A4652685A601A4662
:101AF000526842F480625A601A46526822F44032B8
:101B00005A601A46526842F440325A601A46526885
:101B1000224B1A401F4B5A601A46526842F4501228
:101B20005A601A46126842F080721A6000BF194A61
:101B3000126802F00072002AF9D0174A126842F4C3
:101B40008032154B1A6000BF134A526802F480328B
:101B5000002AF9D0104A126842F400320E4B1A6083
:101B600000BF0D4A526802F40032002AF9D0094A37
:101B7000526822F00302074B5A601A46526842F03C
:101B800002025A6000BF034A526802F00802002AAB
:101B9000F9D070470010024000700040FFFFC3B74B
:101BA00010B5FFF777FF10BD10B5124800684FF46D
:101BB0007A71B0FBF1F4601EB0F1807F01D3012097
:101BC0000FE0601E4FF0E02148610F214FF0FF3021
:101BD000F8F770F900204FF0E021886107200861D4
:101BE000002008B100BFFEE70F214FF0FF30F8F7EB
:101BF00061F910BD1000002010B501202249887540
:101C00000846407A70B90846807A401CC0B2887293
:101C1000052807DD00208872012048721B48016DED
:101C2000002088471848007A401CC0B21649087244
:101C300019280EDD002008721449C869804720B1B8
:101C40001248C16C0220884703E01048C16C012093
:101C500088470D484088401C80B20B49488040F2BC
:101C6000DC51884203DD002007490870488006489F
:101C7000C088401C80B20449C880322802DD0020A0
:101C80000871C88010BD0000F8060020B8020020CE
:101C9000C162704701460020486A70474162704740
:101CA000016841F001010160704700000A8882620A
:101CB0001D4A90420ED0B0F1804F0BD01B4A90428B
:101CC00008D01B4A904205D01A4A904202D01A4AC4
:101CD00090420BD1026822F07002026002684B88C9
:101CE0001A43026002688B881A4302608A68C262E3
:101CF000124A90420AD0124A904207D0026822F457
:101D0000407202600268CB881A430260064A904221
:101D100002D0094A904201D10A7B0263426942F033
:101D20000102426170470000002C014000040040A5
:101D300000080040000C004000340140001000404A
:101D400000140040C2688A43C2607047C2680A43F8
:101D5000C2607047CA43026170470246D06800EA19
:101D600001031069084010B10BB101207047002039
:101D7000FCE781621AB9436943F00103436170478C
:101D800010B540230A2202490248FEF7E7FF10BDC2
:101D9000F0230020E423002010B540230A2202494A
:101DA0000248FEF7DBFF10BD64210020582100200F
:101DB0007047000010B50A48C16B032088474FF4F4
:101DC0007A70FBF7EAFD0748816B01208847002005
:101DD000054908740021092000F094F810BD0000A6
:101DE000B802002038030020CC62002010B507485C
:101DF000C068401C0549C860052805D30020C8609C
:101E0000F8F75CFFF7F70AFE10BD0000CC62002077
:101E10000020704738B504462079012802D00728F1
:101E200065D140E03348A1680160E1684160218AE2
:101E30000181E079012822D12E48807901062D48C0
:101E4000C07901EB00412B48007A01EB00212948C1
:101E5000407A0D18284881696846884725484079A6
:101E6000244A127900EB022081B22A466846F8F72C
:101E70003BFD01201F490874F8F7F8FE0CE0E079FB
:101E8000022809D100201B49087405201B4908704D
:101E90001948816B012088471A23221D16216120D1
:101EA00000F054FE24E01A23221D1621612000F0C8
:101EB0004DFE60791E2803D12046FDF715FF15E081
:101EC000207A15280BDC217A01EB410209491131F6
:101ED00001EB0210302204F10901F6F759F9207ADA
:101EE000152803D10120034981F8310400E000BF27
:101EF00000BF38BDCC620020380300203805002028
:101F00007047704730B589B005460C4618208DF8EB
:101F10000400E1208DF805000A49C86980478DF862
:101F2000060016208DF807008DF8085020128DF855
:101F30000900E0B28DF80A000248416C01A8884708
:101F400009B030BD3803002010B50446D4F8AC0009
:101F50000021826A2046904710BD10B50446D4F88F
:101F6000AC10A06C0022CB6A1146984710BD70B52A
:101F700004460025D4F8AC002946426B2046904721
:101F800000BF70BD416002814381704741600281A2
:101F9000438170474160028143817047417841F03D
:101FA0008001014A116070474C5C004070B50446E6
:101FB0000D46A078032808D1287930B9D4F8A800B4
:101FC0002946C2682046904770BD0120FCE700000A
:101FD00001200849086000200860091D08600549C3
:101FE000103108600348006840F41F400149086050
:101FF00070470000405C0040012004490860002058
:10200000091D08600320091F08607047405C0040FC
:1020100010B50446012C04D101020548FCF736FF37
:1020200004E04FF480710248FCF72EFF10BD000061
:1020300000080140F0B503460024002500266AB9D7
:10204000214800EB0110C068C0F309051E4800EBF1
:10205000011080681D4F07EB400627E0012A23D1BD
:102060001B4F07EB8100D0F8000C00F0400068B176
:10207000154800EB01104068C0F30905124800EB59
:1020800001100068114F07EB40060FE00E4800EB0F
:102090000110C068C0F309050B4800EB011080680F
:1020A0000A4F07EB400601E00020F0BD002405E0E8
:1020B00036F8047B1F809B1C601C84B2681CB4EB48
:1020C000500FF5D32846F0E7006000400060004064
:1020D0000050004070B58AB1134D05EB01152D6815
:1020E000124E06EB4504002303E0058820C4801C43
:1020F0005B1C551CB3EB550FF7D300BF0A4B03EB2A
:1021000001135A6000BF0A4C04EB8103D3F8003C72
:1021100048F6BF74234083F03003054D05EB81047E
:10212000C4F8003C00BF70BD00600040006000408B
:102130000050004070B504460D46D4F8AC00294666
:10214000426A2046904770BD30B5034601F07F00DB
:10215000CA1142B300BF294C04EB8002D2F8002C14
:1021600002F040027AB100BF04EB8002D2F8002CEA
:1021700048F68F74224042F04002204D05EB800467
:10218000C4F8002C00BF00BF00BF1C4C04EB800251
:10219000D2F8002C48F6BF742240184D05EB80049D
:1021A000C4F8002C28E000BF144C04EB8002D2F8E5
:1021B000002C02F480427AB100BF04EB8002D2F816
:1021C000002C48F68F74224042F480420B4D05EB00
:1021D0008004C4F8002C00BF00BF00BF074C04EB14
:1021E0008002D2F8002C4BF68F742240034D05EB91
:1021F0008004C4F8002C00BF30BD00000050004037
:102200002DE9F04104460D4616461F46D4F8AC00B1
:102210003B4632462946D0F820C02046E047BDE87C
:10222000F0812DE9F04104460D4616461F4605F0A3
:102230007F0000EB400104F1140000EB8108002353
:102240003A4631464046FFF79DFED4F8AC00294699
:10225000826A20469047BDE8F081000030B5024612
:10226000002002F14401A023204C2360002363607E
:1022700040230B803039A3600B800B883E2B0AD99A
:102280000B884FF6FF7404EA43135B1E43F40043CC
:10229000164CE36006E00B885B1C23F001035B0235
:1022A000124CE36001200FE0114C04EB8003D3F8E3
:1022B000003C48F68F74A34303430D4D05EB8004A7
:1022C000C4F8003C431CD8B20428EDD3094B1B686A
:1022D0009BB2084C236043F2202323608023054CEB
:1022E0004C3423600123937030BD00000060004037
:1022F00000500040005C004010B500BF4A06094B8A
:1023000003EBD252D2F8002C4BF68F731A4082F4B2
:1023100040524B06034C04EBD353C3F8002C00BFD0
:1023200010BD0000005000402DE9F04705468946E9
:1023300016461F4609F07F0A0AEB4A0105F14400E0
:1023400000EB8108B8F80000B84201DD384601E032
:10235000B8F800000446D5F8AC0022465146C36ADE
:1023600030469847381B82B2311923464046FFF762
:1023700009FEBDE8F08700002DE9F04305460C4654
:102380009E7806F07F009988002793F803C00CF030
:10239000030CDFF8508258F82CC04CEA000CDFF830
:1023A000489209EB8008C8F800CC4FEAE61CBCF163
:1023B000000F62D000EB400805F1440C0CEB8807DD
:1023C0003980B4B9DFF824C20CEB001CCCF8002033
:1023D00000BFC84608EB800CDCF800CC48F6BF789C
:1023E0000CEA080C8CF0200C09EB8008C8F800CC33
:1023F000F6E0012CFCD1DFF8F08108EB800CDCF872
:1024000000CC4CF4807C48F68F780CEA080CDFF89E
:10241000D89109EB8008C8F800CC1FFA82FCDFF8DD
:10242000CC8108EB0018C8F800C04FEA124CDFF866
:10243000BC8108EB0018C8F808C000BFC84608EB0C
:10244000800CDCF800CC48F6BF780CEA080C8CF065
:10245000300C09EB8008C8F800CC00BF00BFC846AC
:1024600008EB800CDCF800CC4BF68F780CEA080CFB
:1024700009EB8008C8F800CCB2E000EB400805F199
:10248000140C0CEB8807398034B9DFF860C10CEB11
:10249000001CCCF808204EE0012C4CD1DFF848811C
:1024A00008EB800CDCF800CC4CF4807C48F68F788C
:1024B0000CEA080CDFF8309109EB8008C8F800CC72
:1024C00000BFC84608EB800CDCF800CC48F68F78DB
:1024D0000CEA080C4CF0400C09EB8008C8F800CC62
:1024E00000BF1FFA82FCDFF8048108EB0018C8F86F
:1024F00000C04FEA124CDFF8F48008EB0018C8F86F
:1025000008C03E290BD9A446CCEB411C4CF4004C2E
:10251000DFF8D88008EB0018C8F804C00BE001F120
:10252000010C2CF0010C4FEA4C2CDFF8C08008EBBA
:102530000018C8F804C03E290CD94FF0010CCCEBB0
:10254000411C4CF4004CDFF8A48008EB0018C8F8DC
:102550000CC00BE001F1010C2CF0010C4FEA4C2CEB
:10256000DFF8888008EB0018C8F80CC09CB900BFE1
:10257000DFF8748008EB800CDCF800CC4BF68F7829
:102580000CEA080C8CF4005CDFF85C9009EB800826
:10259000C8F800CC24E0012C22D100BFDFF848802D
:1025A00008EB800CDCF800CC4BF68F780CEA080CBA
:1025B000DFF8349009EB8008C8F800CC00BF00BFFA
:1025C000C84608EB800CDCF800CC48F6BF780CEA73
:1025D000080C8CF0200C09EB8008C8F800CC00BF78
:1025E000BDE8F083E4340108005000400060004082
:1025F00030B5024601F07F00CB1193B300BF334CDE
:1026000004EB8003D3F8003C03F040037BB100BF30
:1026100004EB8003D3F8003C48F68F74234043F06A
:1026200040032A4D05EB8004C4F8003C00BF00BF06
:10263000002400EB400502F1440303EB85039C708A
:1026400000BF224C04EB8003D3F8003C48F6BF7473
:10265000234083F030031D4D05EB8004C4F8003C9B
:1026600033E0FFE700BF194C04EB8003D3F8003CD4
:1026700003F480437BB100BF04EB8003D3F8003C3C
:1026800048F68F74234043F48043104D05EB8004DB
:10269000C4F8003C00BF00BF002400EB400502F17D
:1026A000140303EB85039C7000BF084C04EB80030C
:1026B000D3F8003C4BF68F74234083F44053034D12
:1026C00005EB8004C4F8003C00BF30BD0050004062
:1026D00030B5024601F07F00A8B900BF244B1B684B
:1026E00048F6BF74234083F01003214C236000BFE1
:1026F00000BF23461B684BF68F74234083F480533E
:102700001B4C236033E0CB11C3B1012400EB400527
:1027100002F1440303EB85039C7000BF154C04EBEE
:102720008003D3F8003C48F6BF74234083F01003C5
:10273000104D05EB8004C4F8003C18E0012400EBC8
:10274000400502F1140303EB85039C7000BF094CA4
:1027500004EB8003D3F8003C4BF68F74234083F4E2
:102760008053044D05EB8004C4F8003C00BF30BD2D
:10277000005C00400050004010B503464806064C7F
:1027800004EBD050D0F8002CC81110B102F030008A
:1027900010BD0020FCE700000050004070B504466A
:1027A0000D46164608201449087001204870400262
:1027B0004880084644607434256366630F48A0630C
:1027C0000F4844F874090F49A1670F49E167D4F82D
:1027D000A4004068C07900F0400040092071012148
:1027E000E171D4F8AC1008688047D4F8A410C96827
:1027F000C868FFF72DF870BD140000201C000020F1
:102800001DBD0008D9BC000887BC000810B50446EF
:10281000A078E0700420A070E07930B100BFD4F857
:10282000AC100869804700BF01E00321A17110BD11
:102830002DE9FC419A48006880B2019098480068F0
:102840009749091F096801F47F41084000909548A5
:102850004468BDF8000000F4004000287DD0A5E0E9
:10286000BDF8040000F00F05BDF8040000F01000F2
:10287000002860D08C4901EB8500D0F8000C00F4F2
:10288000004000281FD000BF01EB8500D0F8000CED
:1028900040F68F710840844A02EB8501C1F8000CB4
:1028A00000BF114601EB8500D0F8000C00F4006079
:1028B00060B14DB905EB450104F1740050F82120D9
:1028C00029462046904770E0BDE8FC8105EB4501B4
:1028D00004F1140000EB81067068D4F8AC100022FB
:1028E0000B6B2946984707467068384470607089BA
:1028F0003844708170893189884202DA3088B84260
:1029000012DD05EB450104F1740000EB8100406825
:1029100080B105EB450104F1740000EB810029460C
:1029200042682046904705E0D4F8AC002946826A08
:102930002046904739E05C4901EB8500D0F8000C57
:1029400000F0800088B300BF01EB8500D0F8000CD8
:1029500048F60F710840544A00E030E002EB850170
:10296000C1F8000C00BF05EB450104F1440000EB89
:102970008106308990B905EB450104F1740000EB44
:102980008100806880B105EB450104F1740000EB23
:102990008100294682682046904705E03389294610
:1029A00020467268FFF7C0FC00BF00BF3C480068CB
:1029B00080B2019000F4004000287FF451AFBDF8D0
:1029C000000000F4805070B16FF48050344908600A
:1029D000E078A070607A30B900BFD4F8AC104869D4
:1029E000804700BF00BFBDF8000000F4006060B188
:1029F0002B48001F006800F0100030B92046FFF798
:102A000005FF6FF4006026490860BDF8000000F47F
:102A1000007058B16FF400702149086023480068C5
:102A200020B122480068016820468847BDF80000B0
:102A300000F4807018B36FF4807019490860A079B1
:102A4000E8B1A079401EC1B2A171C1B9607A50B19C
:102A50001348001F006820F010001149091F08608A
:102A6000002161720BE00E48001F006840F010006A
:102A70000B49091F08600321A17101216172BDF892
:102A8000000000F4806040B16FF480600449086089
:102A9000D4F8AC00C1692046884700BF14E70000A5
:102AA000445C004014000020005000405C00002006
:102AB0000548006820F004000349086008460068E3
:102AC00020F0080008607047405C004005494968F4
:102AD000097A012905D10449096841F01001024A27
:102AE0001160704714000020405C004070B505463E
:102AF0000C466078034951F820202146284690472B
:102B000070BD0000600000200348006840F00C0029
:102B10000149086070470000405C00400246012007
:102B2000704710B5FFF762F910BD000010B5012025
:102B300003490870F9F7FCFC00F098FA10BD00009A
:102B4000B20200207047704770477047F0B589B0F7
:102B500004460D4616461F46202101A8F5F73FFB07
:102B60001F208DF8040004F00F0040F0E0008DF805
:102B700005000949C86980478DF806008DF807509F
:102B80003A46314602A8F5F703FB0348416C01A819
:102B9000884709B0F0BD00003803002070470000EE
:102BA000F0B59DB00446002240210DA8FCF7ACFF13
:102BB0001F208DF83400E0208DF83500FCF702F876
:102BC0008DF8360005208DF837008DF8384099488B
:102BD0000078A0422DDB04EB440000EB8410964902
:102BE000084490F84100022823D104EB440101EB92
:102BF0008411914B194491F8402004EB440101EBFE
:102C00008411C8180DF13901FCF773FF0DA8F8F70E
:102C100098FF04EB440000EB84108749084490F8C7
:102C200042008DF834000DA8FAF760FC01201DB0B9
:102C3000F0BD20218148FEF7C5F8054675B9FF2093
:102C40008DF8380000208DF839008DF83A008DF8A5
:102C50003B000DA8FAF74AFC0020E8E70A950CAA09
:102C60000BA90AA8FCF76EF88DF8340004EB4401B8
:102C700001EB8411704A881800224021FCF744FFC0
:102C80009DF8280004EB440101EB84116A4A50547A
:102C9000012004EB440101EB8411114481F8400050
:102CA00004EB440101EB8411114481F841006148B7
:102CB0000470002694E0701CC6B22023C82202A92A
:102CC0005E480095FEF798F80746012F50D102A9FB
:102CD0002046F8F735FF9DF828000D2820D1012067
:102CE00004EB440101EB8411534A114404EB440208
:102CF00002EB8412504B1A4492F84020885404EBA3
:102D0000440000EB84101946084490F84000401C31
:102D100004EB440101EB84111A46114481F8400090
:102D200004EB440000EB8410434A104404EB4402DB
:102D300002EB8412404B1A4492F8402081189DF80F
:102D400030200DF10900FCF7D4FE04EB440000EB49
:102D500084103949084490F840009DF83010084428
:102D600004EB440101EB8411334A114481F8400023
:102D70001FB19DF82C00864231DBFF2004EB44019B
:102D800001EB84112C4A114404EB440202EB84123F
:102D9000294B1A4492F840208854FF2104EB440048
:102DA00000EB84101A46024404EB440000EB84104C
:102DB000184490F84000401C115404EB440000EB10
:102DC00084101946084490F84000801C04EB44012C
:102DD00001EB84111A46114481F8400005E000BF60
:102DE0009DF82C008642FFF666AF00BF04EB44015D
:102DF00001EB8411104B194491F8402004EB44017D
:102E000001EB8411C8180DF13901FCF772FE9DF831
:102E1000340004EB440101EB8411074A114481F8AA
:102E200042000DA8F8F78DFE0DA8FAF75FFB012010
:102E3000FDE60000E10300207C3F0020702600201A
:102E400010B500F053F800200249487088700870EF
:102E5000C87010BDE303002010B50948C078401CBD
:102E6000C0B20749C870022800DA10BD002004492A
:102E7000C8700120887000F013F800BFF5E700006B
:102E8000E303002010B500F0EFF80120034948707B
:102E9000887000200870C87010BD0000E303002097
:102EA00010B50B48407890B10948007809280EDA2F
:102EB0000748807858B106480078401C04490870DB
:102EC0000878FFF76DFE024948700020887010BD39
:102ED000E303002010B504462023C82221460248FF
:102EE000FDF70EFF10BD00007026002010B5202356
:102EF000C82202490248FDF731FF10BD7C260020A0
:102F000070260020FEB50746002600240CE0385D40
:102F100010B1385D0A2800DD08E0385D0DF80400C6
:102F2000701CC6B2601CC4B20A2CF0DB00BF06B92C
:102F3000FEBD494908688047002410E000201DF8C4
:102F4000041001EB410202EB8111444A114481F863
:102F500041001DF80400F8F7CDFD601CC4B2B44276
:102F6000ECDB3F480078864203DB00203C490870D8
:102F70006CE0012501245FE004EB440000EB8410C9
:102F80003649084490F8410000B953E03548C08BF9
:102F9000401C3449C883022005EB450101EB851133
:102FA0002E4A114481F84100AC4202D1681CC5B2DE
:102FB00040E004EB440303EB8413DFF8A0C0634458
:102FC00093F8402005EB450303EB851303EB0C015D
:102FD00004EB440303EB841303EB0C00FCF789FDC3
:102FE00004EB440000EB84101C49084490F84000B6
:102FF00005EB450101EB8511184A114481F84000A9
:1030000004EB440000EB84101146084490F84200A1
:1030100005EB450101EB8511114481F842000020C8
:1030200004EB440101EB8411114481F84100681C58
:10303000C5B200BF601CC4B20948007884429BDD61
:1030400007480078801B0649087000BF024948689D
:10305000804700BF6CE70000B80200207C3F0020E2
:10306000E1030020F80600207047000010B5144866
:10307000007800B910BD1349486D804738B912482F
:10308000807820B9012010498870F9F711FA0E48AC
:10309000C07800B9EEE70C488088401C80B20A492D
:1030A0008880C82802DA00F011F807E000200649FD
:1030B000C870888008460021C0F8061000BFD9E714
:1030C000EC030020380300204C62002010B588B0CB
:1030D0003648007810B13648C07810B9002008B0E2
:1030E00010BD1C208DF80000324881690DF10100EF
:1030F000884730208DF8050000208DF806008DF8F7
:10310000070014208DF8080004208DF80900132111
:103110000DF10A00F5F763F82548C07801283AD187
:10312000FF208DF806008DF80700214890F87F00F9
:103130001F4991F87E10884203DB00201C4981F86A
:103140007F001B4890F87F10801D10F821008DF83B
:103150000E00174890F87F10801D00EB810040782A
:103160008DF80F00124890F87F10801D00EB810051
:1031700080788DF810000E4890F87F10801D00EBCD
:103180008100C0788DF81100094890F87F00401C3C
:10319000074981F87F000749C86A80470446054807
:1031A0002146426B68469047012098E7EC030020D7
:1031B0004C6200203803002030B591B004460D4623
:1031C000402101A8F5F70BF83C208DF80400E12020
:1031D0008DF805000949C86980478DF806000E2062
:1031E0008DF807002A46214602A8F4F7D1FF0348CC
:1031F000416C01A8884711B030BD000038030020A1
:103200002DE9F04107464FF6FF783846FAF7C4FC3F
:103210000546124800782844C82806DC2A46394664
:103220000E48007800F044F914E00C480078C0F132
:10323000C800C6B2324639460848007800F038F96E
:10324000344605E00120A04028EA0008601CC4B212
:10325000AC42F7DB4046BDE8F08100002F050020BE
:103260002DE9F04106464FF6FF773046FAF794FC19
:1032700005461E2D00DD1E250F4880F87E500024D7
:1032800014E006EB8400FEF797FAB0F1000803D1D2
:103290000120A040874307E03046F9F71FF9AA2232
:1032A00004214046F4F794FF601C84B2AC42E8DB92
:1032B0003846BDE8F08100004C62002070B590B047
:1032C0000446207901280BD0022804D004281DD000
:1032D000052845D11FE06079A11D00F089F800BFE5
:1032E00060790DF1020100F05FF820B928210DF19D
:1032F0000200F4F774FF01208DF8000060798DF86A
:1033000001002A216846FFF757FF2AE0A01DFFF7BA
:1033100077FF054604E0A01DFFF7A2FF054600BFAA
:1033200002208DF80000C5F3090040F2FF31884209
:1033300001D1012000E000208DF80100002608E006
:1033400045FA06F000F00101B01C0DF80010701CE9
:10335000C6B20A2EF4DB0C216846FFF72DFF00E011
:1033600000BF00BF10B070BD00210B4A11700B4AA6
:103370001170002006E00A4901EB800100220A607A
:10338000411C88B2C828F6DB0021064AD170918022
:103390009170118070470000300500202F0500203B
:1033A0002C5F00204C6200202DE9F04106460F46BC
:1033B000142E02DB0020BDE8F0813046FBF7BCFC98
:1033C000054600240DE04FF6FF7000EA840807EB85
:1033D00008002919054A02EB810109680160601C97
:1033E00084B20A2CEFDB0120E5E700002C5F00200F
:1033F0002DE9F04104460E46142C02DB0020BDE806
:10340000F0811CB9FFF7B0FFF9F752F83046FAF730
:10341000C3FB05462046FBF78FFC07462A46F8B259
:10342000314600F045F80120E9E7000030B589B0E9
:1034300005461D480378C21C01A92846F5F7F0FE91
:10344000002409E001A8005D611C01AA515C48400C
:10345000611C5054601CC4B20F2CF3DB13481022C3
:1034600001A9036A900198470F480378C21C01A97B
:1034700005F11000F5F7D4FE002409E001A8005D75
:10348000611C01AA515C4840611C5054601CC4B2CC
:103490000F2CF3DB0548102201A9036A4FF4826068
:1034A000984709B030BD0000D44E0020B80200207B
:1034B00030B50346002009E01C18084D05EB8404D4
:1034C00001EB80052D682560441CA0B29042F3DB1F
:1034D000034C24781444024D2C7030BD2C5F002026
:1034E0002F05002000020000000400000000000082
:1034F0000006000006FFFF09FFA10109FF954075C6
:10350000081580257F810009FF95407508158025E5
:103510007F9100C000140140000C014000140140E4
:10352000001001400020100008004000001401407D
:103530000014014000140140001001400040200030
:10354000100080000E050407001401400014014023
:10355000001401400010014000084000020010006B
:10356000001401400014014000140140001001400B
:1035700000108000040020004053554E564F544523
:103580000053756E566F746531393938264A616358
:103590006B50656931393732436F6F6C426F6239F6
:1035A0003900104E1341144215431644174518466E
:1035B0001947204A304B404D9151925293539454A5
:1035C000A05AB05BC05C00000100000052096AD53F
:1035D0003036A538BF40A39E81F3D7FB7CE3398208
:1035E0009B2FFF87348E4344C4DEE9CB547B943257
:1035F000A6C2233DEE4C950B42FAC34E082EA1669F
:1036000028D924B2765BA2496D8BD12572F8F66475
:1036100086689816D4A45CCC5D65B6926C704850F0
:10362000FDEDB9DA5E154657A78D9D8490D8AB00A5
:103630008CBCD30AF7E45805B8B34506D02C1E8FCE
:10364000CA3F0F02C1AFBD0301138A6B3A9111410A
:103650004F67DCEA97F2CFCEF0B4E67396AC7422F3
:10366000E7AD3585E2F937E81C75DF6E47F11A7171
:103670001D29C5896FB7620EAA18BE1BFC563E4BAA
:10368000C6D279209ADBC0FE78CD5AF41FDDA8336C
:103690008807C731B11210592780EC5F60517FA9AC
:1036A00019B54A0D2DE57A9F93C99CEFA0E03B4DDB
:1036B000AE2AF5B0C8EBBB3C83539961172B047E4F
:1036C000BA77D626E169146355210C7D637C777B3C
:1036D000F26B6FC53001672BFED7AB76CA82C97D0E
:1036E000FA5947F0ADD4A2AF9CA472C0B7FD93269F
:1036F000363FF7CC34A5E5F171D8311504C723C3A3
:103700001896059A071280E2EB27B27509832C1AE6
:103710001B6E5AA0523BD6B329E32F8453D100ED40
:1037200020FCB15B6ACBBE394A4C58CFD0EFAAFB24
:10373000434D338545F9027F503C9FA851A3408FEC
:10374000929D38F5BCB6DA2110FFF3D2CD0C13EC04
:103750005F974417C4A77E3D645D197360814FDC99
:10376000222A908846EEB814DE5E0BDBE0323A0A7D
:103770004906245CC2D3AC629195E479E7C8376D01
:103780008DD54EA96C56F4EA657AAE08BA78252E26
:103790001CA6B4C6E8DD741F4BBD8B8A703EB566AF
:1037A0004803F60E613557B986C11D9EE1F89811A0
:1037B00069D98E949B1E87E9CE5528DF8CA1890D8F
:1037C000BFE6426841992D0FB054BB168D0102042B
:1037D00008102040801B366CD8AB4D9A2F5EBC631E
:1037E000C697356AD4B37DFAEFC5913972E4D3BD7B
:1037F00061C29F254A943366CC831D3A74E8CB8D11
:1038000001020408102040801B366CD8AB4D9A2F63
:103810005EBC63C697356AD4B37DFAEFC591397241
:10382000E4D3BD61C29F254A943366CC831D3A74AC
:10383000E8CB8D01020408102040801B366CD8AB09
:103840004D9A2F5EBC63C697356AD4B37DFAEFC537
:10385000913972E4D3BD61C29F254A943366CC830B
:103860001D3A74E8CB8D01020408102040801B36FD
:103870006CD8AB4D9A2F5EBC63C697356AD4B37DC6
:10388000FAEFC5913972E4D3BD61C29F254A9433E2
:1038900066CC831D3A74E8CB8D01020408102040E9
:1038A000801B366CD8AB4D9A2F5EBC63C697356AC9
:1038B000D4B37DFAEFC5913972E4D3BD61C29F25BF
:1038C0004A943366CC831D3A74E8CB3031323334BA
:1038D000353637383941424344454600000021100F
:1038E000422063308440A550C660E770088129916A
:1038F0004AA16BB18CC1ADD1CEE1EFF10000000067
:1039000009000000637C777BF26B6FC53001672B89
:10391000FED7AB76CA82C97DFA5947F0ADD4A2AFC3
:103920009CA472C0B7FD9326363FF7CC34A5E5F1D1
:1039300071D8311504C723C31896059A071280E27F
:10394000EB27B27509832C1A1B6E5AA0523BD6B3D3
:1039500029E32F8453D100ED20FCB15B6ACBBE3943
:103960004A4C58CFD0EFAAFB434D338545F9027F2F
:10397000503C9FA851A3408F929D38F5BCB6DA21E8
:1039800010FFF3D2CD0C13EC5F974417C4A77E3D14
:10399000645D197360814FDC222A908846EEB8146A
:1039A000DE5E0BDBE0323A0A4906245CC2D3AC622D
:1039B0009195E479E7C8376D8DD54EA96C56F4EA38
:1039C000657AAE08BA78252E1CA6B4C6E8DD741F49
:1039D0004BBD8B8A703EB5664803F60E613557B90C
:1039E00086C11D9EE1F8981169D98E949B1E87E9C6
:1039F000CE5528DF8CA1890DBFE6426841992D0F75
:103A0000B054BB1652096AD53036A538BF40A39EC4
:103A100081F3D7FB7CE339829B2FFF87348E4344AD
:103A2000C4DEE9CB547B9432A6C2233DEE4C950B09
:103A300042FAC34E082EA16628D924B2765BA24969
:103A40006D8BD12572F8F66486689816D4A45CCC88
:103A50005D65B6926C704850FDEDB9DA5E1546575B
:103A6000A78D9D8490D8AB008CBCD30AF7E4580591
:103A7000B8B34506D02C1E8FCA3F0F02C1AFBD039D
:103A800001138A6B3A9111414F67DCEA97F2CFCE6E
:103A9000F0B4E67396AC7422E7AD3585E2F937E809
:103AA0001C75DF6E47F11A711D29C5896FB7620E4B
:103AB000AA18BE1BFC563E4BC6D279209ADBC0FE2C
:103AC00078CD5AF41FDDA8338807C731B1121059D9
:103AD0002780EC5F60517FA919B54A0D2DE57A9FCB
:103AE00093C99CEFA0E03B4DAE2AF5B0C8EBBB3CC0
:103AF00083539961172B047EBA77D626E169146344
:103B000055210C7D000000010000000200000004AF
:103B1000000000080000001000000020000000402D
:103B2000000000800000001B00000036A56363C693
:103B3000847C7CF8997777EE8D7B7BF60DF2F2FF33
:103B4000BD6B6BD6B16F6FDE54C5C5915030306020
:103B500003010102A96767CE7D2B2B5619FEFEE7F4
:103B600062D7D7B5E6ABAB4D9A7676EC45CACA8F2D
:103B70009D82821F40C9C989877D7DFA15FAFAEFB7
:103B8000EB5959B2C947478E0BF0F0FBECADAD4194
:103B900067D4D4B3FDA2A25FEAAFAF45BF9C9C231C
:103BA000F7A4A453967272E45BC0C09BC2B7B7750A
:103BB0001CFDFDE1AE93933D6A26264C5A36366CC9
:103BC000413F3F7E02F7F7F54FCCCC835C3434683D
:103BD000F4A5A55134E5E5D108F1F1F9937171E24D
:103BE00073D8D8AB533131623F15152A0C04040841
:103BF00052C7C795652323465EC3C39D2818183056
:103C0000A19696370F05050AB59A9A2F0907070E50
:103C1000361212249B80801B3DE2E2DF26EBEBCDC7
:103C20006927274ECDB2B27F9F7575EA1B0909122D
:103C30009E83831D742C2C582E1A1A342D1B1B3670
:103C4000B26E6EDCEE5A5AB4FBA0A05BF65252A4E0
:103C50004D3B3B7661D6D6B7CEB3B37D7B29295297
:103C60003EE3E3DD712F2F5E97848413F55353A653
:103C700068D1D1B9000000002CEDEDC160202040DA
:103C80001FFCFCE3C8B1B179ED5B5BB6BE6A6AD4D8
:103C900046CBCB8DD9BEBE674B393972DE4A4A94CA
:103CA000D44C4C98E85858B04ACFCF856BD0D0BB95
:103CB0002AEFEFC5E5AAAA4F16FBFBEDC5434386E5
:103CC000D74D4D9A5533336694858511CF45458A36
:103CD00010F9F9E906020204817F7FFEF05050A03E
:103CE000443C3C78BA9F9F25E3A8A84BF35151A2CE
:103CF000FEA3A35DC04040808A8F8F05AD92923FA6
:103D0000BC9D9D214838387004F5F5F1DFBCBC63DB
:103D1000C1B6B67775DADAAF6321214230101020D0
:103D20001AFFFFE50EF3F3FD6DD2D2BF4CCDCD816E
:103D3000140C0C18351313262FECECC3E15F5FBE97
:103D4000A2979735CC4444883917172E57C4C4938B
:103D5000F2A7A755827E7EFC473D3D7AAC6464C8DD
:103D6000E75D5DBA2B191932957373E6A06060C0E8
:103D700098818119D14F4F9E7FDCDCA366222244BB
:103D80007E2A2A54AB90903B8388880BCA46468C87
:103D900029EEEEC7D3B8B86B3C14142879DEDEA741
:103DA000E25E5EBC1D0B0B1676DBDBAD3BE0E0DBC1
:103DB000563232644E3A3A741E0A0A14DB4949926A
:103DC0000A06060C6C242448E45C5CB85DC2C29F01
:103DD0006ED3D3BDEFACAC43A66262C4A891913957
:103DE000A495953137E4E4D38B7979F232E7E7D5BE
:103DF00043C8C88B5937376EB76D6DDA8C8D8D011E
:103E000064D5D5B1D24E4E9CE0A9A949B46C6CD80A
:103E1000FA5656AC07F4F4F325EAEACFAF6565CA63
:103E20008E7A7AF4E9AEAE4718080810D5BABA6FA0
:103E3000887878F06F25254A722E2E5C241C1C3859
:103E4000F1A6A657C7B4B47351C6C69723E8E8CB0A
:103E50007CDDDDA19C7474E8211F1F3EDD4B4B9679
:103E6000DCBDBD61868B8B0D858A8A0F907070E0FA
:103E7000423E3E7CC4B5B571AA6666CCD84848902F
:103E80000503030601F6F6F7120E0E1CA36161C2CC
:103E90005F35356AF95757AED0B9B969918686173B
:103EA00058C1C199271D1D3AB99E9E2738E1E1D915
:103EB00013F8F8EBB398982B33111122BB6969D230
:103EC00070D9D9A9898E8E07A7949433B69B9B2D60
:103ED000221E1E3C9287871520E9E9C949CECE876C
:103EE000FF5555AA782828507ADFDFA58F8C8C03E0
:103EF000F8A1A15980898909170D0D1ADABFBF658C
:103F000031E6E6D7C6424284B86868D0C3414182F0
:103F1000B0999929772D2D5A110F0F1ECBB0B07B78
:103F2000FC5454A8D6BBBB6D3A16162C50A7F451BE
:103F30005365417EC3A4171A965E273ACB6BAB3B01
:103F4000F1459D1FAB58FAAC9303E34B55FA302073
:103F5000F66D76AD9176CC88254C02F5FCD7E54F11
:103F6000D7CB2AC5804435268FA362B5495AB1DE26
:103F7000671BBA25980EEA45E1C0FE5D02752FC3A6
:103F800012F04C81A397468DC6F9D36BE75F8F0380
:103F9000959C9215EB7A6DBFDA5952952D83BED45C
:103FA000D32174582969E04944C8C98E6A89C27509
:103FB00078798EF46B3E5899DD71B927B64FE1BE22
:103FC00017AD88F066AC20C9B43ACE7D184ADF63DD
:103FD00082311AE560335197457F5362E07764B1CF
:103FE00084AE6BBB1CA081FE942B08F95868487006
:103FF00019FD458F876CDE94B7F87B5223D373ABE2
:10400000E2024B72578F1FE32AAB55660728EBB2CB
:1040100003C2B52F9A7BC586A50837D3F28728300F
:10402000B2A5BF23BA6A03025C8216ED2B1CCF8AAD
:1040300092B479A7F0F207F3A1E2694ECDF4DA6504
:10404000D5BE05061F6234D18AFEA6C49D532E3408
:10405000A055F3A232E18A0575EBF6A439EC830B87
:10406000AAEF6040069F715E51106EBDF98A213E35
:104070003D06DD96AE053EDD46BDE64DB58D54915F
:10408000055DC4716FD40604FF15506024FB9819B8
:1040900097E9BDD6CC434089779ED967BD42E8B049
:1040A000888B8907385B19E7DBEEC879470A7CA162
:1040B000E90F427CC91E84F8000000008386800955
:1040C00048ED2B32AC70111E4E725A6CFBFF0EFD88
:1040D0005638850F1ED5AE3D27392D3664D90F0AC7
:1040E00021A65C68D1545B9B3A2E3624B1670A0C3A
:1040F0000FE75793D296EEB49E919B1B4FC5C0809D
:10410000A220DC61694B775A161A121C0ABA93E294
:10411000E52AA0C043E0223C1D171B120B0D090E1F
:10412000ADC78BF2B9A8B62DC8A91E148519F157D1
:104130004C0775AFBBDD99EEFD607FA39F2601F7AD
:10414000BCF5725CC53B6644347EFB5B7629438BD1
:10415000DCC623CB68FCEDB663F1E4B8CADC31D72A
:1041600010856342402297132011C6847D244A851E
:10417000F83DBBD21132F9AE6DA129C74B2F9E1D60
:10418000F330B2DCEC52860DD0E3C1776C16B32B62
:1041900099B970A9FA4894112264E947C48CFCA823
:1041A0001A3FF0A0D82C7D56EF903322C74E498796
:1041B000C1D138D9FEA2CA8C360BD498CF81F5A6CE
:1041C00028DE7AA5268EB7DAA4BFAD3FE49D3A2C4F
:1041D0000D9278509BCC5F6A62467E54C2138DF676
:1041E000E8B8D8905EF7392EF5AFC382BE805D9FE8
:1041F0007C93D069A92DD56FB31225CF3B99ACC85C
:10420000A77D18106E639CE87BBB3BDB097826CD4D
:10421000F418596E01B79AECA89A4F83656E95E62B
:104220007EE6FFAA08CFBC21E6E815EFD99BE7BAE6
:10423000CE366F4AD4099FEAD67CB029AFB2A431FA
:1042400031233F2A3094A5C6C066A23537BC4E74D0
:10425000A6CA82FCB0D090E015D8A7334A9804F1E2
:10426000F7DAEC410E50CD7F2FF691178DD64D76B3
:104270004DB0EF43544DAACCDF0496E4E3B5D19E94
:104280001B886A4CB81F2CC17F51654604EA5E9DAD
:104290005D358C01737487FA2E410BFB5A1D67B391
:1042A00052D2DB92335610E91347D66D8C61D79A00
:1042B0007A0CA1378E14F859893C13EBEE27A9CE5E
:1042C00035C961B7EDE51CE13CB1477A59DFD29CB5
:1042D0003F73F25579CE1418BF37C773EACDF75341
:1042E0005BAAFD5F146F3DDF86DB447881F3AFCAC4
:1042F0003EC468B92C3424385F40A3C272C31D1673
:104300000C25E2BC8B493C2841950DFF7101A83971
:10431000DEB30C089CE4B4D890C156646184CB7BB6
:1043200070B632D5745C6C484257B8D00000C201F8
:10433000840346020807CA068C044E05100ED20FED
:10434000940D560C1809DA089C0A5E0B201CE21D1D
:10435000A41F661E281BEA1AAC186E193012F2133D
:10436000B41176103815FA14BC167E17403882390D
:10437000C43B063A483F8A3ECC3C0E3D503692370D
:10438000D435163458319A30DC321E336024A225DD
:10439000E42726266823AA22EC202E21702AB22B9D
:1043A000F4293628782DBA2CFC2E3E2F80704271CD
:1043B0000473C67288774A760C74CE75907E527FED
:1043C000147DD67C98795A781C7ADE7BA06C626D5D
:1043D000246FE66EA86B6A6A2C68EE69B06272633D
:1043E0003461F660B8657A643C66FE67C04802498D
:1043F000444B864AC84F0A4E4C4C8E4DD04612470D
:1044000054459644D8411A405C429E43E05422559C
:104410006457A656E8532A526C50AE51F05A325B9C
:104420007459B658F85D3A5C7C5EBE5F00E1C2E04C
:1044300084E246E308E6CAE78CE54EE410EFD2EEEC
:1044400094EC56ED18E8DAE99CEB5EEA20FDE2FC1C
:10445000A4FE66FF28FAEAFBACF96EF830F3F2F23C
:10446000B4F076F138F4FAF5BCF77EF640D982D88C
:10447000C4DA06DB48DE8ADFCCDD0EDC50D792D60C
:10448000D4D416D558D09AD1DCD31ED260C5A2C4DC
:10449000E4C626C768C2AAC3ECC12EC070CBB2CA9C
:1044A000F4C836C978CCBACDFCCF3ECE80914290CC
:1044B0000492C69388964A970C95CE94909F529EEC
:1044C000149CD69D98985A991C9BDE9AA08D628C5C
:1044D000248EE68FA88A6A8B2C89EE88B08372823C
:1044E0003480F681B8847A853C87FE86C0A902A80C
:1044F00044AA86ABC8AE0AAF4CAD8EACD0A712A60C
:1045000054A496A5D8A01AA15CA39EA2E0B522B49B
:1045100064B6A6B7E8B22AB36CB1AEB0F0BB32BA9B
:1045200074B8B6B9F8BC3ABD7CBFBEBE0000201C52
:10453000403860248070A06CC048E05400E120FD49
:1045400040D960C58091A08DC0A9E0B500040101EB
:10455000000000000000010004040101040001014A
:104560000404010004000000000001000004000039
:10457000000401010404010100040000040400011E
:104580000400010100000001040000000404000018
:104590000004000100040001000401000004010007
:1045A00000000101000001010404000104000100F9
:1045B00004000001040000010400010000000000EC
:1045C00004040000040401000000000100000100D8
:1045D00004040101040000000000010100040101C5
:1045E00000000001000000010004000004000101BF
:1045F00000000100000401000400000100040000AC
:10460000040000000404000104040100040401018A
:104610000400010000000101040400010400000185
:10462000040400000404010000040101040400006B
:10463000000400010004000100000000040001006B
:10464000000401000000000004000101208010802F
:10465000008000800080000020801000000010001A
:1046600020000000200010802080008020000080BA
:10467000208010800080108000000080008000807A
:1046800000001000200000002000108000801000BA
:10469000200010002080008000000000000000804A
:1046A000008000002080100000001080200010001A
:1046B000200000800000000000801000208000002A
:1046C00000801080000010802080000000000000AA
:1046D000208010002000108000001000208000804A
:1046E000000010800080108000800000000010801A
:1046F00000800080200000002080108020801000BA
:1047000020000000008000000000008020800000E9
:1047100000801080000010002000008020001000A9
:104720002080008020000080200010000080100009
:104730000000000000800080208000000000008059
:1047400020001080208010800080100008020000EF
:104750000002020800000000080002080002000831
:104760000000000008020200000200080800020029
:104770000800000808000008000002000802020803
:104780000800020000000208080200000000000803
:1047900008000000000202080002000000020200FF
:1047A00000000208080002080802020008020008CF
:1047B00000020200000002000802000808000000D9
:1047C00008020208000200000000000800020208BF
:1047D00000000008080002000802000000000200BB
:1047E00000020208000200080000000000020000B1
:1047F0000800020008020208000200080800000881
:104800000002000000000000080002080802000882
:104810000000020000000008080202080800000072
:10482000080202000002020008000008000002085E
:104830000802000808020000000002080802020046
:1048400008000000080002080002020001208000A9
:104850008120000081200000800000008020800076
:1048600081008000010080000120000000000000A5
:104870000020800000208000812080008100000056
:1048800000000000800080000100800001000000A6
:104890000020000000008000012080008000000057
:1048A00000008000012000008020000081008000C6
:1048B0000100000080200000800080000020000037
:1048C0008020800081208000810000008000800026
:1048D0000100800000208000812080008100000015
:1048E0000000000000000000002080008020000088
:1048F0008000800081008000010000000120800015
:1049000081200000812000008000000081208000C4
:104910008100000001000000002000000100800074
:104920000120000080208000810080000120000024
:104930008020000000008000012080008000000036
:1049400000008000002000008020800000010000A6
:1049500000010802000008020001004200000800F7
:1049600000010000000000400000080200010840B3
:1049700000000800000100020001084000010042A0
:104980000000084200010800000000400000000292
:104990000000084000000840000000000001004046
:1049A0000001084200010842000100020000084224
:1049B0000001004000000000000000420001080269
:1049C0000000000200000042000108000000080092
:1049D0000001004200010000000000020000004051
:1049E000000008020001004200010840000100022E
:1049F00000000040000008420001080200010840D9
:104A0000000100000000000200000842000108420E
:104A100000010800000000420001084200000802F6
:104A200000000000000008400000004200010800F3
:104A3000000100020001004000000800000000002A
:104A400000000840000108020001004010000020A2
:104A500000004020004000001040402000004020A6
:104A600010000000104040200000400000400020E6
:104A700010404000000040001000002010004000E6
:104A80000040002000000020104000000000000056
:104A90001000400010400020004000000040400096
:104AA00010400020100000001000402010004020A6
:104AB0000000000010404000004040201040000076
:104AC0000040400000404020000000200040002046
:104AD0001000000010004020004040001040402026
:104AE00000004000104000001000002000004000C6
:104AF00000400020000000201040000010000020B6
:104B00001040402000404000000040201040400085
:104B10000040402000000000100040201000000075
:104B20000040000000004020104040000040000015
:104B30001000400010400020000000000040402015
:104B40000000002010004000104000200000200065
:104B50000200200402080004000000000008000019
:104B600002080004020820000008200402082004B3
:104B7000000020000000000002000004020000000D
:104B800000000004020020040208000000080004E5
:104B900002082000020020000008000402000004B7
:104BA000000020040008200402002000000020046F
:104BB000000800000208000002082004000820008D
:104BC00002000000000000040008200000000004B3
:104BD0000008200000002000020800040208000471
:104BE0000200200402002004020000000200200055
:104BF0000000000400080004000020000008200459
:104C0000020800000208200000082004020800003A
:104C10000200000402082004000020040008200014
:104C20000000000002000000020820040000000054
:104C30000208200000002004000800000200000418
:104C400000080004000800000200200040100010CE
:104C500000100000000004004010041000000010CC
:104C60004010001040000000000000104000040050
:104C70000000041040100410001004000010041084
:104C8000401004000010000040000000000004106C
:104C90004000001000100010401000000010040040
:104CA00040000400400004100010041040100000F8
:104CB0000000000000000000400004104000001050
:104CC0000010001040100400000004004010040018
:104CD000000004000010041000100000400000005C
:104CE00040000410001000004010040000100010EC
:104CF00040000000400000100000041040000410BC
:104D0000000000100000040040100010000000002F
:104D10004010041040000400400000100000041087
:104D2000001000104010001000000000401004109F
:104D300000100400001004004010000040100000AB
:104D4000400004000000001000100410982F8A4258
:104D500091443771CFFBC0B5A5DBB5E95BC25639CD
:104D6000F111F159A4823F92D55E1CAB98AA07D8E5
:104D7000015B8312BE853124C37D0C55745DBE7208
:104D8000FEB1DE80A706DC9B74F19BC1C1699BE488
:104D90008647BEEFC69DC10FCCA10C246F2CE92D18
:104DA000AA84744ADCA9B05CDA88F97652513E983C
:104DB0006DC631A8C82703B0C77F59BFF30BE0C643
:104DC0004791A7D55163CA0667292914850AB727D1
:104DD00038211B2EFC6D2C4D130D385354730A656E
:104DE000BB0A6A762EC9C281852C7292A1E8BFA245
:104DF0004B661AA8708B4BC2A3516CC719E892D1AD
:104E0000240699D685350EF470A06A1016C1A4192F
:104E1000086C371E4C774827B5BCB034B30C1C392E
:104E20004AAAD84E4FCA9C5BF36F2E68EE828F74ED
:104E30006F63A5781478C8840802C78CFAFFBE9007
:104E4000EB6C50A4F7A3F9BEF27871C60000000025
:104E500022AE28D7982F8A42CD65EF23914437712F
:104E60002F3B4DECCFFBC0B5BCDB8981A5DBB5E9A1
:104E700038B548F35BC2563919D005B6F111F1596E
:104E80009B4F19AFA4823F9218816DDAD55E1CAB9F
:104E9000420203A398AA07D8BE6F7045015B831234
:104EA0008CB2E44EBE853124E2B4FFD5C37D0C55EF
:104EB0006F897BF2745DBE72B196163BFEB1DE80E7
:104EC0003512C725A706DC9B942669CF74F19BC1D8
:104ED000D24AF19EC1699BE4E3254F388647BEEF75
:104EE000B5D58C8BC69DC10F659CAC77CCA10C242D
:104EF00075022B596F2CE92D83E4A66EAA84744A9F
:104F0000D4FB41BDDCA9B05CB5531183DA88F976D6
:104F1000ABDF66EE52513E981032B42D6DC631A80B
:104F20003F21FB98C82703B0E40EEFBEC77F59BFEF
:104F3000C28FA83DF30BE0C625A70A934791A7D5DA
:104F40006F8203E05163CA06706E0E0A6729291446
:104F5000FC2FD246850AB72726C9265C38211B2E8E
:104F6000ED2AC45AFC6D2C4DDFB3959D130D3853BB
:104F7000DE63AF8B54730A65A8B2773CBB0A6A76CE
:104F8000E6AEED472EC9C2813B358214852C729264
:104F90006403F14CA1E8BFA2013042BC4B661AA8E1
:104FA0009197F8D0708B4BC230BE5406A3516CC79A
:104FB0001852EFD619E892D110A96555240699D652
:104FC0002A20715785350EF4B8D1BB3270A06A1013
:104FD000C8D0D2B816C1A41953AB4151086C371EC2
:104FE00099EB8EDF4C774827A8489BE1B5BCB034DD
:104FF000635AC9C5B30C1C39CB8A41E34AAAD84EBF
:1050000073E363774FCA9C5BA3B8B2D6F36F2E6885
:10501000FCB2EF5DEE828F74602F17436F63A5784B
:1050200072ABF0A11478C884EC39641A0802C78CFA
:10503000281E6323FAFFBE90E9BD82DEEB6C50A40C
:105040001579C6B2F7A3F9BE2B5372E3F27871C695
:105050009C6126EACE3E27CA07C2C021C7B886D1C6
:105060001EEBE0CDD67DDAEA78D16EEE7F4F7DF58E
:10507000BA6F1772AA67F006A698C8A2C57D630A20
:10508000AE0DF9BE04983F111B471C13350B711B65
:10509000847D0423F577DB289324C7407BABCA3299
:1050A000BCBEC9150ABE9E3C4C0D109CC4671D4376
:1050B000B6423ECBBED4C54C2A7E65FC9C297F59A6
:1050C000ECFAD63AAB6FCB5F1758474A8C19446C51
:1050D000657870616E642033322D62797465206B5F
:1050E000657870616E642031362D62797465206B4D
:1050F000EDD3F55C1A631258D69CF7A2DEF9DE14E4
:10510000000000000000000000000000000000108F
:105110001B132C0AA3E59CEDA72963085D2106213A
:10512000EBFFFFFFFFFFFFFFFFFFFFFFFFFFFFFFA3
:105130000F000000A3785913CA4DEB75ABD841415D
:105140004D0A700098E879777940C78C73FE6F2B11
:10515000EE6C03521AD5258F602D56C9B2A725953E
:1051600060C72C695CDCD6FD31E2A4C0FE536ECD75
:10517000D3366921586666666666666666666666E2
:1051800066666666666666666666666666666666BF
:105190006666666601000000000000000000000076
:1051A00000000000000000000000000000000000FF
:1051B00000000000A3DDB7A5B38ADE6DF55251777C
:1051C000809FF0207DE3AB648E4EEA6665768BD7D8
:1051D0000F5F876759F1B226949BD6EB56B1838255
:1051E0009A14E00030D1F3EEF2808E19E7FCDF561E
:1051F000DCD90624B0A00E4A271BEEC478E42FADFC
:105200000618432FA7D7FB3D99004D2B0BDFC14F4D
:105210008024832B80004000200010000800040040
:10522000020001000000800000004000000020009B
:105230000000100000000800000004000000020050
:10524000000001000080000000400000002000007D
:105250000010000000080000000400000002000030
:10526000000100008000000040000000200000005D
:105270001000000008000000040000000200000010
:10528000010000008000000000000000000000009D
:10529000000000000000000000000000000000000E
:1052A00000000000000000000000000000000000FE
:1052B00000000000000000000000000000000000EE
:1052C00000000000000000000000000000000000DE
:1052D000000000006363636263636362636363622D
:1052E00063636362C998989BAAFBFBF9C998989B72
:1052F000AAFBFBF950349790FACF6C693357F4F25C
:1053000099AC0F0B7BDA06EE81156A87B2429E7567
:105310002BEE917E882B2E7F093E44F8BB7CDA8DE4
:1053200090924BF3854B61EC8C7525143709FF99EE
:10533000A79BB46A871775210B6250353C6BAFACE5
:105340009BF01BC63303F90E3861A93B040A06978C
:105350009FFA1D51E2D8D4B1DAB97D8ADEB37B1D44
:105360004149664CCB5BEFB411E2923ECF51E92349
:105370008E188F6F03020100070605040B0A090847
:105380000F0E0D0CFD74AAD6FA72AFD2F178A6DA20
:10539000FE76ABD60BCF92B6F1BD3D6400C59BBE89
:1053A000FEB330684E74FFB6BFC9C2D2BF0C596C91
:1053B00041BF6904BCF7F747033E3595BC326CF931
:1053C000FD8D05FDE8A3AA3CEB9D9FA957AFF350C7
:1053D000AA22F6AD7D0F395E9692A6F7C13D55A77C
:1053E0006B1FA30A1A70F9148CE25FE34DDF0A44C5
:1053F00026C0A94E35874347B9651CA4F4BA16E008
:10540000D27ABFAED1329954685785F09CED931093
:105410004E972CBE7F1D1113174A94E38BA707F3F9
:10542000C5302B4D0000000000000000010000000E
:10543000FFFFFFFF01000000FFFFFFFF0000000073
:10544000000000000000000000000000000000005C
:105450000100000000000000010000000100000049
:10546000010000000A0A0A0A0A2A2A2A2A2A2A2AE3
:105470002A2A2A2A2A2A2A2A2A2A2A2A2A2A2A2A8C
:105480002A2A2A2A2A2044617461706F733D256498
:10549000202A2A2A2A2A2A2A2A2A2A2A2A2A2A2A76
:1054A0002A2A2A2A2A2A2A2A2A2A2A2A2A2A2A0A7C
:1054B00000000000D454010800000020F80500009E
:1054C00044820008C4570108F805002018B80000FD
:1054D0001AB80008132FF21408CDF99208840E2789
:1054E000071ED11F0108F9041E112001089D08188C
:1054F0000A092B0108B12A0108CD04180B5D22010D
:105500000879230108492124190C1AD5241A3504D5
:105510001FD1260108F1251C3B27015413CDBF14D0
:1055200008C5BD140895C04C0873C1081A9B041324
:105530007DBE1B086D101A41081AC9101A8D281A51
:10554000E3101B13C22812BC1B0853041A190C4188
:1055500013120132021640702F10EA1009020102E4
:10556000030109022913010125C032090433020392
:105570001509211101140122201607058103402D70
:10558000010705010710080403090410035312550D
:10559000124E1256124F1254027345140C0343124A
:1055A000311A300202774203831A0322DF1B20E301
:1055B000041365011B20E7041AA40C1AB604411356
:1055C0006C023320FF130DDE1408F1DD1B08B9084F
:1055D000811AA5101AA904B94C128F1408CDA3146E
:1055E00008DD9E14080D93140881D9140821EE14C7
:1055F00008F5921B086108138D911B084504780C6F
:10560000A514010879170108ED1601401A050C1AB6
:105610003D1481136DF91B089D04411399C31B08A8
:10562000B54C01148BB11D341B99EC3412CB1B0803
:10563000C5041A670413E1CA1B0865081BE9EB14CB
:1056400019041AD1041EC90C0108DD08132DED1B25
:105650000879941AF1741309D01B08253C1385F8B6
:105660001C08EDD428190C1EC10B010831081AF5CD
:10567000281A01281A0D04811A755401444BA5E912
:1056800048180A69330108BD320108B98C1A79B487
:105690001B3DF574311B89E6081AE7101AE8A019BA
:1056A000041ABD0C1A3108291C180A151E0108011C
:1056B0001F010899341A110C1A030C29181B09D858
:1056C000C412D71B08D9044B09D92C130DC51408D3
:1056D00069FC14086DFB1408D264340401502AFFDD
:1056E0001A311907E32902132DC21C08350C901931
:1056F000081A6104100B09130108CD11010895EB7C
:105700001B08A9040110294A1AC96C100B511A016F
:1057100008F10B0108C1E01F089D2B010847041A7E
:1057200049041A4B042A450412BB1408A1FE1F08A1
:105730001D02010805041B0103BC19081A11081EEB
:10574000D9010108C90C1AF9081AE908011259B05F
:10575000012F323C233F12280D4331303042414269
:1057600043444546474BF264136C052A2004811AD2
:10577000DBAC13B1E31408B5EC140869E11B083580
:10578000048B19DDFC52805951E03A48494A4B4C90
:105790004D4E4F505152535455565758595A6162B5
:1057A000636465666768696A6B6C6D6E6F70717251
:1057B000737475767778797A303132333435363799
:0457C00038392B2F1A
:04000005080081313D
:00000001FF
